:100000000C94B1470C94D2470C9457D10C94D2471E
:100010000C94D2470C94D2470C94D2470C94D247FC
:100020000C94D2470C94D2470C94D2470C9482D3B0
:100030000C94D2470C94D2470C948CB50C94D247B4
:100040000C94D2470C94D2470C94D2470C94D247CC
:100050000C94D2470C94D2470C94D2470C94D247BC
:100060000C94D2470C9471D10C9400D10C94D247CB
:100070000C94D7CA0C9479CA0C94B5CA0C94D24784
:100080000C9422D20C94D2470C94D2470C94D247B1
:100090000C94D2470C94D2470C94D2470C94D2477C
:1000A0000C94D2470C94D2470C94D2470C9465BC64
:1000B0000C9409BD0C94D2470C94D2470C947DB794
:1000C0000C94D2470C94D2470C94D2470C94D2474C
:1000D0000C94D2470C94D2470C94D2470C94D2473C
:1000E0000C9425A70C94D2470C94D2470C94D24779
:1000F0000C94D2470C94D2470C94D2470C94D2471C
:100100000C943CBC0C94E0BC0C9413BC0C94B7BC99
:100110000C94D2470C94D2470C94D2470C94D247FB
:100120000C94D2470C94D2470C94D2470C94D247EB
:100130000C94D2470C94E1B60C94D2470C94D2475D
:100140000C94D2470C94D2470C94D2470C94D247CB
:100150000C94D2470C94D2470C941BA70C94D24712
:100160000C94D2470C94D2470C94D2470C94D247AB
:100170000C94D2470C94D2470C94D2470C94D2479B
:100180000C94D2470C94D2470C94D2470C94D2478B
:100190000C94D2470C94D2470C94D2470C94D2477B
:1001A0000C948EBC0C9432BD0C94D2470C94D24764
:1001B0000C942FB70C94D2470C94D2470C94D2478E
:1001C0000C94D2470C94D2470C94D2470C94D2474B
:1001D0000C94D2470C94D2470C94D2470C94D2473B
:1001E0000C94D2470C94D247D071DA71E471EE715D
:1001F000F971FF77FF77FF77FF77FF77FF71FF7761
:10020000FF77FF77FF77FF77FF7701720B72157229
:100210001F722972FF77FF77FF77FF77FF77FF77EE
:100220003372FF778972FF77FF77FF77FF77FF776A
:10023000FF77FF77C872FF77E475FF77FF77FF7767
:10024000FF77FF77FF77FF77FF77E475FF77FF771B
:10025000FF77F572FA7204730E7310731A732573B5
:10026000FF773073FF77FF776D73FF77FF77FF7747
:10027000FF77FF77FF77FF77FF77FF77FF77FF77CE
:10028000FF77FF77FF77FF777773FF77FF77FF774A
:10029000FF77FF77FF77FF77FF77FF778173BE7375
:1002A000FB7344744E746774677471747B748574E3
:1002B0008F7499749E74A874B274FD77FD77FD777E
:1002C000FD77FD77FD77FD77FD77FD77FD77FD778E
:1002D000FD77FD77FD77FD77FD77FD77FD77FD777E
:1002E000FD777174FD77FD77FD77FD77FD77FD77FD
:1002F000FD77FD77FD77FD77FD77FD77FD77FD775E
:10030000FD77FD77FD77BC74C674D074DA74FD7721
:10031000FD77FD77FD77FD77FD77FD77FD776774D6
:100320008A7749774D775577317735773D774177BC
:10033000617776777E7782778677E277597755751A
:1003400066757775FF77FF77EF74C171FF778875F2
:100350009975AA75E4755874CC75FF770075FF77A9
:10036000BB751175E474FF77FF77FF7722753375DE
:100370004475ACBBB4BBBCBBC4BBCCBBD4BBDCBB4B
:10038000E4BBC4BE28BE30BE38BE40BE48BE50BE70
:1003900058BE60BE68BE70BE78BE80BE88BE90BECD
:1003A000A8BEA8BEA8BEA8BEA8BEA8BEA8BEA8BE1D
:1003B000A8BEA8BEA8BEA8BEA8BEA8BEA8BEA8BE0D
:1003C000A8BEA8BEA8BEA8BEA8BEA8BEA8BEA8BEFD
:1003D000A8BEA8BEA8BEA8BEA8BEA8BEA8BEA8BEED
:1003E000A8BEA8BEA8BE98BEA0BE084AD73B3BCEBA
:1003F000016E84BCBFFDC12F3D6C74319ABD568324
:100400003DDA3D00C77F11BED9E4BB4C3E916BAADB
:10041000AABE000000803F05A84CCDB2D44EB9382A
:1004200036A9020C50B9918688083CA6AAAA2ABE11
:10043000000000803F07634236B79BD8A71A39688F
:100440005618AEBAAB558C1D3CB7CC5763BD6DED9D
:10045000FD753EF6177231BF000000803F080000B6
:1004600000BE922449123EABAAAA2ABECDCCCC4CE7
:100470003E00000080BEABAAAAAA3E00000000BF5A
:10048000000000803F0000000000084178D3BB431B
:1004900087D1133D190E3CC3BD4282AD2B3E68ECA3
:1004A0008276BED98FE1A93E4C80EFFFBE01C4FF2A
:1004B0007F3F0000000000000C9449770C94E4BBDF
:1004C0000C94386F0C9472A80C94FEBD0C941A73A3
:1004D0000C9457BB0C94D9680C94E7630C9488BEB9
:1004E0000C94BF640C94BB790C9435770C945F68C2
:1004F0000C947B740C947EA80C94D0740C94B379F7
:100500000C946D6E0C94E75A0C9433720C945577DE
:100510000C94915E0C94E15B0C9476770C9401AD95
:100520000C944C5A0C94E4AF0C9461570C946B5A95
:100530000C94A7BA0C9401720C944D770C94F1C1F1
:100540000C94A15D0C94F9BA0C9427630C94E847C1
:100550000C948B5F0C948F740C94886E0C94DE4713
:100560000C9461770C9474570C94204F0C947A5E21
:100570000C94F35A0C94C1570C949E740C94D44769
:100580000C9481930C9476A80C94BCBB0C9449AE4B
:100590000C940EC70C9466750C9480CD0C94417825
:1005A0000C948E680C94415D0C94D0710C94B4BB87
:1005B0000C9448BE0C9460BE0C9480BE0C94AA5E51
:1005C0000C9472BB0C9470BE0C94DCC00C947773CA
:1005D0000C94FA720C9492630C94F6590C94D75ABA
:1005E0000C9404730C94B2740C948F7A0C949667E8
:1005F0000C94EB630C94E35A0C94CD5B0C940B724B
:100600000C94AA750C94AE6B0C9486570C94E24E25
:100610000C9405AD0C9404BE0C940F5B0C94C95B58
:100620000C94075B0C94A2570C94734B0C94DF5AF8
:100630000C9472590C940E730C94EF5A0C94C55B85
:100640000C9422750C9433580C9440BE0C947A5739
:100650000C9456810C9414CA0C94765E0C94EE683B
:100660000C94A8740C9430730C9431770C9484AE71
:100670000C94F75A0C9444740C94ECCC0C9455756F
:100680000C9433750C9477750C948A770C9438BE5F
:100690000C94785B0C9497BA0C94CB5E0C94A8BE27
:1006A0000C94F3630C9408BA0C94FB730C94C6740A
:1006B0000C94AB570C94BB750C940B5B0C948C573F
:1006C0000C94C1710C94C6540C9482A80C94035BD6
:1006D0000C9499750C9427480C9450BE0C94DAAC89
:1006E0000C94265A0C94D7570C94B7790C944ABBA7
:1006F0000C94F5720C948AA80C9470AE0C94F97159
:100700000C9461690C9427C90C94C8720C9428BE8F
:100710000C9467740C9426640C945A640C94095CD1
:100720000C9426CA0C945E810C940B5F0C94F2829C
:100730000C94FD5B0C9490BE0C942CC10C94B66B85
:100740000C94FB570C9414BA0C9488C10C949F64BD
:100750000C94647A0C945DA90C94F95B0C94115A76
:100760000C947AA80C9488750C94DA740C94145C2C
:100770000C94FA790C94CB5A0C94ECCD0C945178DF
:100780000C94FB590C9486A80C94D15B0C9499742E
:100790000C94555B0C9485740C942B5F0C94384826
:1007A0000C9458BE0C946EA80C9425730C946EBBDC
:1007B0000C946AA80C945CAE0C94E4710C946A5886
:1007C0000C94397A0C9418810C94FD770C94447530
:1007D0000C9452BB0C949D5D0C94E4750C94E95BF5
:1007E0000C94B5C90C943D5E0C94164F0C94FD58B6
:1007F0000C94785E0C94AC680C945AC10C9498BE1E
:100800000C94EE710C9489720C94E55B0C948277D5
:100810000C94BC740C94D35A0C94525F0C94C9C6BB
:100820000C9459770C94DCBB0C94F1CE0C9415729B
:100830000C94F46E0C94DF640C9455CF0C9471748A
:100840000C94DA710C94E4740C9486770C94D6AC06
:100850000C94185A0C941CBB0C9475CE0C94A0D01C
:100860000C948F790C94165E0C94D4BB0C943ECEF1
:100870000C94C4BB0C94EF740C94C85D0C941ABE19
:100880000C94CC570C94D8AC0C941F5A0C94EB5E7F
:100890000C946ABB0C94ACBB0C94175B0C94746402
:1008A0000C94FFAC0C942D5A0C948EA80C94ED5B18
:1008B0000C9494580C94C75A0C94F15B0C94CC751E
:1008C0000C946D730C9466BB0C9449630C94AF79D3
:1008D0000C94DB5A0C94E2770C94EF5D0C9488AE88
:1008E0000C94FB5A0C9481730C945A810C9480578D
:1008F0000C9497570C947E770C9458740C94107346
:100900000C94CCBB0C94FF770C94D55B0C94417782
:100910000C94114F0C94CD580C9430BE0C946E571F
:100920000C94BE730C948A6D0C94BBAF0C94EB5A70
:100930000C9400750C9420BA0C9437790C94C4BEB6
:100940000C9419680C9494C90C943D770C94EF6343
:100950000C948A790C941ACC0C94DD5B0C94365B65
:100960000C94CF5A0C944C850C94F44E0C941B4F61
:100970000C940A590C944E740C948CAE0C94FF5A3F
:100980000C941F720C94BD5B0C9490AE0C94D95BCC
:100990000C94135B0C9478BE0C94E3630C94B657E0
:1009A0000C9423610C9416BE0C944EBB0C94A0BE08
:1009B0000C94595B0C94C15B0C94BF790C94F55B5F
:1009C0000C9429720C94EA570C9440640C9468BE01
:1009D0000C94CA590C94BFBA0C9411750C94FF7105
:1009E0005B257325735D20257320257320706F733D
:1009F0006974696F6E2531382E336625730A005B82
:100A0000257325735D202573202573206F6666731B
:100A100065742532302E336625730A005B257325F5
:100A2000735D202573207A65726F206261636B6F3E
:100A300066662531392E336625730A005B257325DA
:100A4000735D202573206C61746368206261636B41
:100A50006F66662531382E336625730A005B257371
:100A600025735D202573206C617463682076656C46
:100A70006F636974792531332E306625732F6D6964
:100A80006E0A005B257325735D20257320736561F5
:100A90007263682076656C6F636974792531322ED4
:100AA000306625732F6D696E0A005B257325735DB3
:100AB00020257320737769746368206D6178253110
:100AC0003764205B303D6F66662C313D686F6D6921
:100AD0006E672C323D6C696D69742C333D6C696DA9
:100AE00069742B686F6D696E675D0A005B257325FD
:100AF000735D20257320737769746368206D696E58
:100B000025313764205B303D6F66662C313D686F60
:100B10006D696E672C323D6C696D69742C333D6C68
:100B2000696D69742B686F6D696E675D0A005B257E
:100B30007325735D20257320726164697573207657
:100B4000616C75652532302E346625730A005B258D
:100B50007325735D202573206A756E6374696F6EEB
:100B600020646576696174696F6E2531342E346650
:100B7000257320286C617267657220697320666135
:100B800073746572290A005B257325735D202573D4
:100B9000206A65726B20686F6D696E672531362E2D
:100BA000306625732F6D696E5E33202A2031206DEB
:100BB000696C6C696F6E0A005B257325735D202577
:100BC00073206A65726B206D6178696D756D253172
:100BD000352E306625732F6D696E5E33202A2031E5
:100BE000206D696C6C696F6E0A005B257325735DFF
:100BF0002025732074726176656C206D696E696D55
:100C0000756D2531372E336625730A005B257325F4
:100C1000735D2025732074726176656C206D617838
:100C2000696D756D2531372E336625730A005B2596
:100C30007325735D2025732076656C6F6369747905
:100C4000206D6178696D756D2531312E30662573A3
:100C50002F6D696E0A005B257325735D2025732057
:100C60006665656472617465206D6178696D756D26
:100C70002531312E306625732F6D696E0A005B2594
:100C80007325735D2025732061786973206D6F640F
:100C900065253138642025730A005B6D615D202075
:100CA0006D696E20617263207365676D656E742572
:100CB00031382E336625730A005B736C5D20207318
:100CC0006F6674206C696D697420656E61626C6515
:100CD000253132640A005B63745D202063686F72A3
:100CE00064616C20746F6C6572616E636525313769
:100CF0002E346625730A005B6A615D20206A756E7A
:100D00006374696F6E20616363656C657261746999
:100D10006F6E25382E306625730A005B6764695D47
:100D20002064656661756C742067636F6465206418
:100D3000697374616E6365206D6F6465253264202C
:100D40005B303D4739302C313D4739315D0A005B1E
:100D50006770615D2064656661756C742067636FA0
:100D60006465207061746820636F6E74726F6C25A7
:100D70003364205B303D4736312C313D4736312ED0
:100D8000312C323D4736345D0A005B67636F5D206E
:100D900064656661756C742067636F646520636F5A
:100DA0006F72642073797374656D253364205B31D1
:100DB0002D3620284735342D473539295D0A005B0B
:100DC00067756E5D2064656661756C742067636F1E
:100DD000646520756E697473206D6F646525356474
:100DE000205B303D4732302C313D4732315D0A00C7
:100DF0005B67706C5D2064656661756C7420676309
:100E00006F646520706C616E6525313064205B30E5
:100E10003D4731372C313D4731382C323D47313950
:100E20005D0A00256320776F726B206F66667365BD
:100E3000743A2531322E336625730A002563206DFE
:100E4000616368696E6520706F736E3A2531312E6B
:100E5000336625730A00256320706F736974696FA8
:100E60006E3A2531352E336625730A00546F6F6C48
:100E7000206E756D626572202020202020202020A9
:100E80002025640A00466565642072617465206DE2
:100E90006F64653A20202020202025730A004469D1
:100EA0007374616E6365206D6F64653A2020202045
:100EB00020202025730A0050617468204D6F6465FE
:100EC0003A202020202020202020202025730A00E6
:100ED000506C616E653A20202020202020202020A8
:100EE000202020202025730A004D6F74696F6E202A
:100EF0006D6F64653A20202020202020202025735B
:100F00000A00436F6F7264696E6174652073797350
:100F100074656D3A20202025730A00556E6974733C
:100F20003A202020202020202020202020202020A7
:100F300025730A00486F6D696E672073746174656C
:100F40003A202020202020202025730A00466565B5
:100F500064686F6C642073746174653A202020208B
:100F6000202025730A004D6F74696F6E20737461C1
:100F700074653A202020202020202025730A004379
:100F800079636C652073746174653A202020202099
:100F90002020202025730A00526177206D6163684C
:100FA000696E652073746174653A20202025730A88
:100FB000004D616368696E652073746174653A20E1
:100FC00020202020202025730A004C696E65206EA9
:100FD000756D6265723A2531306C750A004665653B
:100FE0006420726174653A2531362E336625732F7D
:100FF0006D696E0A0056656C6F636974793A2531C4
:10100000372E336625732F6D696E0A006310321018
:101010001210473935202D20756E6974732D706557
:10102000722D7265766F6C7574696F6E206D6F646A
:101030006500473934202D20756E6974732D7065F5
:10104000722D6D696E757465206D6F6465202869F9
:101050002E652E206665656472617465206D6F640F
:10106000652900473933202D20696E7665727365D6
:101070002074696D65206D6F6465009F107F104757
:101080003931202D20696E6372656D656E74616CF7
:101090002064697374616E6365206D6F64650047D9
:1010A0003930202D206162736F6C7574652064691E
:1010B0007374616E6365206D6F646500F010D81005
:1010C000C210473634202D20636F6E74696E756FC1
:1010D0007573206D6F6465004736312E31202D20E9
:1010E00065786163742073746F70206D6F64650040
:1010F000473631202D2065786163742070617468F3
:10110000206D6F6465002A111B110C1147313920C5
:101110002D20595A20706C616E6500473138202DA2
:1011200020585A20706C616E6500473137202D20A1
:10113000585920706C616E6500B611A4118B116A4C
:10114000114311473830202D2063616E63656C2098
:101150006D6F74696F6E206D6F646520286E6F6EA1
:1011600065206163746976652900473320202D204E
:10117000636F756E74657220636C6F636B776973F0
:101180006520617263206665656400473220202D0A
:1011900020636C6F636B776973652061726320668F
:1011A00065656400473120202D206C696E65617291
:1011B000206665656400473020202D206C696E65CF
:1011C000617220747261766572736520287365653B
:1011D0006B29007D12631249122F121512FB11E1C7
:1011E00011473539202D20636F6F7264696E617409
:1011F000652073797374656D203600473538202D6E
:1012000020636F6F7264696E6174652073797374A3
:10121000656D203500473537202D20636F6F726470
:10122000696E6174652073797374656D203400474D
:101230003536202D20636F6F7264696E617465208E
:1012400073797374656D203300473535202D206325
:101250006F6F7264696E6174652073797374656D04
:10126000203200473534202D20636F6F7264696E21
:101270006174652073797374656D2031004735336F
:10128000202D206D616368696E6520636F6F7264E5
:10129000696E6174652073797374656D00B012AA0C
:1012A00012A312486F6D696E6700486F6D65640028
:1012B0004E6F7420486F6D656400E412DF12DA121D
:1012C000D412CF12C612456E6420486F6C64004879
:1012D0006F6C6400446563656C00506C616E005314
:1012E000796E63004F666600F712F312EE12486FD4
:1012F0006C640052756E0053746F700021131713E5
:1013000011130A1306134A6F6700486F6D696E6701
:101310000050726F6265004D616368696E696E6747
:10132000004F666600571351134B13461342133C8C
:1013300013331353687574646F776E004379636C6D
:101340006500456E640053746F7000416C61726D8E
:1013500000526561647900496E697469616C697AEB
:10136000696E6700BA13B413AE13A913A513A113C2
:101370009C1396139013891385137C13536875740B
:10138000646F776E004A6F6700486F6D696E670023
:101390004379636C650050726F626500486F6C64DE
:1013A0000052756E00456E640053746F7000416C9E
:1013B00061726D00526561647900496E697469619A
:1013C0006C697A696E6700E113CB13473231202DC7
:1013D000206D696C6C696D65746572206D6F6465F4
:1013E00000473230202D20696E63686573206D6F71
:1013F0006465001B1410140414FB135B72616469B0
:1014000075735D005B696E686962697465645D002F
:101410005B7374616E646172645D005B64697361C7
:10142000626C65645D00351431142C1420646567AA
:1014300000206D6D0020696E002A2A2A204E4F542C
:10144000494345202A2A2A20526573657474696EBF
:10145000672062617564207261746520746F202555
:1014600073005B626175645D205553422062617553
:1014700064207261746525313564205B313D3936F5
:1014800030302C323D31393230302C333D3338342A
:1014900030302C343D35373630302C353D31313518
:1014A0003230302C363D3233303430305D0A005B20
:1014B00072786D5D2073657269616C205258206D81
:1014C0006F646525313564205B303D636861725F10
:1014D0006D6F64652C313D6C696E655F6D6F646521
:1014E0005D0A005B65785D2020656E61626C652039
:1014F000666C6F7720636F6E74726F6C2531306429
:10150000205B303D6F66662C313D584F4E2F584F53
:1015100046462C323D5254532F4354535D0A005BD0
:1015200065655D2020656E61626C65206563686F2E
:1015300025313864205B303D6F66662C313D6F6E1F
:101540005D0A005B65635D2020657870616E6420D4
:101550004C4620746F2043524C46206F6E205458E6
:10156000253664205B303D6F66662C313D6F6E5DC5
:101570000A00A515A0159A1594158E1587158015C6
:10158000323330343030003131353230300035379D
:1015900036303000333834303000313932303000BA
:1015A0003936303000300073797300666200000015
:1015B000001702AF793D5E765E6A3E3333DC4373DB
:1015C0007973006676000000001703B3793D5E76FC
:1015D0005E6E3EEC51783F737973006870000000D6
:1015E000000700B779EF5D7A5E723E0000803F73BE
:1015F0007973006876000000001700BB793D5E8FAC
:1016000079733E0000004173797300696400000043
:10161000000400BF793779765E663E000000000066
:101620000000006E00000000000000C75AEF5DAA35
:101630005EE13600000000000000006C696E65008D
:10164000000000C75AEA57AA5EE136000000000019
:1016500000000076656C00000010022D5AFB5776E2
:101660005E663E00000000000000006665656400E4
:101670000010024C5A3358765E663E0000000000AF
:101680000000007374617400000000CB5A6157764B
:101690005E663E00000000000000006D61637300A4
:1016A000000000CF5A6E57765E663E0000000000D4
:1016B0000000006379637300000000D35A7457760A
:1016C0005E663E00000000000000006D6F74730055
:1016D000000000D75A7A57765E663E000000000090
:1016E000000000686F6C6400000000DB5A805776D1
:1016F0005E663E0000000000000000756E69740028
:10170000000000E35A8C57765E663E000000000041
:10171000000000636F6F7200000000E75A97577671
:101720005E663E00000000000000006D6F6D6F00FF
:10173000000000EB5AA257765E663E0000000000F3
:10174000000000706C616E00000000EF5AAB57762D
:101750005E663E00000000000000007061746800DA
:10176000000000F35AB657765E663E0000000000A7
:101770000000006469737400000000F75AC15776D6
:101780005E663E000000000000000066726D6F00A3
:10179000000000FB5ACC57765E663E000000000059
:1017A000000000746F6F6C00000000FF5AD757767E
:1017B0005E663E000000006D706F006D706F780017
:1017C000001003095C9458765E663E000000006DD0
:1017D000706F006D706F7900001003095C9458768B
:1017E0005E663E000000006D706F006D706F7A00E5
:1017F000001003095C9458765E663E000000006DA0
:10180000706F006D706F6100001003095C94587672
:101810005E663E000000006D706F006D706F6200CC
:10182000001003095C9458765E663E000000006D6F
:10183000706F006D706F6300001003095C94587640
:101840005E663E00000000706F7300706F7378007A
:10185000001003FD5B6A58765E663E000000007073
:101860006F7300706F737900001003FD5B6A587628
:101870005E663E00000000706F7300706F737A0048
:10188000001003FD5B6A58765E663E000000007043
:101890006F7300706F736100001003FD5B6A587610
:1018A0005E663E00000000706F7300706F73620030
:1018B000001003FD5B6A58765E663E000000007013
:1018C0006F7300706F736300001003FD5B6A5876DE
:1018D0005E663E000000006F6673006F66737800FE
:1018E000001003145CCD58765E663E000000006F69
:1018F0006673006F66737900001003145CCD587630
:101900005E663E000000006F6673006F66737A00CB
:10191000001003145CCD58765E663E000000006F38
:101920006673006F66736100001003145CCD587617
:101930005E663E000000006F6673006F66736200B3
:10194000001003145CCD58765E663E000000006F08
:101950006673006F66736300001003145CCD5876E5
:101960005E663E00000000686F6D00686F6D650088
:10197000000000DF5A8657FB59663E0000000068F1
:101980006F6D00686F6D7800001000FD5BA15D76E3
:101990005EB63600000000686F6D00686F6D7900FC
:1019A000001000FD5BA15D765EB7360000000068A8
:1019B0006F6D00686F6D7A00001000FD5BA15D76B1
:1019C0005EB83600000000686F6D00686F6D6100E2
:1019D000001000FD5BA15D765EB936000000006876
:1019E0006F6D00686F6D6200001000FD5BA15D7699
:1019F0005EBA3600000000686F6D00686F6D6300AE
:101A0000001000FD5BA15D765EBB3600000000703B
:101A10007262007072626500000000DCC0A15D7639
:101A20005EBC360000000070726200707262780066
:101A3000001003DCC03D5E765EBD36000000007025
:101A40007262007072627900001003DCC03D5E7645
:101A50005EC13600000000707262007072627A002F
:101A6000001003DCC03D5E765EC5360000000070ED
:101A70007262007072626100001003DCC03D5E762D
:101A80005EC936000000007072620070726262000F
:101A9000001003DCC03D5E765ECD360000000070B5
:101AA0007262007072626300001003DCC03D5E76FB
:101AB0005ED136000000006A6F67006A6F677800C9
:101AC000001000DCC09D5D115ADB36000000006A8A
:101AD0006F67006A6F677900001000DCC09D5D18B9
:101AE0005ADB36000000006A6F67006A6F677A0091
:101AF000001000DCC09D5D1F5ADB36000000006A4C
:101B00006F67006A6F676100001000DCC09D5D2692
:101B10005ADB360000000070777200707772310077
:101B200000000072BBA7BA765E663E00000000703F
:101B3000777200707772320000000072BBA7BA762D
:101B40005E663E00000000707772007077723300AE
:101B500000000072BBA7BA765E663E00000000700F
:101B6000777200707772340000000072BBA7BA76FB
:101B70005E663E0000000031000000316D61000033
:101B80000003004EBBA15D7A5EE45C000000003102
:101B9000000000317361000000130352BB3D5E087A
:101BA000BAEF5C6666E63F310000003174720000F7
:101BB000001B0457BB3D5E14BAF35C0000204231A9
:101BC000000000316D69000000030066BBA15D20CC
:101BD000BAE55C000000413100000031706F000088
:101BE0000003006ABBA15DCB5EE95C0000803F3171
:101BF00000000031706D00000003006EBBA15D9716
:101C0000BAEA5C0000004032000000326D61000062
:101C10000003004EBBA15D7A5E035D0000803F3291
:101C2000000000327361000000130352BB3D5E08E8
:101C3000BA0E5D6666E63F32000000327472000044
:101C4000001B0457BB3D5E14BA125D0000204232F7
:101C5000000000326D69000000030066BBA15D203A
:101C6000BA045D000000413200000032706F0000D5
:101C70000003006ABBA15DCB5E085D0000803F32BF
:101C800000000032706D00000003006EBBA15D9784
:101C9000BA095D0000004033000000336D610000B0
:101CA0000003004EBBA15D7A5E225D0000803F33E1
:101CB000000000337361000000130352BB3D5E0857
:101CC000BA2D5D6666E63F33000000337472000093
:101CD000001B0457BB3D5E14BA315D000020423347
:101CE000000000336D69000000030066BBA15D20A9
:101CF000BA235D000000413300000033706F000024
:101D00000003006ABBA15DCB5E275D0000000033CD
:101D100000000033706D00000003006EBBA15D97F2
:101D2000BA285D0000004034000000346D610000FE
:101D30000003004EBBA15D7A5E415D0000004034AF
:101D4000000000347361000000130352BB3D5E08C5
:101D5000BA4C5D6666E63F340000003474720000E1
:101D6000001B0457BB3D5E14BA505D6076074034DB
:101D7000000000346D69000000030066BBA15D2017
:101D8000BA425D000000413400000034706F000072
:101D90000003006ABBA15DCB5E465D0000803F345E
:101DA00000000034706D00000003006EBBA15D9761
:101DB000BA475D000000407800000078616D0000C7
:101DC000000300785BFD580A5972350000803F78A7
:101DD00000000078766D0000001B00C15B3D5E9244
:101DE00063773500007A467800000078667200005C
:101DF000001B00BD5B3D5E9263733500007A467840
:101E000000000078746E0000001B03C95B3D5E9209
:101E1000637F35000000007800000078746D0000DA
:101E2000001B03C55B3D5E92637B350000914378E8
:101E3000000000786A6D0000001B00CD5B3D5E7203
:101E400059833500409C4578000000786A6800009E
:101E5000001B00D15B3D5ECA59873500401C4678A7
:101E6000000000786A640000001B04D55B3D5E92B0
:101E7000638F350AD7233C7800000078736E00002A
:101E8000000300DD5BA15D04BE96340000803F7856
:101E90000000007873780000000300E15BA15D049E
:101EA000BE973400000000780000007873760000D0
:101EB000001B00E55B3D5E9263973500803B4578F3
:101EC000000000786C760000001B00E95B3D5E922C
:101ED000639B350000C84278000000786C62000007
:101EE000001B03ED5B3D5E92639F3500002041784F
:101EF000000000787A620000001B03F15B3D5E92F7
:101F000063A335000000407900000079616D000096
:101F1000000300785BFD580A59A7350000803F791F
:101F200000000079766D0000001B00C15B3D5E92F1
:101F300063AC3500007A46790000007966720000D3
:101F4000001B00BD5B3D5E9263A83500007A4679B8
:101F500000000079746E0000001B03C95B3D5E92B7
:101F600063B435000000007900000079746D000052
:101F7000001B03C55B3D5E9263B0350000A0437952
:101F8000000000796A6D0000001B00CD5B3D5E72B1
:101F900059B83500409C4579000000796A68000016
:101FA000001B00D15B3D5ECA59BC3500401C467920
:101FB000000000796A640000001B04D55B3D5E925E
:101FC00063C4350AD7233C7900000079736E0000A2
:101FD000000300DD5BA15D04BE98340000803F7902
:101FE0000000007973780000000300E15BA15D044C
:101FF000BE9934000000007900000079737600007B
:10200000001B00E55B3D5E9263CC3500803B45796B
:10201000000000796C760000001B00E95B3D5E92D9
:1020200063D0350000C84279000000796C6200007E
:10203000001B03ED5B3D5E9263D4350000204179C7
:10204000000000797A620000001B03F15B3D5E92A4
:1020500063D835000000407A0000007A616D00000E
:10206000000300785BFD580A59DC350000803F7A98
:102070000000007A766D0000001B00C15B3D5E929F
:1020800063E13500007A447A0000007A667200004D
:10209000001B00BD5B3D5E9263DD3500007A447A33
:1020A0000000007A746E0000001B03C95B3D5E9265
:1020B00063E9350000F0C27A0000007A746D000018
:1020C000001B03C55B3D5E9263E535000000007AAE
:1020D0000000007A6A6D0000001B00CD5B3D5E725F
:1020E00059ED35000048427A0000007A6A68000025
:1020F000001B00D15B3D5ECA59F13500007A447A7D
:102100000000007A6A640000001B04D55B3D5E920B
:1021100063F9350AD7233C7A0000007A736E000019
:10212000000300DD5BA15D04BE9A34000000007A6C
:102130000000007A73780000000300E15BA15D04F9
:10214000BE9B340000803F7A0000007A7376000066
:10215000001B00E55B3D5E9263013600007A447A25
:102160000000007A6C760000001B00E95B3D5E9287
:102170006305360000C8427A0000007A6C620000F5
:10218000001B03ED5B3D5E92630936000020417A3F
:102190000000007A7A620000001B03F15B3D5E9252
:1021A000630D36000040406100000061616D000079
:1021B000000300785BFD580A591136000040406169
:1021C00000000061766D0000001300C15B3D5E52AF
:1021D0005F16360080CA466100000061667200002A
:1021E000001300BD5B3D5E525F123600804A4661BF
:1021F00000000061746E0000001303C95B3D5E9235
:10220000631E36000080BF6100000061746D000035
:10221000001303C55B3D5E525F1A36000080BF614C
:10222000000000616A6D0000001300CD5B3D5E722E
:1022300059223600349E4861000000616A6800003F
:10224000001300D15B3D5ECA59263600349E4861BA
:10225000000000616A640000001304D55B3D5E521B
:102260005F2E36CDCCCC3D61000000617261000074
:10227000001B03D95B3D5E525F3236DFC3A940616C
:1022800000000061736E0000000300DD5BA15D04CF
:10229000BE9C340000803F61000000617378000044
:1022A000000300E15BA15D04BE9D340000000061FD
:1022B0000000006173760000001300E55B3D5E5294
:1022C0005F36360000FA4461000000616C76000061
:1022D000001300E95B3D5E525F3A360000FA44614C
:1022E000000000616C620000001303ED5B3D5E5274
:1022F0005F3E360000A04061000000617A6200008D
:10230000001303F15B3D5E525F4236000000406205
:1023100000000062616D0000000300785BFD580A58
:10232000594636000000006200000062766D000031
:10233000001300C15B3D5E525F4B36000061456299
:102340000000006266720000001300BD5B3D5E523B
:102350005F4736000061456200000062746E000055
:10236000001303C95B3D5E92635336000080BF6279
:1023700000000062746D0000001303C55B3D5E52F7
:102380005F4F36000080BF62000000626A6D00008F
:10239000001300CD5B3D5E725957360000A04162CC
:1023A000000000626A640000001300D55B3D5E52CD
:1023B0005F63360AD7233C6200000062726100004E
:1023C000001B03D95B3D5E525F67360000803F63B0
:1023D00000000063616D0000000300785BFD580A97
:1023E000597B36000000006300000063766D00003A
:1023F000001300C15B3D5E525F80360000614563A3
:102400000000006366720000001300BD5B3D5E5279
:102410005F7C36000061456300000063746E00005D
:10242000001303C95B3D5E92638836000080BF6382
:1024300000000063746D0000001303C55B3D5E5235
:102440005F8436000080BF63000000636A6D000097
:10245000001300CD5B3D5E72598C360000A04163D5
:10246000000000636A640000001300D55B3D5E520B
:102470005F98360AD7233C63000000637261000056
:10248000001B03D95B3D5E525F9C360000803F70AD
:1024900031000070316672710013006AA83D5E520F
:1024A0005FC05B0000C84270310000703163736C24
:1024B0000013006EA83D5E525FC45B00007A44705A
:1024C000310000703163736800130072A83D5E52E2
:1024D0005FC85B0000FA4470310000703163706CBB
:1024E00000130376A83D5E525FCC5B0000003E7097
:1024F00031000070316370680013037AA83D5E52AA
:102500005FD05BCDCC4C3E70310000703177736C86
:102510000013007EA83D5E525FD45B00007A4470D9
:10252000310000703177736800130082A83D5E525D
:102530005FD85B0000FA4470310000703177706C36
:1025400000130386A83D5E525FDC5B0000003E7016
:1025500031000070317770680013038AA83D5E5225
:102560005FE05BCDCC4C3E703100007031706F6627
:102570000013038EA83D5E525FE45BCDCCCC3D677B
:102580003534006735347800001B03F55B3D5E92FF
:1025900063E23400000000673534006735347900A9
:1025A000001B03F55B3D5E9263E6340000000067AC
:1025B0003534006735347A00001B03F55B3D5E92CD
:1025C00063EA340000000067353400673534610089
:1025D000001B03F55B3D5E525FEE340000000067B8
:1025E0003534006735346200001B03F55B3D5E52F5
:1025F0005FF2340000000067353400673534630053
:10260000001B03F55B3D5E525FF63400000000677F
:102610003535006735357800001B03F55B3D5E926C
:1026200063FA3400001143673535006735357900AA
:10263000001B03F55B3D5E9263FE340000204367A0
:102640003535006735357A00001B03F55B3D5E923A
:1026500063023500000000673535006735356100DD
:10266000001B03F55B3D5E525F063500000000670E
:102670003535006735356200001B03F55B3D5E5262
:102680005F0A3500000000673535006735356300A7
:10269000001B03F55B3D5E525F0E350000000067D6
:1026A0003536006735367800001B03F55B3D5E92DA
:1026B0006312350000000067353600673536790053
:1026C000001B03F55B3D5E9263163500000000675A
:1026D0003536006735367A00001B03F55B3D5E92A8
:1026E000631A350000000067353600673536610033
:1026F000001B03F55B3D5E525F1E35000000006766
:102700003536006735366200001B03F55B3D5E52CF
:102710005F223500000000673536006735366300FC
:10272000001B03F55B3D5E525F263500000000672D
:102730003537006735377800001B03F55B3D5E9247
:10274000632A3500000000673537006735377900A8
:10275000001B03F55B3D5E92632E350000000067B1
:102760003537006735377A00001B03F55B3D5E9215
:102770006332350000000067353700673537610088
:10278000001B03F55B3D5E525F36350000000067BD
:102790003537006735376200001B03F55B3D5E523D
:1027A0005F3A350000000067353700673537630052
:1027B000001B03F55B3D5E525F3E35000000006785
:1027C0003538006735387800001B03F55B3D5E92B5
:1027D00063423500000000673538006735387900FE
:1027E000001B03F55B3D5E92634635000000006709
:1027F0003538006735387A00001B03F55B3D5E9283
:10280000634A3500000000673538006735386100DD
:10281000001B03F55B3D5E525F4E35000000006714
:102820003538006735386200001B03F55B3D5E52AA
:102830005F523500000000673538006735386300A7
:10284000001B03F55B3D5E525F56350000000067DC
:102850003539006735397800001B03F55B3D5E9222
:10286000635A350000000067353900673539790053
:10287000001B03F55B3D5E92635E35000000006760
:102880003539006735397A00001B03F55B3D5E92F0
:102890006362350000000067353900673539610033
:1028A000001B03F55B3D5E525F663500000000676C
:1028B0003539006735396200001B03F55B3D5E5218
:1028C0005F6A3500000000673539006735396300FD
:1028D000001B03F55B3D5E525F6E35000000006734
:1028E0003932006739327800001103F55B3D5E76BE
:1028F0005E533700000000673932006739327900D3
:10290000001103F55B3D5E765E57370000000067FF
:102910003932006739327A00001103F55B3D5E768B
:102920005E5B3700000000673932006739326100B2
:10293000001103F55B3D5E765E5F370000000067C7
:102940003932006739326200001103F55B3D5E7673
:102950005E63370000000067393200673932630078
:10296000001103F55B3D5E765E673700000000678F
:102970003238006732387800001103F95B3D5E762B
:102980005E6B37000000006732380067323879002C
:10299000001103F95B3D5E765E6F37000000006753
:1029A0003238006732387A00001103F95B3D5E76F9
:1029B0005E7337000000006732380067323861000C
:1029C000001103F95B3D5E765E773700000000671B
:1029D0003238006732386200001103F95B3D5E76E1
:1029E0005E7B3700000000673238006732386300D2
:1029F000001103F95B3D5E765E7F370000000067E3
:102A00003330006733307800001103F95B3D5E76A8
:102A10005E83370000000067333000673330790091
:102A2000001103F95B3D5E765E87370000000067AA
:102A30003330006733307A00001103F95B3D5E7676
:102A40005E8B370000000067333000673330610071
:102A5000001103F95B3D5E765E8F37000000006772
:102A60003330006733306200001103F95B3D5E765E
:102A70005E93370000000067333000673330630037
:102A8000001103F95B3D5E765E9737000000006A37
:102A90006964006A69646100000000DCC0165E2B96
:102AA0005F863E000000006A6964006A6964620033
:102AB000000000DCC0165E2B5F8A3E000000006A4A
:102AC0006964006A69646300000000DCC0165E2B64
:102AD0005F8E3E000000006A6964006A69646400F9
:102AE000000000DCC0165E2B5F923E000000007309
:102AF0007973006A61000000001F00175B3D5E9261
:102B000063B0340024F449737973006374000000E7
:102B1000001F04365B3D5E9263B4340AD7233C73D6
:102B2000797300736C000000000700555BA15D7AAB
:102B30005EB8340000000073797300737400000005
:102B400000070016BEA15DFEBD8B340000803F7300
:102B50007973006D740000000017024ABB3D5EBF30
:102B6000BAE05C00000040000000006D650000005D
:102B70000000002CC11CBB1CBB663E000000000016
:102B80000000006D640000000000002CC1F9BAF9DB
:102B9000BA663E0000000073797300656A000000A9
:102BA0000007005681A15DCB5E783E0000803F7338
:102BB0007973006A760000000007005A81A15D1851
:102BC0008150410000A040737973006A73000000D7
:102BD0000007005E81A15DCB5E51410000803F7324
:102BE0007973007476000000000700F1C1A15DCB8D
:102BF0005E535E0000803F737973007176000000C1
:102C000000070090AEA15D0B5F195C00000000732F
:102C1000797300737600000000070005ADA15DEB3D
:102C20005E265C0000803F737973007369000000CA
:102C300000070001ADEF5DDAAC275C00007A43735A
:102C40007973006563000000000700E363A15DDFA6
:102C5000646834000000007379730065650000004B
:102C6000000700E763A15DBF6469340000000073E2
:102C70007973006578000000000700EB63A15D9F99
:102C8000646A34000000407379730072786D00004C
:102C9000000700EF63A15DCB5E6B340000803F73E3
:102CA0007973006261756400000400F363A15D49FB
:102CB0006366340000A04000000000737200000052
:102CC000000000FFACD6ACD8AC663E0000000000AF
:102CD000000000717200000000000084AE49AE7672
:102CE0005E663E0000000000000000716900000008
:102CF00000000088AE5CAE765E663E00000000001C
:102D0000000000716F0000000000008CAE70AE7615
:102D10005E663E00000000000000006572000000DA
:102D2000000000DCC05DA9765E663E000000000089
:102D30000000007166000000000000DCC09D5DF630
:102D400059663E000000000000000072780000009C
:102D50000000005AC12763765E663E000000000056
:102D60000000006D736700000000002CC19D5D76BF
:102D70005E663E0000000000000000636C6561724A
:102D8000000000DCC0F44EF44E663E00000000007F
:102D90000000007061757365000000DCC0114F1108
:102DA0004F663E0000000000000000737461727402
:102DB000000000DCC0164F164F663E000000000009
:102DC000000000666C757368000000DCC01B4F1BC0
:102DD0004F663E00000000000000007265736574DD
:102DE000000000DCC0204F204F663E0000000000C5
:102DF000000000616C61726D000000DCC0E24EE218
:102E00004E663E0000000000000000747874000070
:102E1000000000DCC09D5D785E663E0000000000A2
:102E200000000074696400000001005AC1EF5DAA4F
:102E30005E963E00000000000000007465737400A0
:102E4000000000DCC0397A1ABE663E0000000000B7
:102E50000000006465666100000000DCC0647A4127
:102E60005D663E0000000000000000626F6F7400AD
:102E7000000000DCC08F7A8A79663E000000000006
:102E800000000068656C7000000000DCC0FA797614
:102E90005E663E00000000000000006800000000C8
:102EA000000000DCC0FA79765E663E000000007328
:102EB00079730067706C0000000700035BA15DEB95
:102EC0005EC634000000007379730067756E000001
:102ED000000700075BA15DCB5EC7340000803F7335
:102EE00079730067636F00000007000B5BA15D7AD8
:102EF0005EC5340000803F73797300677061000025
:102F00000007000F5BA15DEB5EC83400000040735A
:102F10007973006764690000000700135BA15DCB53
:102F20005EC934000000000000000067630000007C
:102F3000000000DCC041785178663E0000000000CF
:102F40000000006D61000000001B04595B3D5E92B3
:102F500063BD34CDCCCC3D000000006664000000B1
:102F60000003005AC1A15DCB5E5241000000007514
:102F700064610075646130000003005AC1165E2B65
:102F80005F223E00000000756461007564613100DD
:102F90000003005AC1165E2B5F263E00000000753C
:102FA00064610075646132000003005AC1165E2B33
:102FB0005F2A3E00000000756461007564613300A3
:102FC0000003005AC1165E2B5F2E3E000000007504
:102FD00064620075646230000003005AC1165E2B03
:102FE0005F323E000000007564620075646231006B
:102FF0000003005AC1165E2B5F363E0000000075CC
:1030000064620075646232000003005AC1165E2BD0
:103010005F3A3E0000000075646200756462330030
:103020000003005AC1165E2B5F3E3E000000007593
:1030300064630075646330000003005AC1165E2BA0
:103040005F423E00000000756463007564633100F8
:103050000003005AC1165E2B5F463E00000000755B
:1030600064630075646332000003005AC1165E2B6E
:103070005F4A3E00000000756463007564633300BE
:103080000003005AC1165E2B5F4E3E000000007523
:1030900064640075646430000003005AC1165E2B3E
:1030A0005F523E0000000075646400756464310086
:1030B0000003005AC1165E2B5F563E0000000075EB
:1030C00064640075646432000003005AC1165E2B0C
:1030D0005F5A3E000000007564640075646433004C
:1030E0000003005AC1165E2B5F5E3E000000005FC9
:1030F0007465005F7465780000100288C13D5E76DB
:103100005E8959000000005F7465005F7465790096
:1031100000100288C13D5E765E8D59000000005FA0
:103120007465005F74657A0000100288C13D5E76A8
:103130005E9159000000005F7465005F7465610076
:1031400000100288C13D5E765E9559000000005F68
:103150007465005F7465620000100288C13D5E7690
:103160005E9959000000005F7465005F746563003C
:1031700000100288C13D5E765E9D59000000005F30
:103180007472005F7472780000100288C13D5E7630
:103190005EAE5A000000005F7472005F74727900C6
:1031A00000100288C13D5E765EB25A000000005FEA
:1031B0007472005F74727A0000100288C13D5E76FE
:1031C0005EB65A000000005F7472005F74726100A6
:1031D00000100288C13D5E765EBA5A000000005FB2
:1031E0007472005F7472620000100288C13D5E76E6
:1031F0005EBE5A000000005F7472005F747263006C
:1032000000100288C13D5E765EC25A000000005F79
:103210007473005F7473310000100288C13D5E76E4
:103220005E195A000000005F7073005F7073310018
:1032300000100288C13D5E765E295A000000005FE2
:103240006373005F6373310000100288C13D5E76D6
:103250005E395A000000005F6573005F65733100DE
:1032600000100288C13D5E765E495A000000005F92
:103270007873005F7873310000100288C13D5E767C
:103280005E7B5D000000005F6665005F6665310083
:1032900000100288C13D5E765E595A000000005F52
:1032A0007473005F7473320000100288C13D5E7653
:1032B0005E1D5A000000005F7073005F7073320083
:1032C00000100288C13D5E765E2D5A000000005F4E
:1032D0006373005F6373320000100288C13D5E7645
:1032E0005E3D5A000000005F6573005F6573320049
:1032F00000100288C13D5E765E4D5A000000005FFE
:103300007873005F7873320000100288C13D5E76EA
:103310005E935D000000005F6665005F66653200D9
:1033200000100288C13D5E765E5D5A000000005FBD
:103330007473005F7473330000100288C13D5E76C1
:103340005E215A000000005F7073005F70733300ED
:1033500000100288C13D5E765E315A000000005FB9
:103360006373005F6373330000100288C13D5E76B3
:103370005E415A000000005F6573005F65733300B3
:1033800000100288C13D5E765E515A000000005F69
:103390007873005F7873330000100288C13D5E7659
:1033A0005EAB5D000000005F6665005F6665330030
:1033B00000100288C13D5E765E615A000000005F29
:1033C0007473005F7473340000100288C13D5E7630
:1033D0005E255A000000005F7073005F7073340058
:1033E00000100288C13D5E765E355A000000005F25
:1033F0006373005F6373340000100288C13D5E7622
:103400005E455A000000005F6573005F657334001D
:1034100000100288C13D5E765E555A000000005FD4
:103420007873005F7873340000100288C13D5E76C7
:103430005EC35D000000005F6665005F6665340086
:1034400000100288C13D5E765E655A0000000000F3
:103450000000005F64616D00000000DCC06B5A6B0F
:103460005A663E0000000000000000736530300026
:10347000000200DCC0C85D915E325C00000000000C
:103480000000007365303100000200DCC0C85D91AF
:103490005E345C0000000000000000736530320004
:1034A000000200DCC0C85D915E365C0000000000D8
:1034B0000000007365303300000200DCC0C85D917D
:1034C0005E385C00000000000000007365303400CE
:1034D000000200DCC0C85D915E3A5C0000000000A4
:1034E0000000007365303500000200DCC0C85D914B
:1034F0005E3C5C0000000000000000736530360098
:10350000000200DCC0C85D915E3E5C00000000006F
:103510000000007365303700000200DCC0C85D9118
:103520005E405C0000000000000000736530380061
:10353000000200DCC0C85D915E425C00000000003B
:103540000000007365303900000200DCC0C85D91E6
:103550005E445C0000000000000000736531300034
:10356000000200DCC0C85D915E465C000000000007
:103570000000007365313100000200DCC0C85D91BD
:103580005E485C00000000000000007365313200FE
:10359000000200DCC0C85D915E4A5C0000000000D3
:1035A0000000007365313300000200DCC0C85D918B
:1035B0005E4C5C00000000000000007365313400C8
:1035C000000200DCC0C85D915E4E5C00000000009F
:1035D0000000007365313500000200DCC0C85D9159
:1035E0005E505C0000000000000000736531360092
:1035F000000200DCC0C85D915E525C00000000006B
:103600000000007365313700000200DCC0C85D9126
:103610005E545C000000000000000073653138005B
:10362000000200DCC0C85D915E565C000000000036
:103630000000007365313900000200DCC0C85D91F4
:103640005E585C000000000000000073653230002E
:10365000000200DCC0C85D915E5A5C000000000002
:103660000000007365323100000200DCC0C85D91CB
:103670005E5C5C00000000000000007365323200F8
:10368000000200DCC0C85D915E5E5C0000000000CE
:103690000000007365323300000200DCC0C85D9199
:1036A0005E605C00000000000000007365323400C2
:1036B000000200DCC0C85D915E625C00000000009A
:1036C0000000007365323500000200DCC0C85D9167
:1036D0005E645C000000000000000073653236008C
:1036E000000200DCC0C85D915E665C000000000066
:1036F0000000007365323700000200DCC0C85D9135
:103700005E685C0000000000000000736532380055
:10371000000200DCC0C85D915E6A5C000000000031
:103720000000007365323900000200DCC0C85D9102
:103730005E6C5C0000000000000000737973000004
:10374000000000DCC023618B5F663E0000000000CB
:103750000000007031000000000000DCC023618B1D
:103760005F663E0000000000000000310000000025
:10377000000000DCC023618B5F663E00000000009B
:103780000000003200000000000000DCC023618B5C
:103790005F663E00000000000000003300000000F3
:1037A000000000DCC023618B5F663E00000000006B
:1037B0000000003400000000000000DCC023618B2A
:1037C0005F663E000000000000000078000000007E
:1037D000000000DCC023618B5F663E00000000003B
:1037E0000000007900000000000000DCC023618BB5
:1037F0005F663E00000000000000007A000000004C
:10380000000000DCC023618B5F663E00000000000A
:103810000000006100000000000000DCC023618B9C
:103820005F663E0000000000000000620000000033
:10383000000000DCC023618B5F663E0000000000DA
:103840000000006300000000000000DCC023618B6A
:103850005F663E0000000000000000673534000095
:10386000000000DCC023618B5F663E0000000000AA
:103870000000006735350000000000DCC023618BCC
:103880005F663E0000000000000000673536000063
:10389000000000DCC023618B5F663E00000000007A
:1038A0000000006735370000000000DCC023618B9A
:1038B0005F663E0000000000000000673538000031
:1038C000000000DCC023618B5F663E00000000004A
:1038D0000000006735390000000000DCC023618B68
:1038E0005F663E0000000000000000673932000003
:1038F000000000DCC023618B5F663E00000000001A
:103900000000006732380000000000DCC023618B3B
:103910005F663E00000000000000006733300000DA
:10392000000000DCC023618B5F663E0000000000E9
:103930000000006D706F0000000000DCC023618B90
:103940005F663E0000000000000000706F73000022
:10395000000000DCC023618B5F663E0000000000B9
:103960000000006F66730000000000DCC023618B64
:103970005F663E0000000000000000686F6D000000
:10398000000000DCC023618B5F663E000000000089
:103990000000007072620000000000DCC023618B38
:1039A0005F663E00000000000000007077720000BB
:1039B000000000DCC023618B5F663E000000000059
:1039C0000000006A6F670000000000DCC023618B0C
:1039D0005F663E00000000000000006A69640000AD
:1039E000000000DCC023618B5F663E000000000029
:1039F0000000007564610000000000DCC023618BE2
:103A00005F663E0000000000000000756462000078
:103A1000000000DCC023618B5F663E0000000000F8
:103A20000000007564630000000000DCC023618BAF
:103A30005F663E0000000000000000756464000046
:103A4000000000DCC023618B5F663E0000000000C8
:103A50000000005F74650000000000DCC023618B83
:103A60005F663E00000000000000005F747200000E
:103A7000000000DCC023618B5F663E000000000098
:103A80000000005F74730000000000DCC023618B45
:103A90005F663E00000000000000005F70730000E1
:103AA000000000DCC023618B5F663E000000000068
:103AB0000000005F63730000000000DCC023618B26
:103AC0005F663E00000000000000005F65730000BC
:103AD000000000DCC023618B5F663E000000000038
:103AE0000000005F78730000000000DCC023618BE1
:103AF0005F663E00000000000000005F6665000099
:103B0000000000DCC023618B5F663E000000000007
:103B10000000006D00000000000000DCC05A647668
:103B20005E663E0000000000000000710000000022
:103B3000000000DCC04064765E663E0000000000CD
:103B40000000006F00000000000000DCC02664766A
:103B50005E663E000000000000000024000000003F
:103B6000000000DCC07464765E663E000000004821
:103B70006F6D696E67206572726F72202D202563EC
:103B800020617869732073657474696E6773206D42
:103B90006973636F6E666967757265640050726FF2
:103BA00062696E67206572726F72202D2025632016
:103BB000617869732063616E6E6F74206D6F7665D6
:103BC00020647572696E672070726F62696E67003B
:103BD0005B69645D202054696E7947204944253330
:103BE00030730A005B68765D2020686172647761DB
:103BF00072652076657273696F6E2531362E326676
:103C00000A005B68705D202068617264776172658C
:103C100020706C6174666F726D253132640A005BCE
:103C200066765D20206669726D77617265207665C3
:103C30007273696F6E2531362E32660A005B6662DA
:103C40005D20206669726D77617265206275696CAE
:103C5000642531382E32660A00456E746572202460
:103C6000626F6F743D3120746F20656E74657220D1
:103C700074686520626F6F74206C6F616465722E6A
:103C80000A000A0A0A2323232054696E7947204236
:103C90004F4F54204C4F414445522048656C702092
:103CA0002323230A00456E746572202464656661CF
:103CB0003D3120746F2072657365742074686520CF
:103CC00073797374656D20746F2074686520666104
:103CD00063746F72792064656661756C74207661B7
:103CE0006C7565732E0A546869732077696C6C2053
:103CF0006F766572777269746520616E792063688A
:103D0000616E67657320796F752068617665206DD7
:103D10006164652E0A000A0A0A2323232054696E6F
:103D2000794720524553544F52452044454641550A
:103D30004C54532048656C70202323230A00496E9D
:103D4000766F6B652073656C662074657374206292
:103D50007920656E746572696E672024746573746A
:103D60003D4E207768657265204E206973206F6E26
:103D700065206F663A0A202024746573743D3120F3
:103D800020736D6F6B6520746573740A2020247432
:103D90006573743D322020686F6D696E67207465AD
:103DA000737420202028796F75206D7573742074CA
:103DB00072697020686F6D696E67207377697463CC
:103DC000686573290A202024746573743D332020AC
:103DD0007371756172652074657374202020286189
:103DE00020736572696573206F66207371756172E7
:103DF0006573290A202024746573743D3420206182
:103E00007263207465737420202020202028736F33
:103E10006D65206C6172676520636972636C6573A0
:103E2000290A202024746573743D35202064776549
:103E30006C6C207465737420202020286D6F76656B
:103E4000732073706163656420627920312073652B
:103E5000636F6E64206477656C6C73290A2020247C
:103E6000746573743D36202066656564686F6C64A4
:103E700020746573742028656E746572202120613A
:103E80006E64207E20746F20686F6C6420616E64A5
:103E900020726573746172742C207265737065632F
:103EA000746976656C79290A202024746573743DE1
:103EB0003720204D20636F64657320746573742010
:103EC00020284D20636F64657320696E7465726D80
:103ED000696E676C65642077697468206D6F7665BC
:103EE00073290A202024746573743D3820204A53B6
:103EF0004F4E20746573742020202020286D6F742D
:103F0000696F6E20746573742072756E20757369A5
:103F10006E67204A534F4E20636F6D6D616E647300
:103F2000290A202024746573743D392020696E7637
:103F3000657273652074696D6520746573740A20F9
:103F40002024746573743D313020726F746172790E
:103F5000206D6F74696F6E20746573740A2020245D
:103F6000746573743D313120736D616C6C206D6FBD
:103F700076657320746573740A20202474657374E5
:103F80003D313220736C6F77206D6F7665732074CE
:103F90006573740A202024746573743D3133206383
:103FA0006F6F7264696E6174652073797374656D87
:103FB000206F6666736574207465737420284739B2
:103FC000322C204735342D473539290A0A54657378
:103FD000747320617373756D6520612063656E7401
:103FE00065726564205859206F726967696E206137
:103FF0006E64206174206C656173742038306D6D5F
:1040000020636C656172616E636520696E20616C0E
:104010006C20646972656374696F6E730A546573AA
:10402000747320617373756D65205A206861732005
:104030006174206C656173742034306D6D20706F15
:104040007369697469766520636C656172616E631A
:10405000650A546573747320737461727420776990
:1040600074682061204730205830205930205A3061
:10407000206D6F76650A486F6D696E6720697320E1
:1040800074686520657863657074696F6E2E204E64
:104090006F20696E697469616C20706F73697469EF
:1040A0006F6E206F7220636C656172616E63652054
:1040B000697320617373756D65640A000A0A0A23C7
:1040C00023232054696E79472053454C462054459C
:1040D00053542048656C70202323230A00456163F4
:1040E00068202420636F6D6D616E642061626F765D
:1040F0006520616C736F20646973706C61797320E3
:1041000074686520746F6B656E20666F72206561E0
:1041100063682073657474696E6720696E205B2024
:104120005D20627261636B6574730A546F207669F7
:1041300065772073657474696E677320656E746546
:1041400072206120746F6B656E3A0A0A2020243C4D
:10415000746F6B656E3E0A0A466F72206578616DFA
:10416000706C65202479667220746F2064697370A6
:104170006C6179207468652059206D6178206665CE
:10418000656420726174650A0A546F2075706461F9
:1041900074652073657474696E677320656E7465E9
:1041A0007220746F6B656E20657175616C7320761B
:1041B000616C75653A0A0A2020243C746F6B656E49
:1041C0003E3D3C76616C75653E0A0A466F7220651D
:1041D00078616D706C6520247966723D38303020CE
:1041E000746F20736574207468652059206D617840
:1041F0002066656564207261746520746F203830B4
:1042000030206D6D2F6D696E7574650A466F722072
:10421000636F6E66696775726174696F6E2064653D
:104220007461696C73207365653A20687474707387
:104230003A2F2F6769746875622E636F6D2F7379DB
:104240006E746865746F732F54696E79472F776940
:104250006B692F54696E79472D436F6E6669677578
:10426000726174696F6E0A00546865736520636FCC
:104270006D6D616E6473206172652061637469762F
:104280006520666F7220636F6E6669677572617410
:10429000696F6E3A0A2020247379732053686F7710
:1042A0002073797374656D202867656E6572616C23
:1042B000292073657474696E67730A202024312085
:1042C000202053686F77206D6F746F7220312073D8
:1042D000657474696E677320286F722077686174E3
:1042E00065766572206D6F746F7220796F752077B7
:1042F000616E7420312C322C332C34290A20202476
:104300007820202053686F772058206178697320C7
:1043100073657474696E677320286F7220776861A3
:104320007465766572206178697320796F7520777E
:10433000616E7420782C792C7A2C612C622C632984
:104340000A2020246D20202053686F7720616C6C38
:10435000206D6F746F722073657474696E67730A71
:104360002020247120202053686F7720616C6C20FE
:10437000617869732073657474696E67730A2020AD
:10438000246F20202053686F7720616C6C206F664B
:10439000667365742073657474696E67730A202090
:1043A000242420202053686F7720616C6C20736573
:1043B0007474696E67730A20202468202020536873
:1043C0006F7720746869732068656C7020736372FE
:1043D00065656E0A0A000A0A0A2323232054696EBF
:1043E000794720434F4E46494755524154494F4E15
:1043F0002048656C70202323230A000A466F722030
:1044000064657461696C65642054696E79472069DC
:104410006E666F207365653A2068747470733A2F06
:104420002F6769746875622E636F6D2F73796E7470
:104430006865746F732F54696E79472F77696B695C
:104440002F0A466F7220746865206C6174657374FE
:10445000206669726D77617265207365653A2068C0
:10446000747470733A2F2F6769746875622E636F66
:104470006D2F73796E746865746F732F54696E79DC
:10448000470A506C65617365206C6F6720616E79B7
:104490002069737375657320617420687474703A51
:1044A0002F2F7777772E73796E746865746F732EFC
:1044B000636F6D2F666F72756D730A486176652044
:1044C00066756E0A000A4E6F74653A2054696E79FB
:1044D000472067656E657261746573206175746FDE
:1044E0006D61746963207374617475732072657093
:1044F0006F7274732062792064656661756C740AEA
:10450000546869732063616E206265206469736119
:10451000626C656420627920656E746572696E678D
:10452000202473763D300A536565207468652077D2
:10453000696B692062656C6F7720666F72206D6FA2
:1045400072652064657461696C732E0A0054686535
:10455000736520636F6D6D616E6473206172652099
:104560006163746976652066726F6D20746865207A
:10457000636F6D6D616E64206C696E653A0A205ED2
:10458000782020202020202020202020202052655C
:104590007365742028636F6E74726F6C20782920A5
:1045A0002D20736F66747761726520726573657410
:1045B0000A20203F202020202020202020202020F2
:1045C000204D616368696E6520706F736974696FEF
:1045D0006E20616E642067636F6465206D6F646533
:1045E0006C2073746174650A202024202020202010
:1045F000202020202020202053686F7720616E64C7
:104600002073657420636F6E666967757261746983
:104610006F6E2073657474696E67730A20202120A1
:104620002020202020202020202020204665656496
:10463000686F6C64202D2073746F70206D6F7469C7
:104640006F6E20776974686F7574206C6F73696E14
:104650006720706F736974696F6E0A20207E202056
:1046600020202020202020202020204379636C65FA
:10467000205374617274202D20726573746172749A
:104680002066726F6D2066656564686F6C640A20D1
:10469000206820202020202020202020202020539F
:1046A000686F7720746869732068656C7020736325
:1046B0007265656E0A20202468202020202020209A
:1046C000202020202053686F7720636F6E66696713
:1046D00075726174696F6E2068656C7020736372A7
:1046E00065656E0A202024746573742020202020C4
:1046F000202020204C6973742073656C662D7465CE
:104700007374730A202024746573743D4E20202036
:104710002020202052756E2073656C662D746573A1
:1047200074204E0A202024686F6D653D31202020C2
:104730002020202052756E206120686F6D696E67A1
:10474000206379636C650A202024646566613D31CD
:1047500020202020202020526573746F7265206114
:104760006C6C2073657474696E677320746F20229B
:10477000666163746F7279222064656661756C741A
:10478000730A000A0A0A2323232054696E794720FA
:1047900048656C70202323230A0022007B227222AA
:1047A0003A7B226D7367223A22007B723A7B6D73EB
:1047B000673A22005B6A735D20206A736F6E207314
:1047C000657269616C697A65207374796C652539E5
:1047D00064205B303D72656C617865642C313D739B
:1047E00074726963745D0A005B6A765D20206A7387
:1047F0006F6E20766572626F7369747925313564E6
:10480000205B303D73696C656E742C313D666F6F53
:104810007465722C323D6D657373616765732C33FB
:104820003D636F6E666967732C343D6C696E656EAF
:10483000756D2C353D766572626F73655D0A005B40
:10484000656A5D2020656E61626C65206A736F6EBB
:10485000206D6F646525313364205B303D7465786D
:10486000742C313D4A534F4E5D0A00B959B359ACCF
:1048700059A7599E59935988597C59705962594B77
:10488000593C592F5923590F590259ED58D958D627
:1048900058D358C458AF589A588B587B58695852B7
:1048A0005835581858FF57E957D857C657B957A71A
:1048B000578D578A578757845781577E577B57782C
:1048C00057755772576F576C5769576657635760DC
:1048D000575D575A575757545751574E574B57488C
:1048E00057455742573F573C57395736573357303C
:1048F000572D572A572757245721571E571B5718EC
:1049000057155712570F570C57095706570357009B
:1049100057FD56FA56F756F456F156EE56C756A3BB
:1049200056835669564F5635561156F455DC55C6C2
:1049300055AC5588556B555955395522550955E78C
:1049400054CE54B05494547C546A544C5437541636
:104950005412540E540A5406540254FE53FA53F699
:1049600053F253EE53EA53E653E253DE53DA53C0A5
:1049700053A6539353775365534E532D531C53FCF7
:1049800052DC52C252A85291525E5231521152EF31
:1049900051C951A251865167514D5133510E51E5C4
:1049A00050CD50A250765040500B50F94FE74FD8A1
:1049B0004FC54FAC4F8A4F784F664F544F424F30E0
:1049C0004F1E4F0C4FFA4EE84ED64EC44EB24EA07C
:1049D0004E8E4E8A4E864E824E7E4E7A4E764E7267
:1049E0004E6E4E6A4E664E624E5E4E5A4E564E5257
:1049F0004E4E4E4A4E464E424E3E4E2A4E0C4EF0C3
:104A00004DC54DA04D7B4D774D734D6F4D6B4D6733
:104A10004D634D5F4D5B4D574D534D4F4D4B4D4786
:104A20004D434D2F4D134DF74CDB4CBF4CA34C87E2
:104A30004C6B4C4F4C334C174CFB4BDF4BDB4BD789
:104A40004BD34BCF4BCB4BC74BC34BAF4B874B6081
:104A50004B3A4B0D4BE74ABA4AB64AB24AAE4A9B6A
:104A60004A7A4A654A4A6F6767696E672063796365
:104A70006C65206661696C65640050726F626520C8
:104A8000656E64706F696E742069732073746172EF
:104A900074696E6720706F696E740050726F626522
:104AA000206379636C65206661696C6564003234EB
:104AB00039003234380032343700486F6D696E6720
:104AC000204572726F72202D20486F6D696E6720CD
:104AD0007377697463686573206D6973636F6E665D
:104AE00069677572656400486F6D696E672045720D
:104AF000726F72202D204E65676174697665206C37
:104B000061746368206261636B6F666600486F6DF5
:104B1000696E67204572726F72202D205472617623
:104B2000656C206D696E2026206D6178206172654C
:104B3000207468652073616D6500486F6D696E67EC
:104B4000204572726F72202D204C6174636820764C
:104B5000656C6F63697479206973207A65726F0080
:104B6000486F6D696E67204572726F72202D2053F9
:104B700065617263682076656C6F6369747920691A
:104B800073207A65726F00486F6D696E6720457299
:104B9000726F72202D20426164206F72206E6F2030
:104BA000617869732073706563696669656400483C
:104BB0006F6D696E67206379636C65206661696CEF
:104BC0006564003233390032333800323337003213
:104BD000333600323335003233340032333300534E
:104BE0006F6674206C696D697420657863656564AF
:104BF0006564202D2043206D617800536F6674201A
:104C00006C696D6974206578636565646564202DE1
:104C10002043206D696E00536F6674206C696D6966
:104C200074206578636565646564202D2042206D7D
:104C3000617800536F6674206C696D6974206578C3
:104C4000636565646564202D2042206D696E0053A4
:104C50006F6674206C696D6974206578636565643E
:104C60006564202D2041206D617800536F667420AB
:104C70006C696D6974206578636565646564202D71
:104C80002041206D696E00536F6674206C696D69F8
:104C900074206578636565646564202D205A206DF5
:104CA000617800536F6674206C696D697420657853
:104CB000636565646564202D205A206D696E00531C
:104CC0006F6674206C696D697420657863656564CE
:104CD0006564202D2059206D617800536F66742023
:104CE0006C696D6974206578636565646564202D01
:104CF0002059206D696E00536F6674206C696D6970
:104D000074206578636565646564202D2058206D86
:104D1000617800536F6674206C696D6974206578E2
:104D2000636565646564202D2058206D696E0053AD
:104D30006F6674206C696D6974206578636565645D
:104D40006564003231390032313800323137003297
:104D500031360032313500323134003231330032F5
:104D600031320032313100323130003230390032EC
:104D7000303800323037003230360054726170659E
:104D80007A6F696420706C616E6E6572206661690D
:104D90006C656420746F20636F6E76657267650062
:104DA0004C696D69742073776974636820686974ED
:104DB000202D2053687574646F776E206F63637560
:104DC00072726564004D616368696E652069732065
:104DD000616C61726D6564202D20436F6D6D616E35
:104DE00064206E6F742070726F6365737365640006
:104DF0004D6F7665206C657373207468616E206DED
:104E0000696E696D756D2074696D65004D6F7665AD
:104E1000206C657373207468616E206D696E696DB6
:104E2000756D206C656E6774680047656E657269A4
:104E3000632054696E7947206572726F7200313950
:104E400039003139380031393700313936003139DC
:104E500035003139340031393300313932003139DC
:104E600031003139300031383900313838003138CB
:104E700037003138360031383500313834003138B8
:104E800033003138320031383100313830005420AD
:104E9000776F726420697320696E76616C69640053
:104EA0005420776F7264206973206D697373696E23
:104EB00067005220776F726420697320696E766193
:104EC0006C6964005220776F7264206973206D6989
:104ED0007373696E67005120776F72642069732065
:104EE000696E76616C6964005120776F7264206925
:104EF00073206D697373696E67004C20776F7264FD
:104F000020697320696E76616C6964004C20776F4C
:104F10007264206973206D697373696E670048203D
:104F2000776F726420697320696E76616C696400C2
:104F30004820776F7264206973206D697373696E9E
:104F400067004520776F726420697320696E76610F
:104F50006C6964004520776F7264206973206D6905
:104F60007373696E67004420776F726420697320E1
:104F7000696E76616C6964004420776F72642069A1
:104F800073206D697373696E67005020776F726468
:104F9000206973206E6F7420612076616C696420D3
:104FA000746F6F6C206E756D626572005020776F44
:104FB0007264206973206E6F7420616E20696E7454
:104FC00065676572005020776F7264206973206E88
:104FD00065676174697665005020776F7264206937
:104FE00073207A65726F005020776F726420697346
:104FF00020696E76616C6964005020776F7264205E
:105000006973206D697373696E6700417263207301
:10501000706563696669636174696F6E2065727239
:105020006F72202D20656E64706F696E74206973D5
:10503000207374617274696E6720706F696E74009A
:105040004172632073706563696669636174696F37
:105050006E206572726F72202D20726164697573A3
:1050600020617263206F7574206F6620746F6C65A9
:1050700072616E6365004172632073706563696677
:1050800069636174696F6E206572726F72202D2082
:105090006D697373696E67206F66667365742873D4
:1050A0002900417263207370656369666963617486
:1050B000696F6E206572726F72202D206D69737337
:1050C000696E67206178697328657329004172638E
:1050D0002073706563696669636174696F6E2065CA
:1050E00072726F72005370696E646C65206D7573B7
:1050F00074206265207475726E696E6720666F72C7
:10510000207468697320636F6D6D616E6400537005
:10511000696E646C65206D757374206265206F66BE
:105120006620666F72207468697320636F6D6D61AD
:105130006E64005370696E646C65205320776F72E3
:105140006420697320696E76616C696400537069CC
:105150006E646C65205320776F7264206973206DD4
:10516000697373696E67005370696E646C65207350
:1051700070656564206578636565646564206D614C
:1051800078696D756D005370696E646C652073701D
:105190006565642062656C6F77206D696E696D75F9
:1051A0006D0050726F6772616D6D656420706F691C
:1051B0006E742073616D6520617320637572726512
:1051C0006E7420706F696E7400437574746572201C
:1051D000636F6D70656E736174696F6E2063616E6D
:1051E0006E6F7420626520656E61626C656400524A
:1051F00065717565737465642076656C6F63697439
:10520000792065786365656473206C696D69747372
:10521000004730206F72204731206D757374206213
:10522000652061637469766520666F722047353347
:1052300000526F7461727920617865732063616ECA
:105240006E6F742062652075736564207769746879
:10525000207468697320636F6D6D616E6400496EC0
:1052600076657273652074696D65206D6F64652065
:1052700063616E6E6F74206265207573656420775C
:10528000697468207468697320636F6D6D616E6402
:10529000004665656472617465206E6F742073707A
:1052A000656369666965640053656C65637465640C
:1052B00020706C616E6520697320696E76616C691F
:1052C000640053656C656374656420706C616E6521
:1052D000206973206D697373696E67004178697323
:1052E0002074617267657420706F736974696F6E82
:1052F00020697320696E76616C6964004178697316
:105300002074617267657420706F736974696F6E61
:10531000206973206D697373696E670041786973E2
:105320002069732064697361626C65640041786907
:105330007320697320696E76616C696420666F7290
:10534000207468697320636F6D6D616E64004178CD
:1053500069732063616E6E6F742062652070726580
:1053600073656E74004178697320776F7264206D85
:10537000697373696E670047636F6465206D6F645E
:10538000616C2067726F75702076696F6C617469EB
:105390006F6E004D20636F646520756E737570705D
:1053A0006F727465640047636F646520636F6D6D31
:1053B000616E6420756E737570706F7274656400D1
:1053C00047656E657269632047636F646520696E27
:1053D000707574206572726F72003132390031322B
:1053E0003800313237003132360031323500313257
:1053F0003400313233003132320031323100313257
:10540000300031313900313138003131370031313C
:105410003600313135004A534F4E2074787420667F
:1054200069656C64732063616E6E6F7420626520C1
:105430006E6573746564004A534F4E2073747269CD
:105440006E6720746F6F206C6F6E67004A534F4E0B
:1054500020696E7075742068617320746F6F206DA1
:10546000616E79207061697273004A534F4E2073E8
:10547000796E746178206572726F7200496E707512
:10548000742076616C75652072616E676520657247
:10549000726F7200496E707574206578636565641B
:1054A00073206D6178696D756D2076616C7565002E
:1054B000496E707574206C657373207468616E201A
:1054C0006D696E696D756D2076616C756500496EEC
:1054D0007075742065786365656473206D617820EC
:1054E0006C656E67746800436F6D6D616E64206EED
:1054F0006F742061636365707465642061742074E7
:105500006869732074696D6500506172616D6574BE
:1055100065722063616E6E6F7420626520726561D2
:105520006400506172616D657465722069732072E8
:105530006561642D6F6E6C7900556E737570706F58
:1055400072746564206E756D626572206F72204A98
:10555000534F4E207479706500426164206E756D02
:1055600062657220666F726D617400496E76616C5F
:105570006964206F72206D616C666F726D65642066
:10558000636F6D6D616E6400556E7265636F676EFB
:10559000697A656420636F6D6D616E64206F72203F
:1055A000636F6E666967206E616D650047656E6545
:1055B00072696320617373657274696F6E206661CE
:1055C000696C757265004D656D6F727920666175E5
:1055D0006C742064657465637465640053746163FE
:1055E0006B206F766572666C6F7720646574656397
:1055F00074656400436F6E74726F6C6C65722061C9
:105600007373657274696F6E206661696C7572651B
:105610000043616E6F6E6963616C206D61636869E0
:105620006E6520617373657274696F6E206661695F
:105630006C75726500506C616E6E6572206173737B
:10564000657274696F6E206661696C75726500536E
:1056500074657070657220617373657274696F6EC2
:10566000206661696C75726500456E636F64657272
:1056700020617373657274696F6E206661696C7501
:10568000726500494F207375622D73797374656D6F
:1056900020617373657274696F6E206661696C75E1
:1056A000726500436F6E666967207375622D73794A
:1056B0007374656D20617373657274696F6E2066B3
:1056C00061696C75726500494F206D656D6F727907
:1056D00020616C6C6F636174696F6E2061737365B8
:1056E0007274696F6E206661696C75726500383816
:1056F0000038370038360038350038340038330089
:105700003832003831003830003739003738003748
:10571000370037360037350037340037330037323B
:105720000037310037300036390036380036370060
:105730003636003635003634003633003632003621
:105740003100363000353900353800353700353610
:105750000035350035340035330035320035310041
:1057600035300034390034380034370034360034F2
:1057700035003434003433003432003431003430F6
:105780000033390033380033370033360042616468
:1057900020737461747573207265706F72742073F6
:1057A000657474696E670050657273697374656EB1
:1057B0006365206572726F7200466C6F6174206958
:1057C00073204E414E00466C6F61742069732069EE
:1057D0006E66696E697465004D6F76652074696DDB
:1057E00065206973204E414E004D6F7665207469C7
:1057F0006D6520697320696E66696E69746500471E
:10580000656E6572696320657863657074696F6E33
:10581000207265706F7274004661696C65642074F3
:105820006F2067657420706C616E6E6572206275A2
:10583000666665720053797374656D20616C617280
:105840006D202D207368757474696E6720646F779E
:105850006E00496E697469616C697A6174696F6E12
:10586000206661696C75726500526561642D6F6EAA
:105870006C79206164647265737300496E76616C43
:105880006964204164647265737300446976696475
:1058900065206279207A65726F00466C6F61746969
:1058A0006E6720706F696E74206572726F72004946
:1058B0006E7465726E616C2072616E6765206572D0
:1058C000726F7200496E7465726E616C20657272DF
:1058D0006F720031390031380046756E6374696F3C
:1058E0006E206973207374756262656400456E741E
:1058F0006572696E6720626F6F74206C6F6164659A
:105900007200496E697469616C697A696E670042F8
:1059100075666665722066756C6C202D20666174F4
:10592000616C004275666665722066756C6C00423B
:10593000756666657220656D707479004E6F2073B0
:1059400075636820646576696365004D61782066DB
:10595000696C652073697A6520657863656564653F
:10596000640046696C65206E6F74206F70656E0010
:10597000456E64206F662066696C6500456E642024
:105980006F66206C696E6500486172642072657391
:105990006574005465726D696E6174656400436F6F
:1059A0006D706C657465004E6F6F70004561676166
:1059B000696E004572726F72004F4B005B70317000
:1059C0006F665D2070776D207068617365206F660B
:1059D000662020202531352E3366205B302E2E3177
:1059E0005D0A005B70317770685D2070776D2063B1
:1059F00063772070686173652068692531352E33BF
:105A000066205B302E2E315D0A005B703177706C42
:105A10005D2070776D206363772070686173652007
:105A20006C6F2531352E3366205B302E2E315D0AAA
:105A3000005B70317773685D2070776D20636377EA
:105A40002073706565642068692531352E306620C5
:105A500052504D0A005B703177736C5D2070776D2A
:105A600020636377207370656564206C6F25313522
:105A70002E30662052504D0A005B70316370685DB5
:105A80002070776D20637720706861736520686986
:105A9000202531352E3366205B302E2E315D0A00F5
:105AA0005B703163706C5D2070776D206377207060
:105AB00068617365206C6F202531352E3366205B5D
:105AC000302E2E315D0A005B70316373685D20708B
:105AD000776D206377207370656564206869202581
:105AE00031352E30662052504D0A005B70316373A1
:105AF0006C5D2070776D206377207370656564201E
:105B00006C6F202531352E30662052504D0A005BD7
:105B100070316672715D2070776D20667265717587
:105B2000656E63792020202531352E306620487A35
:105B30000A0053595354454D205245414459004C95
:105B40006F6164696E6720636F6E66696773206654
:105B5000726F6D20454550524F4D00496E69746912
:105B6000616C697A696E6720636F6E66696773201E
:105B7000746F2053686170656F6B6F322035303001
:105B80006D6D2070726F66696C65007B2265722294
:105B90003A7B226662223A25302E32662C227374BA
:105BA000223A25642C226D7367223A222573227DC6
:105BB0007D0A007B65723A7B66623A25302E32663A
:105BC0002C73743A25642C6D73673A222573227DF9
:105BD0007D0A005B71765D202071756575652072A8
:105BE00065706F727420766572626F73697479255F
:105BF0003764205B303D6F66662C313D73696E679C
:105C00006C652C323D747269706C655D0A00716F51
:105C10003A25640A0071693A25640A0071723A25CE
:105C2000640A005B73765D20207374617475732061
:105C30007265706F727420766572626F73697479C1
:105C4000253664205B303D6F66662C313D66696C9D
:105C500074657265642C323D766572626F73655D42
:105C60000A005B73695D2020737461747573206929
:105C70006E74657276616C2531346C75206D730AB3
:105C8000004D6F746F7220256320706F77657220EE
:105C9000656E61626C65642073746174653A253267
:105CA0002E30660A005B257325735D206D257320F9
:105CB000706F776572206D616E6167656D656E747A
:105CC00025313064205B303D64697361626C6564CA
:105CD0002C313D616C77617973206F6E2C323D6998
:105CE0006E206379636C652C333D7768656E206D3B
:105CF0006F76696E675D0A005B257325735D206DA5
:105D0000257320706F6C6172697479253138642055
:105D10005B303D6E6F726D616C2C313D72657665E6
:105D20007273655D0A005B257325735D206D2573B5
:105D3000206D6963726F73746570732531366420EA
:105D40005B312C322C342C385D0A005B25732573B3
:105D50005D206D25732074726176656C20706572AC
:105D6000207265766F6C7574696F6E2531302E34D4
:105D70006625730A005B257325735D206D257320EE
:105D80007374657020616E676C652532302E3366E2
:105D900025730A005B257325735D206D2573206DC7
:105DA000617020746F206178697325313564205BE0
:105DB000303D582C313D592C323D5A2E2E2E5D0A45
:105DC000005B6D745D20206D6F746F722069646C70
:105DD000652074696D656F75742531342E326620C7
:105DE0005365630A00F45DF05DEB5D206465670058
:105DF000206D6D0020696E005B73745D20207377E9
:105E000069746368207479706525313864205B306B
:105E10003D4E4F2C313D4E435D0A00546573742056
:105E2000232564206E6F7420666F756E640A004EC1
:105E3000312054314D360A4E32204731370A4E3325
:105E4000204732310A4E382046313830300A4E3938
:105E50002047310A4E3130302047393220582D3218
:105E6000352E313737592D33342E303732205A2DD5
:105E7000312E303030202854454D502C2052454D85
:105E80004F5645204C41544552290A4E3334332055
:105E9000582D32352E353935592D33342E3334398A
:105EA0000A4E33343420582D32352E373031592DA7
:105EB00033342E3433360A4E33343520582D3235B0
:105EC0002E373931592D33342E3532300A4E333492
:105ED0003620582D32352E383634592D33342E365F
:105EE00030310A4E33343720582D32352E39323086
:105EF000592D33342E3637390A4E33343820582D45
:105F000032352E393630592D33342E3735340A4E4A
:105F100033343920582D32352E393832592D333417
:105F20002E3832360A4E33353020582D32352E3940
:105F30003837592D33342E3839350A4E3335312020
:105F4000582D32352E393736592D33342E393631D6
:105F50000A4E33353220582D32352E393438592DEA
:105F600033352E3032330A4E33353320582D323507
:105F70002E393033592D33352E3038320A4E3335E1
:105F80003420582D32352E383431592D33352E31B9
:105F900033380A4E33353520582D32352E373633C7
:105FA000592D33352E3139300A4E33353620582DA0
:105FB00032352E363639592D33352E3233390A4E95
:105FC00033353720582D32352E353539592D333567
:105FD0002E3238340A4E33353820582D32352E348F
:105FE0003333592D33352E3332350A4E333539207C
:105FF000582D32352E323931592D33352E33363333
:106000000A4E33363020582D32352E313334592D47
:1060100033352E3339370A4E33363120582D32344A
:106020002E393633592D33352E3432380A4E333625
:106030003220582D32342E373737592D33352E3400
:1060400035350A4E33363320582D32342E35373716
:10605000592D33352E3437370A4E33363420582DE8
:1060600032342E333637592D33352E3439360A4EE5
:1060700033363520582D32342E313434592D3335C2
:106080002E3531310A4E33363620582D32332E39E3
:106090003039592D33352E3532320A4E33363720CA
:1060A000582D32332E363631592D33352E3532397F
:1060B0000A4E33363820582D32332E343033592D92
:1060C00033352E3533320A4E33363920582D32339C
:1060D0002E313333592D33352E3533320A4E333783
:1060E0003020582D32322E383533592D33352E3558
:1060F00032370A2F4E3235313820473058302E3360
:106100003237592D33332E3532315A2D312E30302E
:10611000300A4E32353139204D3330004E31204770
:1061200032300A4E3520473430204731370A4E315D
:1061300030205431204D30360A284E313520473931
:1061400030204730205830205930205A30290A4E0C
:106150003230205335303030204D3033200A4E322B
:10616000352058302E3036342059302E33323620F8
:106170005A300A4E343020473031204631362E30E6
:106180000A4E35302058302E3036342059302E33D8
:1061900032360A4E35352058302E303630205930C0
:1061A0002E3239330A4E36302058302E30373720D1
:1061B00059302E3236370A4E36352058302E31318E
:1061C000312059302E3235370A4E37302058302E94
:1061D0003134392059302E3235320A4E3735205875
:1061E000302E3138382059302E3235350A4E38307D
:1061F0002058302E3232372059302E3236380A4E5F
:1062000038352058302E3235372059302E3237313C
:106210000A4E39302058302E3333352059302E3243
:1062200036350A4E39352058302E34313220593027
:106230002E3237310A4E3130302058302E34373438
:106240002059302E3238370A4E3130352058302E12
:106250003439312059302E3238390A4E313130201C
:1062600058302E3531372059302E3237330A4E31DF
:1062700031352058302E3534342059302E323633D3
:106280000A4E3132302058302E3538302059302ED9
:106290003236310A4E3132352058302E35393520DC
:1062A00059302E3236330A4E3133302058302E36A4
:1062B00032312059302E3237340A4E31333520589E
:1062C000302E3635392059302E3330360A4E31349F
:1062D000302058302E3637332059302E3333350A9C
:1062E0004E3134352058302E3637392059302E3340
:1062F00036310A4E3135302058302E363738205955
:10630000302E3338390A4E3135352058302E363755
:10631000302059302E3432300A4E31363020583049
:106320002E3637302059302E3434360A4E31363539
:106330002058302E3638302059302E3437340A4E1B
:106340003137302058302E3730342059302E343900
:10635000370A4E3137352058302E373332205930F6
:106360002E3531350A4E3138302058302E373934F9
:106370002059302E3533350A4E3138352058302EDD
:106380003837322059302E3536370A4E31393020E1
:1063900058302E3935302059302E3630340A4E31AF
:1063A00039352058312E3033312059302E3634379C
:1063B0000A4E3230302058312E3134392059302EA7
:1063C0003732320A4E3230352058312E33303820B1
:1063D00059302E3835340A4E3231302058312E346F
:1063E00033302059302E3938340A4E323135205866
:1063F000312E3434372059302E3938360A4E323265
:10640000302058312E3632382059302E3832320A68
:106410004E3232352058312E3733322059302E3714
:1064200031340A4E3233302058322E303039205930
:10643000302E3338310A4E3233352058322E313136
:10644000362059302E3236360A4E32343020583209
:106450002E3232382059302E3135370A4E3234350B
:106460002058322E3238302059302E3132330A4EF5
:106470003235302058322E3333322059302E3039D5
:10648000340A4E3235352058322E343233205930CA
:106490002E3037300A4E3236302058322E343839CA
:1064A0002059302E3036350A4E3236352058322EAD
:1064B0003535372059302E3036360A4E32373020B7
:1064C00058322E3632372059302E3038340A4E3278
:1064D00037352058322E3639332059302E31303965
:1064E0000A4E3238302058322E3733302059302E71
:1064F0003133330A4E3238352058322E3830352079
:1065000059302E3139300A4E3239302058322E3837
:1065100032392059302E3231360A4E323935205830
:10652000322E3838302059302E3239310A4E33303D
:10653000302058322E3838342059302E3330300A3B
:106540004E3330352058322E3839382059302E33DA
:1065500033320A4E3331302058322E3930352059FB
:10656000302E3336370A4E3331352058322E3931FA
:10657000302059302E3430370A4E333230205832E2
:106580002E3930382059302E3434360A4E333235D5
:106590002058322E3930312059302E3439350A4EB8
:1065A0003333302058322E3839372059302E343991
:1065B000350A4E3333352058322E38393020593091
:1065C0002E3532340A4E3334302058322E3834329D
:1065D0002059302E3630340A4E3334352058322E7E
:1065E0003831342059302E3636350A4E3335302086
:1065F00058322E3739342059302E3735300A4E3341
:1066000035352058322E3739312059302E3833382D
:106610000A4E3336302058322E3831392059302E38
:106620003937360A4E3336352058322E3833372034
:1066300059312E3034340A4E3337302058322E3808
:1066400036322059312E3131320A4E333735205807
:10665000322E3837372059312E3134350A4E3338FF
:10666000302058322E3931322059312E3231370A0A
:106670004E3338352058322E3931372059312E32A9
:1066800032360A4E3339302058322E3935312059BE
:10669000312E3238310A4E3339352058322E3937BF
:1066A000302059312E3239350A4E343030205832AC
:1066B0002E3939362059312E3239350A4E3430359B
:1066C0002058332E3031332059312E3237350A4E8F
:1066D0003431302058332E3032342059312E323577
:1066E000340A4E3431352058332E3037302059316A
:1066F0002E3135310A4E3432302058332E30373770
:106700002059312E3133340A4E3432352058332E4D
:106710003132352059312E3033390A4E343330205E
:1067200058332E3133382059312E3031390A4E3416
:1067300033352058332E3230352059302E39303809
:106740000A4E3434302058332E3238322059302E0D
:106750003739370A4E3434352058332E333631200A
:1067600059302E3639310A4E3435302058332E34D4
:1067700032362059302E3539320A4E3435352058CC
:10678000332E3435362059302E3534330A4E3436D4
:10679000302058332E3437392059302E3439330ACB
:1067A0004E3436352058332E3439342059302E3477
:1067B00037320A4E3437302058332E353035205991
:1067C000302E3434360A4E3437352058332E353196
:1067D000382059302E3431370A4E3438302058336F
:1067E0002E3533302059302E3339310A4E34383576
:1067F0002058332E3536342059302E3330300A4E5F
:106800003439302058332E3537372059302E323531
:10681000330A4E3439352058332E35363820593026
:106820002E3231320A4E3530302058332E35343442
:106830002059302E3137360A4E3530352058332E18
:106840003534312059302E3134360A4E353130202E
:1068500058332E3535332059302E3131390A4E35E3
:1068600031352058332E3537362059302E313036D9
:106870000A4E3532302058332E3539372059302ED4
:106880003130320A4E3532352058332E36313820E9
:1068900059302E3130390A4E3533302058332E36A8
:1068A00033392059302E3132390A4E35333520589C
:1068B000332E3635302059302E3135390A4E3534A5
:1068C000302058332E3636332059302E3137380A9F
:1068D0004E3534352058332E3637382059302E3146
:1068E00039320A4E3535302058332E363939205951
:1068F000302E3139370A4E3535352058332E373260
:10690000332059302E3139360A4E3536302058333F
:106910002E3736342059302E3137390A4E35363538
:106920002058332E3830352059302E3136350A4E26
:106930003537302058332E3838342059302E313501
:10694000390A4E3537352058332E393439205930ED
:106950002E3136350A4E3538302058332E393636FA
:106960002059302E3137350A4E3538352058332EE0
:106970003937382059302E3139340A4E35393020E4
:1069800058332E3937382059302E3232330A4E35AB
:1069900039352058332E3936302059302E3234359F
:1069A0000A4E3630302058332E3833342059302EAA
:1069B0003331310A4E3630352058332E37363220B7
:1069C00059302E3334350A4E3631302058332E3775
:1069D00032362059302E3338390A4E363135205868
:1069E000332E3730332059302E3435380A4E363274
:1069F000302058332E3638322059302E3533300A75
:106A00004E3632352058332E3637392059302E3510
:106A100033340A4E3633302058332E36323620592E
:106A2000302E3638310A4E3633352058332E35362F
:106A3000382059302E3832380A4E36343020583308
:106A40002E3434342059312E3038300A4E36343515
:106A50002058332E3430352059312E3136370A4EF6
:106A60003635302058332E3430342059312E3136DB
:106A7000370A4E3635352058332E333837205931C2
:106A80002E3230380A4E3636302058332E333834D2
:106A90002059312E3230380A4E3636352058332EB2
:106AA0003336352059312E3236350A4E36373020BE
:106AB00058332E3335352059312E3238350A4E367B
:106AC00037352058332E3334382059312E3330386F
:106AD0000A4E3638302058332E3333332059312E76
:106AE0003335300A4E3638352058332E3332312084
:106AF00059312E3339310A4E3639302058332E333E
:106B000031312059312E3432380A4E363935205839
:106B1000332E3333392059312E3432330A4E373045
:106B2000302058332E3434302059312E3430360A48
:106B30004E3730352058332E3531302059312E34F0
:106B400030380A4E3731302058332E3538352059F9
:106B5000312E3432310A4E3731352058332E36310A
:106B6000312059312E3433390A4E373230205833E0
:106B70002E3631312059312E3434310A4E373235E8
:106B80002058332E3631352059312E3434310A4EC7
:106B90003733302058332E3633362059312E34389F
:106BA000380A4E3733352058332E36333420593196
:106BB0002E3531370A4E3734302058332E363232A4
:106BC0002059312E3534330A4E3734352058332E80
:106BD0003630352059312E3536330A4E3735302090
:106BE00058332E3537362059312E3537350A4E3742
:106BF00035352058332E3534342059312E3538313F
:106C00000A4E3736302058332E3437392059312E3A
:106C10003539320A4E3736352058332E3435312047
:106C200059312E3539380A4E3737302058332E3304
:106C300038372059312E3632360A4E3737352058FC
:106C4000332E3339302059312E3633360A4E373809
:106C5000302058332E3533322059312E3630320A17
:106C60004E3738352058332E3630312059312E35B5
:106C700039370A4E3739302058332E3636382059B6
:106C8000312E3539380A4E3739352058332E3738BA
:106C9000322059312E3631320A4E383030205833B6
:106CA0002E3739342059312E3631380A4E383035A6
:106CB0002058332E3836382059312E3633360A4E86
:106CC0003831302058332E3931382059312E36356D
:106CD000350A4E3831352058332E39343520593164
:106CE0002E3636370A4E3832302058332E39363465
:106CF0002059312E3638350A4E3832352058332E49
:106D00003936372059312E3638350A4E383330204F
:106D100058332E3937342059312E3639390A4E3806
:106D200033352058332E3938342059312E37323507
:106D30000A4E3834302058332E3938342059312E09
:106D40003735380A4E3834352058332E393730200D
:106D500059312E3739300A4E3835302058332E39D4
:106D600034352059312E3831370A4E3835352058D0
:106D7000332E3931382059312E3832360A4E3836D2
:106D8000302058332E3839312059312E3832370AD5
:106D90004E3836352058332E3834322059312E387B
:106DA00030390A4E3837302058332E373938205989
:106DB000312E3738340A4E3837352058332E373491
:106DC000362059312E3737320A4E38383020583372
:106DD0002E3639382059312E3736340A4E38383568
:106DE0002058332E3633352059312E3736360A4E59
:106DF0003839302058332E3535332059312E373835
:106E0000350A4E3839352058332E34373820593129
:106E10002E3832300A4E3930302058332E34303943
:106E20002059312E3836340A4E3930352058332E19
:106E30003334352059312E3931380A4E393130202A
:106E400058332E3236342059322E3032330A4E39EE
:106E500031352058332E3234382059322E303531E6
:106E60000A4E3932302058332E3234302059322EE7
:106E70003038310A4E3932352058332E33313620EE
:106E800059322E3038360A4E3933302058332E33AB
:106E900039302059322E3130340A4E3933352058AA
:106EA000332E3431342059322E3132310A4E3934B6
:106EB000302058332E3433312059322E3135330AB5
:106EC0004E3934352058332E3433332059322E3155
:106ED00038300A4E3935302058332E343237205965
:106EE000322E3230350A4E3935352058332E343172
:106EF000332059322E3232340A4E3936302058334C
:106F00002E3339322059322E3234320A4E39363548
:106F10002058332E3333352059322E3234340A4E32
:106F20003937302058332E3237382059322E323309
:106F3000360A4E3937352058332E323536205932FD
:106F40002E3234320A4E3938302058332E3233390B
:106F50002059322E3235310A4E3938352058332EE9
:106F60003231312059322E3238300A4E3939302000
:106F700058332E3137342059322E3335360A4E39B4
:106F800039352058332E3135392059322E3339379F
:106F90000A4E313030302058332E313530205932BE
:106FA0002E3433380A4E313030352058332E3134B8
:106FB000302059322E3438310A4E31303130205899
:106FC000332E3133322059322E3531300A4E3130A2
:106FD00031352058332E3131382059322E35343363
:106FE0000A4E313032302058332E30393920593260
:106FF0002E3537360A4E313032352058332E303563
:10700000312059322E3633310A4E31303330205848
:10701000332E3030332059322E3636360A4E313048
:1070200033352058322E3935372059322E363835FF
:107030000A4E313034302058322E39303720593210
:107040002E3639390A4E313034352058322E383602
:10705000302059322E3731310A4E313035302058F8
:10706000322E3831392059322E3732370A4E3130EC
:1070700035352058322E3736382059322E373435B0
:107080000A4E313036302058322E373136205932C0
:107090002E3735370A4E313036352058322E3637B6
:1070A000352059322E3735370A4E31303730205897
:1070B000322E3537392059322E3733310A4E31309E
:1070C00037352058322E3537302059322E3732336B
:1070D0000A4E313038302058322E35353920593269
:1070E0002E3732300A4E313038352058322E353373
:1070F000302059322E3730310A4E31303930205855
:10710000322E3530312059322E3639330A4E313055
:1071100039352058322E3437312059322E36383313
:107120000A4E313130302058322E34343320593227
:107130002E3636380A4E313130352058322E33391A
:10714000362059322E3633340A4E31313130205800
:10715000322E3335342059322E3539310A4E313101
:1071600031352058322E3335322059322E353931CF
:107170000A4E313132302058322E333235205932D6
:107180002E3534330A4E313132352058322E3331D8
:10719000352059322E3532310A4E313133302058B4
:1071A000322E3330372059322E3439380A4E3131AD
:1071B00033352058322E3239362059322E34363477
:1071C0000A4E313134302058322E32393320593280
:1071D0002E3432370A4E313134352058322E32397E
:1071E000352059322E3336360A4E3131353020585B
:1071F000322E3332312059322E3330330A4E313170
:1072000035352058322E3335382059322E32343726
:107210000A4E313136302058322E3431392059322D
:107220002E3230330A4E313136352058322E343139
:10723000392059322E3137390A4E31313730205802
:10724000322E3430352059322E3135380A4E313114
:1072500037352058322E3336322059322E313233E0
:107260000A4E313138302058322E333534205932DD
:107270002E3130340A4E313138352058322E3335E4
:10728000342059322E3039310A4E313139302058BC
:10729000322E3338302059322E3036350A4E3131C5
:1072A00039352058322E3431302059322E30353194
:1072B0000A4E313230302058322E3431302059329B
:1072C0002E3034370A4E313230352058322E343099
:1072D000352059322E3032380A4E31323130205872
:1072E000322E3430382059322E3031300A4E31327D
:1072F00031352058322E3431362059312E39393536
:107300000A4E313232302058322E34333320593144
:107310002E3938320A4E313232352058322E34333B
:10732000382059312E3936330A4E31323330205815
:10733000322E3434372059312E3934380A4E313216
:1073400033352058322E3436312059312E393338E6
:107350000A4E313234302058322E343830205931F0
:107360002E3933310A4E313234352058322E3437EB
:10737000382059312E3839390A4E313235302058BB
:10738000322E3438372059312E3837350A4E3132C3
:1073900035352058322E3530342059312E38353499
:1073A0000A4E313236302058322E3532372059319C
:1073B0002E3834380A4E313236352058322E353494
:1073C000392059312E3834390A4E3132373020586D
:1073D000322E3537372059312E3836310A4E313278
:1073E00037352058322E3630342059312E38363643
:1073F0000A4E313238302058322E3633312059314E
:107400002E3835340A4E313238352058322E363443
:10741000302059312E3832370A4E31323930205827
:10742000322E3634302059312E3739320A4E31322D
:1074300039352058322E3632392059312E373539E8
:107440000A4E313330302058322E36313220593105
:107450002E3732370A4E313330352058322E3537F9
:10746000362059312E3639340A4E313331302058D6
:10747000322E3533362059312E3636320A4E3133DC
:1074800031352058322E3437302059312E363136AE
:107490000A4E313332302058322E333435205931B0
:1074A0002E3535310A4E313332352058322E3330B5
:1074B000372059312E3532310A4E3133333020588E
:1074C000322E3236302059312E3438320A4E313392
:1074D00033352058322E3234332059312E34373759
:1074E0000A4E313334302058322E3232382059315E
:1074F0002E3436390A4E313334352058322E32325A
:10750000322059312E3434380A4E31333530205838
:10751000322E3232382059312E3432350A4E313340
:1075200035352058322E3235342059312E3430350D
:107530000A4E313336302058322E32363820593107
:107540002E3337330A4E313336352058322E323708
:10755000392059312E3334320A4E313337302058E6
:10756000322E3330382059312E3238370A4E3133EB
:1075700037352058322E3334302059312E323534BD
:107580000A4E313338302058322E343037205931BA
:107590002E3230310A4E313338352058322E3434C1
:1075A000312059312E3135360A4E31333930205899
:1075B000322E3435342059312E3133310A4E3133A5
:1075C00039352058322E3436302059312E3130366C
:1075D0000A4E313430302058322E3436342059316E
:1075E0002E3130320A4E313430352058322E343775
:1075F000312059312E3033360A4E31343130205853
:10760000322E3436362059302E3937310A4E313445
:1076100031352058322E3435312059302E38393713
:107620000A4E313432302058322E34313520593020
:107630002E3739310A4E313432352058322E34301B
:10764000332059302E3736370A4E313433302058F4
:10765000322E3338382059302E3736350A4E3134F1
:1076600033352058322E3330362059302E383431CD
:107670000A4E313434302058322E323232205930D2
:107680002E3931310A4E313434352058322E3131D1
:10769000342059302E3939350A4E3134353020589E
:1076A000322E3030322059312E3037360A4E3134B6
:1076B00035352058312E3930352059312E31333976
:1076C0000A4E313436302058312E37353420593176
:1076D0002E3232330A4E313436352058312E36337D
:1076E000372059312E3237380A4E3134373020584E
:1076F000312E3538322059312E3330310A4E313463
:1077000037352058312E3535382059312E33313523
:107710000A4E313438302058312E34363020593129
:107720002E3335320A4E313438352058312E333924
:10773000392059312E3336300A4E31343930205801
:10774000312E3333382059312E3335340A4E31340B
:1077500039352058312E3238372059312E333239CD
:107760000A4E313530302058312E323438205931DC
:107770002E3239340A4E313530352058312E3231DF
:10778000372059312E3235340A4E313531302058B8
:10779000312E3231342059312E3235320A4E3135C4
:1077A00031352058312E3137322059312E3139358B
:1077B0000A4E313532302058312E3132382059318D
:1077C0002E3133390A4E313532352058312E313190
:1077D000302059312E3131370A4E3135333020586F
:1077E000302E3935382059302E3934310A4E313562
:1077F00033352058302E3839312059302E38373330
:107800000A4E313534302058302E38323520593038
:107810002E3830380A4E313534352058302E373531
:10782000352059302E3734370A4E3135353020580F
:10783000302E3631392059302E3633330A4E313519
:1078400035352058302E3437372059302E353236E2
:107850000A4E313536302058302E343737205930E3
:107860002E3532340A4E313536352058302E3431EB
:10787000312059302E3437360A4E313537302058C2
:10788000302E3333312059302E3435340A4E3135D1
:1078900037352058302E3237382059302E34323791
:1078A0000A4E313538302058302E3233312059309D
:1078B0002E3339370A4E313538352058302E31388D
:1078C000332059302E3337390A4E3135393020586C
:1078D000302E3133352059302E3336350A4E31357E
:1078E00039352058302E3037362059302E33343148
:1078F0000A4E3136303520473030204633302E3076
:107900000A4E31363130204D3035200A4E31363175
:107910003520473930205830205930205A300A4E0F
:1079200031363135204D33300A28456E64206F667C
:1079300020434E432050726F6772616D2900284DBD
:1079400053472A2A2A2A204D6963726F737465701F
:107950002054657374205B76315D202A2A2A2A29F7
:107960000A47303020473137204732312047343002
:107970002047343920473830204739300A6730787B
:107980003079307A300A7B22316D69223A317D0AB2
:107990007B22326D69223A317D0A7B22336D692266
:1079A0003A317D0A7B22346D69223A317D0A673093
:1079B000207831300A7B22316D69223A327D0A7893
:1079C000300A7B22316D69223A347D0A7831300ADF
:1079D0007B22316D69223A387D0A78300A6730207F
:1079E0007931300A7B22326D69223A327D0A793050
:1079F0000A7B22326D69223A347D0A7931300A7B62
:107A000022326D69223A387D0A79300A6730207A4D
:107A100031300A7B22336D69223A327D0A7A300A8C
:107A20007B22336D69223A347D0A7A31300A7B2217
:107A3000336D69223A387D0A7A300A673020613125
:107A4000300A7B22346D69223A327D0A61300A7B2A
:107A500022346D69223A347D0A6131300A7B223446
:107A60006D69223A387D0A61300A6D3200284D5323
:107A7000472A2A2A2A20436F6F7264696E617465EF
:107A8000206F6666736574732074657374205B760B
:107A9000315D202A2A2A2A290A6730306731376760
:107AA00032316734306734396738306739300A67C4
:107AB00035340A673932783079307A300A663630B0
:107AC000300A284D53472A2A2A2A207465737420C5
:107AD000473932206F6666736574732A2A2A2A2909
:107AE0000A286D73675374657020313A204D6F76A4
:107AF000652066726F6D20302C3020746F2033301B
:107B00002C30206D6D20696E20706F7369746976FA
:107B100065205820646972656374696F6E290A284C
:107B20006D73675374657020323A205265736574C3
:107B3000206F726967696E20746F20302E30207557
:107B400073696E6720473932290A286D7367537449
:107B5000657020333A204D6F766520746F20323087
:107B60002C302E2053686F756C64206D6F76652005
:107B70003230206D6D20696E20706F736974697684
:107B800065205820646972656374696F6E20616E48
:107B90006420737461747573207265706F727420E1
:107BA00073686F756C642073746172742066726F91
:107BB0006D20302C30290A286D736753746570204E
:107BC000343A204D6F766520746F20302E3020209F
:107BD0002053686F756C64206D6F7665203230209D
:107BE0006D6D20696E206E656761746976652058D9
:107BF00020646972656374696F6E20616E642073BE
:107C00007461747573207265706F72742073686F1D
:107C1000756C642073746172742066726F6D2032AB
:107C2000302C30290A67317833300A67393278309E
:107C30000A67317832300A6731783079300A247334
:107C4000720A67393278300A673470302E350A2864
:107C50004D53472A2A2A2A207465737420473535E4
:107C6000206F6666736574732A2A2A2A290A286D8A
:107C700073675374657020313A2053657420436FE5
:107C80006F7264696E6174652073797374656D20B9
:107C900032205B6735355D20746F206F66667365D3
:107CA00074206F662035302C3530290A286D7367B3
:107CB0005374657020323A2053656C6563742047B5
:107CC000353520636F6F7264696E617465207379F6
:107CD0007374656D290A286D73675374657020335A
:107CE0003A204D6F766520746F20302C302E20485E
:107CF0006561642073686F756C64206D6F766520B4
:107D0000646961676F6E616C6C7920696E202B58B5
:107D100020616E64202B5920616E6420737461743D
:107D20007573207265706F72742073686F756C6400
:107D30002073746172742066726F6D20302C30294C
:107D40000A6731304C3270327835307935300A6715
:107D500035350A6730783079300A673470302E351F
:107D60000A284D53472A2A2A2A207465737420470B
:107D70003533206162736F6C757465206F76657240
:107D80007269646573202A2A2A2A290A286D736772
:107D90005374657020313A2052756E2061207371E2
:107DA0007561726520696E2047353520737973746B
:107DB000656D290A286D73675374657020323A2007
:107DC00052756E20612073717561726520772F473F
:107DD0003533206F76657272696465290A67307879
:107DE0003079300A673078323079300A673078324B
:107DF000307932300A673078307932300A6730783B
:107E00003079300A673470302E350A673533673081
:107E1000783079300A673533673078323079300A14
:107E200067353367307832307932300A67353367F7
:107E30003078307932300A673533673078307930CE
:107E40000A6730783079300A673470302E350A2866
:107E50004D53472A2A2A2A20746573742052657468
:107E600075726E20746F20686F6D65202A2A2A2A29
:107E7000290A286D73675374657020313A20526562
:107E80007475726E20746F20686F6D6520757369EC
:107E90006E6720473238290A286D736753746570FE
:107EA00020323A20526573657420746F2047353450
:107EB00020636F6F72642073797374656D290A672C
:107EC00032380A6735340A6D333000284D53472A5B
:107ED0002A2A2A2054657374206163637572616372
:107EE00079206F6620736C6F77206D6F76657320D5
:107EF0005B76315D202A2A2A2A290A6735350A67E6
:107F000030783079300A673470302E350A67347033
:107F1000302E350A67317831306632320A673534AF
:107F20000A6730783079300A6D333000284D534776
:107F30002A2A2A2A20546573742076657279207360
:107F4000686F7274206D6F766573205B76315D208B
:107F50002A2A2A2A290A6730783079300A67347049
:107F6000302E350A673178302E3166313030300AA4
:107F700078300A78302E310A78300A78302E310A7B
:107F800078300A78302E310A78300A78302E310A6B
:107F900078300A78302E310A78300A78302E310A5B
:107FA00078300A78302E310A78300A78302E310A4B
:107FB00078300A78302E310A78300A78302E310A3B
:107FC00078300A78302E310A78300A78302E310A2B
:107FD00078300A78302E310A78300A78302E310A1B
:107FE000673470302E350A78300A78302E30310AF6
:107FF00078300A78302E30310A78300A78302E30D6
:10800000310A78300A78302E30310A78300A7830E8
:108010002E30310A78300A78302E30310A78300A22
:1080200078302E30310A78300A78302E30310A78A4
:10803000300A78302E30310A78300A78302E3031DC
:108040000A78300A78302E30310A78300A78302EAB
:1080500030310A78300A78302E30310A78300A7898
:10806000302E30310A6730783079300A6D3200288E
:108070004D53472A2A2A2A20526F7461727920416F
:10808000786973204D6F74696F6E20546573742026
:108090005B76315D202A2A2A2A290A673030673127
:1080A0003767323167343067343967383067393091
:1080B0000A6730783079307A306130623063300A64
:1080C0006735350A6730783079300A6633363030B4
:1080D000300A6730613336300A623336300A633330
:1080E00036300A61300A62300A63300A6731613122
:1080F0003434300A62313434300A63313434300A73
:1081000061300A62300A63300A67316131343430D9
:1081100062373230633336300A783079307A306102
:1081200030623063300A6731783630613134343050
:1081300062373230633336300A783079307A3061E2
:1081400030623063300A67317836307935306131EA
:1081500034343062373230633336300A7830793035
:108160007A306130623063300A6731783630793581
:1081700030783235613134343062373230633336FF
:10818000300A783079307A306130623063300A6793
:1081900035340A6730783079300A6D333000284D35
:1081A00053472A2A2A2A20496E766572736520541D
:1081B000696D65204D6F74696F6E2054657374200E
:1081C0005B76315D202A2A2A2A290A6730306731F6
:1081D0003767323167343067343967383067393060
:1081E0000A6735350A6730783079300A6739330ADB
:1081F00066302E30310A67317831300A7931300AF1
:108200007A31300A6131300A78300A79300A7A30AE
:108210000A61300A67317831307931307A2D313066
:108220006131300A6730783079307A3061300A66EF
:10823000302E310A6732783130792D31307A2D3253
:10824000306931300A6730783079307A300A6733F4
:10825000783130792D31307A2D32306931300A67FA
:1082600030783079307A300A673278323079307A43
:108270002D32306931300A6730783079307A300AFF
:10828000673378323079306931300A673078307945
:10829000307A300A6732783079307A2D333069316C
:1082A000300A6733783079307A306931300A673094
:1082B000783079307A300A67327830793069323004
:1082C0002028435720333630206465677265657314
:1082D000290A673378307930693230202843435790
:1082E000203336302064656772656573290A673903
:1082F000340A6735340A6730783079300A6D3330A4
:10830000007B226763223A22673030673137673259
:1083100031673430673439673830673930227D0A45
:108320007B226763223A22673535227D0A7B2267EA
:1083300063223A22673078307930227D0A7B2267C7
:1083400063223A2266353030227D0A7B226763221F
:108350003A22284D53477371756172657329227DE6
:108360000A7B226763223A226730783230227D0A04
:108370007B226763223A22793230227D0A7B226790
:1083800063223A227830227D0A7B226763223A22D6
:108390007930227D0A7B226763223A226731783165
:1083A00030227D0A7B226763223A22793130227D96
:1083B0000A7B226763223A227830227D0A7B226779
:1083C00063223A227930227D0A7B226763223A2295
:1083D000284D5347636972636C657329227D0A7B5C
:1083E000226763223A226732783130792D31306941
:1083F0003130227D0A7B226763223A22673078304F
:108400007930227D0A7B226763223A2267337831F2
:1084100030792D3130693130227D0A7B2267632229
:108420003A22673078307930227D0A7B22676322D6
:108430003A2267327832307930693130227D0A7BD6
:10844000226763223A22673078307930227D0A7BB6
:10845000226763223A2267337832307930693130CB
:10846000227D0A7B226763223A2267307830793096
:10847000227D0A7B226763223A2267327830793084
:10848000693130227D0A7B226763223A2267337882
:10849000307930693130227D0A7B226763223A22AB
:1084A000673534227D0A7B226763223A226730785F
:1084B000307930227D0A7B226763223A226D333085
:1084C000227D00284D53472A2A2A2A204D636F64B3
:1084D00065732074657374205B76315D202A2A2AC7
:1084E0002A290A6735350A6730783079300A6D33C2
:1084F0000A673470310A6D350A673470310A6D3499
:108500000A673470310A6D350A673470310A6D3785
:108510000A673470310A6D390A673470310A6D3870
:108520000A673470310A6D390A663530300A6730AF
:108530007832300A7932300A6D330A78300A6D3475
:108540000A79300A6D350A67317831300A6D370A99
:108550007931300A6D380A78300A6D390A79300A73
:108560006732783130792D31306931300A6D330A14
:108570006730783079300A6D340A67337831307972
:108580002D31306931300A6D350A673078307930F5
:108590000A6D370A673278323079306931300A6DC6
:1085A000380A6730783079300A6D390A67337832A3
:1085B0003079306931300A6730783079300A673283
:1085C000783079306931300A673378307930693101
:1085D000300A6735340A6730783079300A6D3330C5
:1085E00000284D53472A2A2A2A2046656564686F69
:1085F0006C642054657374205B76315D202A2A2ACE
:108600002A290A284D53472A2A2A2A204D616E75A5
:10861000616C6C7920656E746572202120616E64D6
:10862000207E20647572696E67206D6F76656D655A
:108630006E7420746F2074657374202A2A2A2A2984
:108640000A6735350A6730783079300A6734703315
:108650000A67303067313767323167343067343911
:108660006738306739300A663630300A673078311B
:1086700030307637362E3736350A783079300A671B
:1086800035340A6730783079300A6D333000284D40
:1086900053472A2A2A2A204477656C6C2054657334
:1086A00074205B76315D202A2A2A2A290A67303015
:1086B0006731376732316739300A6735350A6730D5
:1086C000783079300A663530300A67307831300AD0
:1086D000673470310A67307832300A673470310A93
:1086E00067307831300A673470310A67307830305B
:1086F0000A673470310A79350A6735340A67307889
:108700003079300A6D330A673470310A6730783156
:10871000307931300A6D350A673470310A67307844
:1087200032307932300A6D340A673470310A67307A
:108730007833307933300A6D380A673470310A671C
:10874000307834307934300A6D390A673470310A40
:1087500067307835307935300A6730783079300ACB
:108760006D3330004E31206730306731376732313A
:108770006734306734396738306739300A4E313002
:10878000206730783079300A4E323020663530300C
:108790000A4E3330206732783130792D31306931EB
:1087A0003020284357203237302064656772656572
:1087B00073290A4E3430206730783079300A4E35CC
:1087C00030206733783130792D31306931302028CD
:1087D0004343572039302064656772656573290A01
:1087E0004E3630206730783079300A4E3830206786
:1087F000327832307930693130202843572031388F
:10880000302064656772656573290A4E37302067CA
:1088100030783079300A4E3830206733783230790A
:108820003069313020284343572031383020646587
:108830006772656573290A4E393020673078307960
:10884000300A4E39392046313230300A4E3130301C
:10885000206732783079306932302028435720330E
:1088600036302064656772656573290A4E31313090
:1088700020673278307930693230202843572033EE
:10888000363020616761696E290A4E3132302066C8
:1088900037303020284368616E67652066656564FF
:1088A0002072617465207768696C6520696E204765
:1088B00032206D6F74696F6E206D6F6465290A4E8A
:1088C00031333020673278307930693230202843B4
:1088D0005720333630203372642074696D65290A5D
:1088E0004E31343020673278307930693230202888
:1088F000435720333630203474682074696D6529FD
:108900000A4E31353020663530300A4E313630204F
:108910006733783079307A343069323020284343F5
:108920005720333630206465677265657320776938
:108930007468206C696E6561722074726176656C12
:10894000290A4E313730206733783079307A3069F0
:108950003230202843435720333630206167616925
:108960006E290A4E313830206637303020286D733A
:10897000672A2A2A2A4368616E67652066656564EE
:108980002072617465207768696C6520696E204784
:1089900033206D6F74696F6E206D6F64652A2A2AAB
:1089A0002A290A4E313930206733783079306932DC
:1089B00030202843435720333630203372642074EC
:1089C000696D65290A4E323030206733783079304E
:1089D00069323020284343572033363020347468BE
:1089E0002074696D65290A4E32313020286D736715
:1089F0002A2A2A2A473138204576616C207465730B
:108A0000742A2A2A2A290A4E323230204731205825
:108A100033302E373037205A35302E373237204614
:108A20003530300A4E32333020473138204730322B
:108A3000205836372E373338205A32332E363137D6
:108A40002052323520463235300A4E3234302067DB
:108A500038300A4E323530206730783079307A300D
:108A60000A4E323630206D333000284D53472A2AC3
:108A70002A2A2053717561726573204D6F74696F76
:108A80006E2054657374205B76315D202A2A2A2A71
:108A9000290A6730306731376732316734306734DD
:108AA000396738306739300A6730783079300A678B
:108AB0003078323020287472617665727365206177
:108AC0002032306D6D2073717561726520696E2082
:108AD0005820616E642059290A7932300A78300AA8
:108AE00079300A6731783130663530302028647249
:108AF000617720612031306D6D2073717561726511
:108B000020696E205820616E6420592061742046CF
:108B1000353030290A7931300A78300A79300A67DD
:108B2000307A323020287472617665727365206104
:108B30002032306D6D2073717561726520696E2011
:108B40005820616E64205A290A7832300A7A300A35
:108B500078300A67317832307932307A323066359F
:108B6000303020286665656420612032306D6D20CC
:108B7000646961676F6E616C20696E20582C2059A2
:108B800020616E64205A290A783079307A300A7868
:108B900034307934307A34302028747261766572DA
:108BA000736520612034306D6D20637562652069C6
:108BB0006E20582C205920616E64205A290A78347E
:108BC0003079307A300A78307934307A34300A7833
:108BD00034307934307A300A783079307A34300A67
:108BE00078307934307A300A78343079307A3430E9
:108BF0000A783079307A300A6738300A673078304E
:108C000079300A673078310A673078300A6D33304E
:108C100000284D53472A2A2A2A20486F6D696E671B
:108C20002054657374205B76315D202A2A2A2A2914
:108C30000A6732382E32783079307A300A6D333024
:108C400000284D53472A2A2A2A20536D6F6B65202E
:108C500054657374205B76315D202A2A2A2A290AFA
:108C600047303020473137204732312047343020D9
:108C700047343920473830204739300A6D3367345C
:108C800070310A6D35673470310A6D346734703174
:108C90000A6D33673470310A6D35673470310A6D8F
:108CA00037673470310A6D39673470310A6D38674F
:108CB0003470310A6D390A6730783079307A300A89
:108CC000673030207832300A78300A7932300A79C9
:108CD000300A7A32300A7A300A6132300A61300A58
:108CE0004730302078323020793230207A323020CC
:108CF0006132300A473030207830207930207A30A5
:108D00002061300A473031206633302078322079B4
:108D100032207A322061320A7830207930207A305D
:108D20002061300A673078310A673078300A6D3256
:108D3000005B74765D2020746578742076657262BD
:108D40006F7369747925313564205B303D73696CCC
:108D5000656E742C313D766572626F73655D0A00D5
:108D600025660A00256C750A0025730A0074696E71
:108D70007967205B25735D206572723A2025733A0E
:108D8000202573200074696E7967205B25735D2050
:108D90006F6B3E2000456E64206F6620636F6D6DC3
:108DA000616E642066696C650A0027C9C9C694C9EA
:108DB000B5C914CA0EC7ECCCC9C680CDECCD1ACC4F
:108DC0000EC70000400640061040B800B8ECCCC901
:108DD000C680CDECCD1ACC0EC70000400620060898
:108DE00040B800B855CFC9C675CEF1CEA0D03ECEA2
:108DF000A0084006050609010855CFC9C675CEF181
:108E0000CE26CA0EC7B00840060540B0308000002C
:108E1000000000F0E0D0C0100100CF673322211F16
:108E20001B1301016E616E00696E66004E414E4972
:108E30004E495459494E46CDCCCC3D0AD7233C1718
:108E4000B7D13877CC2B329595E6241FB14F0A0065
:108E50000020410000C84200401C4620BCBE4CCA55
:108E60001B0E5AAEC59D7400407A10F35A00A072D2
:108E70004E18090010A5D4E80000E8764817000055
:108E8000E40B54020000CA9A3B000000E1F5050023
:108E90000080969800000040420F000000A086016C
:108EA000000000102700000000E80300000000643C
:108EB00000000000000A00000000000100000000A7
:108EC000002C76D888DC674F0823DFC1DFAE59E17C
:108ED000B1B796E5E3E453C63AE651997696E8E6EB
:108EE000C28426EB898C9B62ED407C6FFCEFBC9CBE
:108EF0009F40F2BAA56FA5F490055A2AF75C936BD0
:108F00006CF9676DC11BFCE0E40D47FEF520E6B58A
:108F100000D0ED902E0300943577050080841E0864
:108F20000000204E0A000000C80C333333330F9882
:108F30006E12831141EF8D2114893BE65516CFFE49
:108F4000E6DB18D1844B381BF77C1D901DA4BBE4D5
:108F500024203284725E228100C9F124ECA1E53D17
:108F6000270011241FBECFEFCDBFDFE5DEBF00E03D
:108F70000CBF13E2A0E0B0E2E4E8F8EC01E00BBFC4
:108F800002C007900D92AA38B107D9F72EE5AAE8DA
:108F9000B3E201C01D92A636B207E1F70E9400823B
:108FA0000C9440E40C940000FC016081718182818A
:108FB00093810E94EED5609333370895FC01608160
:108FC0007181828193810E94EED56093323708953A
:108FD000AF92BF92CF92DF92EF92FF920F931F93C7
:108FE000CF93DF937B018C0186EBC82E86E3D82ECE
:108FF000E601AA24A394BC2EBC18F70161917191DB
:10900000819191917F012CEA35EC47E257E30E9470
:109010007DD718164CF4F80140815181628173812B
:109020008B2D0E942F83A8820C5F1F4F2196F6E3A1
:10903000CC3BDF0701F7DF91CF911F910F91FF909C
:10904000EF90DF90CF90BF90AF900C943A83FC01EB
:1090500060817181828193810E94EED56093343763
:10906000613019F481E00E94567881E00C947778A1
:10907000CF93DF93CDB7DEB76897CDBFDEBFFC01DE
:1090800060817181828193810E94EED56093353732
:1090900081E0613019F40E9456780CC00E94777804
:1090A000CE01019628E1FC0111922A95E9F7BC0155
:1090B0000E9427486896CDBFDEBFDF91CF9108950B
:1090C0000F931F93CF93DF93CDB7DEB72D97CDBF0F
:1090D000DEBF27E0E8EDF0E28E010F5F1F4FD80101
:1090E00001900D922A95E1F7BC01660F771F680F7A
:1090F000791F660F771F660F771F660F771F6555FD
:109100007A4E45E050E0CE0108960E94B4E16885B1
:1091100070E0C8010E94E2E1009739F46B8570E0CD
:10912000C8010E94E2E1009711F0801B01C08FEF9F
:109130002D96CDBFDEBFDF91CF911F910F91089586
:109140000F931F93CF93DF93CDB7DEB7C058D109EC
:10915000CDBFDEBFFC010D9624852F9323852F9371
:1091600022852F9321852F939F938F937196FF9341
:10917000EF939F938F937F936F938E010F5F1F4F9A
:109180001F930F930E946BE3C8010E94DDC0CDBF07
:10919000DEBFC058DF4FCDBFDEBFDF91CF911F9143
:1091A0000F910895EF92FF920F931F93CF93DF9348
:1091B000CDB7DEB7C058D109CDBFDEBF8C01F62ECA
:1091C000E72EFC01848195810E94604883309CF5E4
:1091D0008F3F09F03BC02FC09801235F3F4F9F9303
:1091E0008F93F80184858F9383858F9382858F93E6
:1091F00081858F933F932F930F5E1F4F1F930F9384
:109200003F932F93EF92FF928E010F5F1F4F1F939B
:109210000F930E946BE3C8010E94DDC0CDBFDEBF8B
:10922000C058DF4FCDBFDEBFDF91CF911F910F91AF
:10923000FF90EF900895EAE2F4E1659174914FE4B4
:1092400050E08AE591E40E94B4E1C6CFE0912C376A
:10925000F0E0EE0FFF1FEA5DFB4E659174914FE465
:1092600050E08AE591E40E94B4E1B6CFEF92FF921C
:109270000F931F93CF93DF93CDB7DEB7C058D109BB
:10928000CDBFDEBF8C01F62EE72EFC0184819581D7
:109290000E9460488330B4F58F3F09F03EC032C071
:1092A000A8014F5E5F4F9801235F3F4F9F938F93BD
:1092B000F80184858F9383858F9382858F93818531
:1092C0008F935F934F933F932F935F934F933F936E
:1092D0002F93EF92FF928E010F5F1F4F1F930F93FB
:1092E0000E946BE3C8010E94DDC0CDBFDEBFC05845
:1092F000DF4FCDBFDEBFDF91CF911F910F91FF9068
:10930000EF900895EAE2F4E1659174914FE450E042
:109310008AE591E40E94B4E1C3CFE0912C37F0E0FC
:10932000EE0FFF1FEA5DFB4E659174914FE450E034
:109330008AE591E40E94B4E1B3CFDF92EF92FF920D
:109340000F931F93CF93DF93CDB7DEB7C858D109E2
:10935000CDBFDEBF8B01E42ED52E37E0EFEDF0E27E
:10936000DE01AF57BF4F01900D923A95E1F7C85714
:10937000DF4F2883C858D0400E946048F82EC85755
:10938000DF4F2881C858D04082E08F1518F0E22FB7
:10939000F0E002C0E2E0F0E0EE0FFF1FEA5DFB4EFE
:1093A000659174914FE450E08AE591E40E94B4E144
:1093B0009F938F93F80183818F9382818F93818113
:1093C0008F9380818F93E1E8F0E0EC0FFD1FEF0DAC
:1093D000F11D80811F928F93DF92EF928E010F5FBC
:1093E0001F4F1F930F930E946BE3C8010E94DDC0C3
:1093F000CDBFDEBFC857DF4FCDBFDEBFDF91CF91FE
:109400001F910F91FF90EF90DF9008954F925F9220
:109410006F927F92AF92BF92CF92DF92EF92FF92C4
:109420000F931F93CF93DF93C6EBD6E30BE715E3C0
:109430005C018991813009F042C0F801C480D58077
:10944000E680F7804080518062807380A3019201A2
:10945000C701B6010E94D1D39F772CEA35EC47E2D1
:1094600057E30E947AD587FD2AC020E034E244E722
:1094700059ECC701B6010E947DD718165CF4F501BE
:109480002081318142815381C701B6010E947DD77D
:10949000181604F120E034E244E759ECC301B201AC
:1094A0000E947DD718165CF4F5012081318142813C
:1094B0005381C301B2010E947AD587FD0BC00B5CBA
:1094C0001F4FF4E0AF0EB11C86E3CC3BD80709F088
:1094D000B0CF02C08CED01C080E0DF91CF911F9131
:1094E0000F91FF90EF90DF90CF90BF90AF907F9063
:1094F0006F905F904F9008958091B236811105C0B2
:109500008091B1368093B03629C0823031F487E043
:109510008093B0368091B13621C0833031F489E038
:109520008093B0368091B13619C0843031F48AE02E
:109530008093B0368091B13611C08091B3368130BE
:1095400031F485E08093B0368091B13607C0823027
:1095500019F486E08093B0368091B136863019F0E8
:109560008091B03608958BE08093B0360895809155
:10957000B13608958093B336813059F018F08230B7
:1095800041F0089581EE96E38093DF369093E036C4
:10959000089589EA9AE58093DF369093E03608953E
:1095A000FC0184810895845B9F4FFC0180810895B4
:1095B000855B9F4FFC0180810895825B9F4FFC017A
:1095C00080810895815B9F4FFC0180810895875BB6
:1095D0009F4FFC01808108950C943098CD96FC013A
:1095E00060817181828193810895FC016483089573
:1095F0008B5A9F4FFC01608308958F5B9F4FFC0146
:10960000408351836283738308956093E13670933E
:10961000E2368093E3369093E43688EE91E20C9440
:10962000B262BF92CF92DF92EF92FF920F931F939D
:10963000CF93DF93D0902E377C0103E517E3809121
:109640002D3790E0EC01CC0FDD1FC80FD91FCC0FD8
:10965000DD1FCC0FDD1FCC0FDD1FC653DB4C81E0BF
:10966000D816A9F0B881A981CA80BB804091A637DD
:10967000413091F4F80120813181428153816B2F77
:109680007A2F8C2D9B2D0E94D2D39B0109C020E004
:1096900030E080E090E004C02B2F3A2F8C2D9B2DE2
:1096A000A901BC01F701458F568F678F70A3F4E0C5
:1096B000EF0EF11C0C5F1F4F249687E30B36180743
:1096C00071F6DF91CF911F910F91FF90EF90DF9096
:1096D000CF90BF900895835B9F4FFC01608381EE24
:1096E00096E30C94114B4F925F926F927F928F9200
:1096F0009F92AF92BF92CF92DF92EF92FF920F9321
:109700001F93CF93DF93CDB7DEB76897CDBFDEBF92
:109710008C016091A63770E080E090E00E941CD63A
:109720002B013C01F80160817181828193810E944B
:10973000EED570E05B01AA0CBB1CA60EB71EAA0CEE
:10974000BB1CAA0CBB1CAA0CBB1CC50186539B4CA2
:109750005C0103E517E3FE0131964F01F501C1906D
:10976000D190E190F1905F01F80161917191819147
:1097700091918F01A30192010E941FD89B01AC011E
:10978000C701B6010E94D2D3F40161937193819312
:1097900091934F01F7E30B361F0701F7CE010196B6
:1097A0000E94139881EE96E30E94114B6896CDBFFC
:1097B000DEBFDF91CF911F910F91FF90EF90DF906F
:1097C000CF90BF90AF909F908F907F906F905F9061
:1097D0004F900895815E964369F4E62FF0E0EE0F16
:1097E000FF1FEE0FFF1FE55CF84C608171818281E5
:1097F00093810895862F0C940898CF92DF92EF9270
:10980000FF920F931F93CF93DF93EC0186E3C13E4A
:10981000D80709F04AC070E0FB01EE0FFF1FEE0F02
:10982000FF1FE55CF84CC080D180E280F38080911E
:109830002E37813059F180912D3790E0FC01EE0FE9
:10984000FF1FE80FF91FEE0FFF1FE60FF71FEE0FC8
:10985000FF1FEE0FFF1FE653FB4C00811181B28109
:10986000A3812091A6372130B1F4FB01EE0FFF1F39
:10987000EE0FFF1FED5AF84C208131814281538158
:10988000B8018B2F9A2F0E94D2D308C060E070E0FD
:1098900080E090E003C0B8018B2F9A2F9B01AC01B0
:1098A000C701B6010E94D1D303C0862F0E941C9825
:1098B000C55BDF4F2881211106C023E333E34BEC66
:1098C00051E40E9481D5DF91CF911F910F91FF90BC
:1098D000EF90DF90CF90089588E1E6EEF6E3ABE3FA
:1098E000B7E301900D928A95E1F780912A378111B3
:1098F0000CC08091E536813041F410921E371092F1
:109900001F37109220371092213708954F925F929F
:109910006F927F928F929F92AF92BF92CF92DF927F
:10992000EF92FF920F931F93CF93DF93CDB7DEB7E4
:109930006997CDBFDEBF8091B236811155C080914D
:10994000D736813009F050C00E9468C681114CC0E2
:109950001092D73692EE692E94E3792E26E3822E6A
:10996000912C8E010E5E1F4F36EEA32E30E2B32EE9
:1099700033C0F70181917F011F928F935F924F92C5
:10998000BF92AF921F930F930E9442E3B80187E406
:1099900093E20E94D45F8D839E83F6018191919121
:1099A000A191B1916F018A879B87AC87BD87CE015A
:1099B00001960E949C5CCDBFDEBF9EEDE91690E251
:1099C000F906B9F6E8E16E0E711CFFEF8F1A9F0AD7
:1099D0008CE38816910441F0240189EDE82E80E2A1
:1099E000F82E630188E7C8CF80E06996CDBFDEBF5F
:1099F000DF91CF911F910F91FF90EF90DF90CF906B
:109A0000BF90AF909F908F907F906F905F904F909E
:109A100008952F923F924F925F926F927F928F9212
:109A20009F92AF92BF92CF92DF92EF92FF920F93ED
:109A30001F93CF93DF93CDB7DEB72997CDBFDEBF9E
:109A40004C015B014090303750902E3720902D37DD
:109A50006090A63770902C376B0186EE96E388876E
:109A6000998752E7E52E55E3F52E98E1299E1001DE
:109A700011248401D6016D917D918D919D916D018F
:109A80002CEA35EC47E257E30E947AD587FD80C087
:109A9000F70180818150823008F07AC041104CC0BB
:109AA000F1E05F1609F1E885F985E20DF31DEC514F
:109AB000F2408081898391819D83B281A381E1E01D
:109AC0006E1217C0E885F985E359FF4F2081318177
:109AD00042815381BC018B2F9A2F0E94D2D369837C
:109AE0007D838E839F8307C019821D821E821F8201
:109AF00002C0BE83AF8371100CC023E333E34BEC91
:109B000051E4D8016D917D918D919C910E941FD857
:109B100005C0F801608171818281938129813D8135
:109B20004E815F810E94D2D3A885B9856D937D93C4
:109B30008D939C9313972CC0A885B9858D919D9189
:109B40000D90BC91A02D89839A83AB83BC83711047
:109B50000EC023E333E34BEC51E4F80160817181E3
:109B6000828193810E941FD89B01AC0105C0D8015E
:109B70002D913D914D915C9169817A818B819C8180
:109B80000E94D2D3E885F9856083718382839383B1
:109B90008885998504968887998795E3E90EF11C55
:109BA0000C5F1F4FA885B985A25FB64309F062CF4D
:109BB00060902C3770903037F0912E37F983C09039
:109BC0002D372091A6372D838CE0A80EB11CA1E182
:109BD000B6E3A887B98742EFE42E46E3F42EB8E156
:109BE000CB9E600111248401F501619171918191F5
:109BF00091915F012CEA35EC47E257E30E947AD558
:109C000087FD8CC0A885B9858C91882309F486C00E
:109C10008150823030F4F80124843584468457849E
:109C20003BC0611016C023E333E34BEC51E4D80191
:109C30001C966D917D918D919C911F970E941FD8CC
:109C400020E030E044EB53E40E941FD81B012C01BC
:109C50000DC020E030E044EB53E4F80164857585E5
:109C6000868597850E941FD81B012C012BED3FE0B4
:109C700049EC50E4A885B98591966D917D918D91BF
:109C80009C9194970E941FD89B01AC01C201B10125
:109C90000E9481D51B012C01711031C0B981B130F6
:109CA000E1F0F701EC0DFD1DEC51F240A081B18116
:109CB00092808380ED81E130A1F4F701E359FF4FF9
:109CC0002081318142815381BD01892D982D0E94CF
:109CD000D2D3DB01982E892E04C0A0E0B0E0912CF5
:109CE000812CA2019101BD01892D982D0E94D2D312
:109CF000D7016D937D938D939C9313970FC0A20111
:109D00009101F70160817181828193810E94D2D398
:109D1000D7016D937D938D939C931397E885F98577
:109D2000F596E887F987F4E0EF0EF11C0C5F1F4F02
:109D300088859985805B964309F056CF2996CDBFDB
:109D4000DEBFDF91CF911F910F91FF90EF90DF90D9
:109D5000CF90BF90AF909F908F907F906F905F90CB
:109D60004F903F902F9008958091AE349091AF34F2
:109D70008F3E924111F08FE5089580916538909162
:109D800066388F3E9241B9F78091373790913837D6
:109D90008F3E924181F78091AD379091AE378F3EE3
:109DA000924149F78091015B9091025B8F3E924115
:109DB00011F78091BE5B9091BF5B8F3E9241D9F6C7
:109DC00080E008958BE10E941FA982E08093B13664
:109DD00080E00895CF93C82F0E941FA982E080934E
:109DE000B1368C2FCF9108958091B236811104C085
:109DF00083E08093B13603C085E08093B13680E084
:109E00000895CF93C82F0E9461B480E00E94F6AFFE
:109E10008C2F0E941FA986E08093B1368C2FCF91A2
:109E2000089581E08093D83680E0089581E08093A2
:109E3000DA3680E0089581E08093D93680E0089595
:109E40000E94107980E0089580932B3780E0089578
:109E500080932C3780E008958093303780E0089518
:109E60004F925F926F927F929F92AF92BF92CF92EA
:109E7000DF92EF92FF920F931F93CF93DF93C82F40
:109E8000B62E8A01F22ED32F8FEF8C0F863008F07A
:109E900082C06091393870E080E090E00E941CD66A
:109EA0002CEA35EC47E257E30E947AD587FD75C06E
:109EB00082E0B81619F0E4E1BE1271C090902C3720
:109EC000CF2CDD2E8C2F90E0EC01CC0FDD1FC80FC6
:109ED000D91FCC0FDD1FCC0FDD1FCC0FDD1FC653EC
:109EE000DB4C78010BE317E3AA24A394F6016191FC
:109EF0007191819191916F012CEA35EC47E257E322
:109F00000E947DD71816DCF5F2E0BF1214C0911044
:109F10000CC023E333E34BEC51E4F7016081718122
:109F2000828193810E941FD824C0F70160817181D2
:109F3000828193811EC0F8014080518062807380CD
:109F400091100EC023E333E34BEC51E4F701608141
:109F50007181828193810E941FD89B01AC0105C051
:109F6000F7012081318142815381C301B2010E94F6
:109F7000D1D3688379838A839B83A092D736249632
:109F8000F4E0EF0EF11C0C5F1F4F87E30335180759
:109F900009F0ACCF06C081EA05C08CEA03C08DEAA7
:109FA00001C080E0DF91CF911F910F91FF90EF9062
:109FB000DF90CF90BF90AF909F907F906F905F9019
:109FC0004F900895CF93DF93CDB7DEB76897CDBF9D
:109FD000DEBF80932D37682F70E080E090E00E9414
:109FE0001AD669837A838B839C831D821E821F828B
:109FF000188619861A861B861C861D861E861F8655
:10A00000188A198A1A8A1B8A1C8A1D8A1E8A1F8A24
:10A01000188EAE014F5F5F4FBA0183E79BE40E9449
:10A02000718480E06896CDBFDEBFDF91CF91089547
:10A03000CF93DF93E1EEF6E386E5DF011D928A958B
:10A04000E9F78BE5AFEAB7E3ED01982F19929A95FE
:10A05000E9F7AAE0B8E3ED0119928A95E9F78FEEE6
:10A0600092E18093AE349093AF34809365389093AF
:10A07000663880933737909338378093AD37909315
:10A08000AE378093015B9093025B8093BE5B9093AD
:10A09000BF5BE093DF36F093E0368091C734809366
:10A0A0002C378091C5340E94E24F8091C634809352
:10A0B0002B378091C83480932F378091C934809397
:10A0C000303781E080932A378093A73794E09093CC
:10A0D000E5361092D8361092D9361092DA3680933F
:10A0E000B1368093B0360E9494AEDF91CF910C943C
:10A0F000B385CF92DF92EF92FF92CF93C82F6A0180
:10A100007B01E82FF0E0DF01AA0FBB1FAA0FBB1FE6
:10A11000A55CB84C4D935D936D937C931397EE0FB4
:10A12000FF1FEE0FFF1FEA51F94C408351836283FA
:10A1300073838C2F0E942483B701A6018C2F0E9469
:10A140002F83CF91FF90EF90DF90CF900C943A83C4
:10A150009F92AF92BF92CF92DF92EF92FF920F93B6
:10A160001F93CF93DF93CDB7DEB76897CDBFDEBF28
:10A17000962EA72EC62ED72E7C0100E010E0B12C23
:10A18000F60161917191819191916F012CEA35EC09
:10A1900047E257E30E947DD71816A4F580912C372B
:10A1A00081110EC023E333E34BEC51E4F7016081EE
:10A1B0007181828193810E941FD8AB01BC0105C0CF
:10A1C000F7014081518162817381E1E0F0E0EC0FA1
:10A1D000FD1FE00FF11F4083518362837383C80129
:10A1E00082559B4CFC01E357FD4F408351836283B2
:10A1F0007383E555F10940835183628373838B2D0B
:10A200000E942483B3940C5F1F4FF4E0EF0EF11C07
:10A210000831110509F0B4CF492D5A2DBE016F5FE9
:10A220007F4F88EE97E40E94718480E06896CDBFEE
:10A23000DEBFDF91CF911F910F91FF90EF90DF90E4
:10A24000CF90BF90AF909F9008954F925F926F9282
:10A250007F928F929F92AF92BF92CF92DF92EF92B6
:10A26000FF920F931F93CF93DF93CDB7DEB768971D
:10A27000CDBFDEBF21E02093A63780902D37909090
:10A280002C375B016C010BE317E3882D90E07C0118
:10A29000EE0CFF1CE80EF91EEE0CFF1CEE0CFF1C72
:10A2A000EE0CFF1CC70186539B4C7C01F5016191AC
:10A2B0007191819191915F012CEA35EC47E257E36E
:10A2C0000E947DD7181664F5F70120813181428103
:10A2D0005381F80160817181828193810E94D1D381
:10A2E0002B013C0191100EC023E333E34BEC51E40E
:10A2F000F60160817181828193810E941FD89B0148
:10A30000AC0105C0F6012081318142815381C30136
:10A31000B2010E94D1D3F801608F718F828F938F29
:10A32000F4E0CF0ED11C0C5F1F4F84E0E80EF11C4F
:10A3300097E30335190709F0B9CF682D70E080E085
:10A3400090E00E941AD669837A838B839C831D8256
:10A350001E821F82188619861A861B861C861D86F9
:10A360001E861F86188A198A1A8A1B8A1C8A1D8AC9
:10A370001E8A1F8A188EAE014F5F5F4FBA0183E7B6
:10A380009BE40E94718480E06896CDBFDEBFDF91C0
:10A39000CF911F910F91FF90EF90DF90CF90BF90E2
:10A3A000AF909F908F907F906F905F904F900895A7
:10A3B000CF93DF93CDB7DEB76897CDBFDEBF1092E6
:10A3C000A637109253371092543710925537109287
:10A3D00056371092573710925837109259371092BB
:10A3E0005A3710925B3710925C3710925D3710929B
:10A3F0005E3710925F37109260371092613710927B
:10A40000623710926337109264371092653710925A
:10A41000663710926737109268371092693710923A
:10A420006A3760912D3770E080E090E00E941AD684
:10A4300069837A838B839C831D821E821F82188688
:10A4400019861A861B861C861D861E861F86188AFC
:10A45000198A1A8A1B8A1C8A1D8A1E8A1F8A188ECC
:10A46000AE014F5F5F4FBA0183E79BE40E947184A6
:10A4700080E06896CDBFDEBFDF91CF910895CF9386
:10A48000DF93CDB7DEB76897CDBFDEBF1092A6379A
:10A4900060912D3770E080E090E00E941AD66983C9
:10A4A0007A838B839C831D821E821F821886198665
:10A4B0001A861B861C861D861E861F86188A198A88
:10A4C0001A8A1B8A1C8A1D8A1E8A1F8A188EAE0150
:10A4D0004F5F5F4FBA0183E79BE40E94718480E085
:10A4E0006896CDBFDEBFDF91CF910895CF93DF9304
:10A4F000CDB7DEB76897CDBFDEBF81E08093A637CA
:10A5000060912D3770E080E090E00E941AD6698358
:10A510007A838B839C831D821E821F8218861986F4
:10A520001A861B861C861D861E861F86188A198A17
:10A530001A8A1B8A1C8A1D8A1E8A1F8A188EAE01DF
:10A540004F5F5F4FBA0183E79BE40E94718480E014
:10A550006896CDBFDEBFDF91CF910895CF93109263
:10A56000E5360E94094D8091B834813069F486EE59
:10A5700096E30E94064AC82F882331F00E941FA943
:10A5800082E08093B13617C081EE96E30E94114BB2
:10A5900085E08093B1368091B236811105C081E0AB
:10A5A0008093B2360E9409AD81EE96E30E943D98F9
:10A5B0000E946C4CC0E08C2FCF91089588E1EBE3B2
:10A5C000F7E3ABE6B7E301900D928A95E1F780E0FF
:10A5D00008950F931F93CF93DF93CDB7DEB76A979C
:10A5E000CDBFDEBF8C0181E080932E3781EE96E3F4
:10A5F000698F7A8F0E94114B698D7A8DC8010E94F4
:10A60000AE520E94AB838823E1F388E1E0E0F0E200
:10A61000DE01119601900D928A95E1F7BE016F5F00
:10A620007F4F8BE697E30E94AE526A96CDBFDEBFA6
:10A63000DF91CF911F910F91089588E1EBE3F7E34C
:10A64000A3E8B7E301900D928A95E1F780E00895C1
:10A650000F931F93CF93DF93CDB7DEB76A97CDBF2C
:10A66000DEBF8C0181E080932E3781EE96E3698F07
:10A670007A8F0E94114B698D7A8DC8010E94AE526B
:10A680000E94AB838823E1F388E1E0E0F0E2DE01A1
:10A69000119601900D928A95E1F7BE016F5F7F4F91
:10A6A00083E897E30E94AE526A96CDBFDEBFDF918A
:10A6B000CF911F910F910895FB01DC0180912A3702
:10A6C000811111C09B01AD0160E070E080E89FE363
:10A6D0000E9481D560931E3770931F378093203777
:10A6E0009093213718C080912C37811109C023E342
:10A6F00033E34BEC51E4CD010E941FD8FB0101C0B4
:10A70000CD01AF01BC0140931E3750931F376093BA
:10A7100020377093213780E0089580932A3780E0B6
:10A72000089580932F3780E00895609326377093C3
:10A73000273780932837909329370E94C98480E077
:10A7400008950F931F93CF93DF93EC018B018091BA
:10A750002A37882399F080911E3790911F37A09156
:10A760002037B0912137BC01CD019F772CEA35EC21
:10A7700047E257E30E947AD587FD30C081E080939D
:10A78000E536B801CE010E94094D8091B834813080
:10A7900069F486EE96E30E94064AC82F882331F0BA
:10A7A0000E941FA982E08093B13619C081EE96E322
:10A7B0000E94114B85E08093B1368091B2368111B1
:10A7C00005C081E08093B2360E9409AD81EE96E328
:10A7D0000E943D98C82F0E946C4C01C0CEE88C2F7F
:10A7E000DF91CF911F910F910895CF93DF93CDB754
:10A7F000DEB76897CDBFDEBF682F70E080E090E0E5
:10A800000E941AD669837A838B839C831D821E8261
:10A810001F82188619861A861B861C861D861E8630
:10A820001F86188A198A1A8A1B8A1C8A1D8A1E8A00
:10A830001F8A188EAE014F5F5F4FBA0184ED97E417
:10A840000E94718480E06896CDBFDEBFDF91CF911A
:10A850000895CF93DF93CDB7DEB76897CDBFDEBF46
:10A860006091333770E080E090E00E941AD66983EF
:10A870007A838B839C831D821E821F821886198691
:10A880001A861B861C861D861E861F86188A198AB4
:10A890001A8A1B8A1C8A1D8A1E8A1F8A188EAE017C
:10A8A0004F5F5F4FBA018EED97E40E94718480E0A4
:10A8B0006896CDBFDEBFDF91CF910895CF93DF9330
:10A8C000CDB7DEB76897CDBFDEBF682F70E080E000
:10A8D00090E00E941AD669837A838B839C831D82C1
:10A8E0001E821F82188619861A861B861C861D8664
:10A8F0001E861F86188A198A1A8A1B8A1C8A1D8A34
:10A900001E8A1F8A188EAE014F5F5F4FBA0187E221
:10A9100098E40E94718480E06896CDBFDEBFDF912D
:10A92000CF910895CF93DF93CDB7DEB76897CDBFB2
:10A93000DEBF682F70E080E090E00E941AD6698345
:10A940007A838B839C831D821E821F8218861986C0
:10A950001A861B861C861D861E861F86188A198AE3
:10A960001A8A1B8A1C8A1D8A1E8A1F8A188EAE01AB
:10A970004F5F5F4FBA0188E398E40E94718480E0E2
:10A980006896CDBFDEBFDF91CF910895CF93FC01D4
:10A9900060817181828193810E94EED56093B1368E
:10A9A0001092B33681EE96E38093DF369093E036D3
:10A9B0008091B236813011F41092B2361092B436D2
:10A9C0001092DA360E94F697C091B136C430C9F4BD
:10A9D0000E94D8518091C5340E94E24F8091C634C4
:10A9E00080932B378091C9348093303780E00E9468
:10A9F000F6AF80E00E94925481E080932A37C093A2
:10AA0000E53681E0CF910C94E7AB8093A337809338
:10AA1000A4378093AC3780E008952CEA35EC47E208
:10AA200057E360915138709152388091533890912A
:10AA300054380E947DD71816B4F48091F63790915F
:10AA4000F737A091F837B091F937BC01CD019F7766
:10AA50002CEA35EC47E257E30E947AD587FF03C022
:10AA60001092A33703C081E08093A33780E008955C
:10AA70008093A3378091F6379091F737A091F837FC
:10AA8000B091F93780939B3790939C37A0939D3773
:10AA9000B0939E3780E008952CEA35EC47E257E307
:10AAA0006091513870915238809153389091543858
:10AAB0000E947DD71816B4F48091F6379091F7373D
:10AAC000A091F837B091F937BC01CD019F772CEAFE
:10AAD00035EC47E257E30E947AD587FF03C0109216
:10AAE000A43703C081E08093A43780E00895809369
:10AAF000A4378091F6379091F737A091F837B0914D
:10AB0000F93780939F379093A037A093A137B093E4
:10AB1000A23780E008952CEA35EC47E257E36091D4
:10AB200051387091523880915338909154380E9426
:10AB30007DD71816B4F48091F6379091F737A0912D
:10AB4000F837B091F937BC01CD019F772CEA35EC8D
:10AB500047E257E30E947AD587FF03C01092AC37D3
:10AB600003C081E08093AC3780E008958093AC37D8
:10AB70008091F6379091F737A091F837B091F93777
:10AB80008093A8379093A937A093AA37B093AB3797
:10AB900080E00895BC018DEE90E20C94D56281E0D6
:10ABA0008093D836089581E08093D936089581E066
:10ABB0008093DA3608951F93CF93DF93CDB7DEB736
:10ABC0006897CDBFDEBF0E9430988130C9F10E94E6
:10ABD00018D20E941CC90E942E8480E00E941EADE3
:10ABE00010E0812F0E940898AB01BC01812F0E94C8
:10ABF00079501F5F1630A9F780E090E0A0E4B0E440
:10AC000089839A83AB83BC831D821E821F82188630
:10AC100019861A861B861C861D861E861F86188A24
:10AC2000198A1A8A1B8A1C8A1D8A1E8A1F8A188EF4
:10AC3000BE016F5F7F4FCB010E94C65480E001C010
:10AC40008AE66896CDBFDEBFDF91CF911F91089550
:10AC50008091D8368130A9F42091B336213079F42F
:10AC60008091B43681110BC082E08093B33689EABB
:10AC70009AE58093DF369093E0362093B4361092B5
:10AC8000D8368091D936813091F48091B3368823BB
:10AC900031F0823061F49091B436943051F40E94D6
:10ACA0003098811104C01092D9360E94DB559091E2
:10ACB000B4368091DA368130C1F42091D936211131
:10ACC00014C09150933088F01092DA3695E090934A
:10ACD000B4369093B1369091B236911104C08093FE
:10ACE000B2360E9409AD0E94A2A080E0089585E0DE
:10ACF0008093B1368091B236811105C081E0809396
:10AD0000B2360C9409AD0895CF93DF93CDB7DEB77B
:10AD10006897CDBFDEBF8091B236882311F180E005
:10AD200090E0A0E4B0E489839A83AB83BC831D8266
:10AD30001E821F82188619861A861B861C861D860F
:10AD40001E861F86188A198A1A8A1B8A1C8A1D8ADF
:10AD50001E8A1F8A188EBE016F5F7F4FCB010E9433
:10AD6000C6546896CDBFDEBFDF91CF910895CF93D3
:10AD7000DF93CDB7DEB76897CDBFDEBF80E090E050
:10AD8000A0E4B0E489839A83AB83BC831D821E82D6
:10AD90001F82188619861A861B861C861D861E86AB
:10ADA0001F86188A198A1A8A1B8A1C8A1D8A1E8A7B
:10ADB0001F8A188EAE014F5F5F4FBA0186EC94E593
:10ADC0000E9471846896CDBFDEBFDF91CF91089558
:10ADD000CF93DF93CDB7DEB76897CDBFDEBF80E0FE
:10ADE00090E0A0E8B0E489839A83AB83BC831D82A2
:10ADF0001E821F82188619861A861B861C861D864F
:10AE00001E861F86188A198A1A8A1B8A1C8A1D8A1E
:10AE10001E8A1F8A188EAE014F5F5F4FBA0186EC03
:10AE200094E50E9471846896CDBFDEBFDF91CF911B
:10AE30000895CF93DF93CDB7DEB72797CDBFDEBFA1
:10AE400097E0EFEDF0E2DE01119601900D929A95F8
:10AE5000E1F7873050F4E1E0F0E0EC0FFD1FE80F80
:10AE6000F11D87FDFA95808101C080E22796CDBF54
:10AE7000DEBFDF91CF9108950F931F93CF93DF93A0
:10AE8000EC01042F10E020E030E009871A872B87BF
:10AE90003C8782E08F8350E0440F551F640F751F7D
:10AEA000FB01659174914FE450E08AE591E40E94C2
:10AEB000B4E1BC01CE01DF91CF911F910F910C94B1
:10AEC0007762CF93DF93EC010E947C4A482F64E6BF
:10AED00073E1CE01DF91CF910C943C574091B13694
:10AEE00065E273E10C943C574091B2366CEF72E12D
:10AEF0000C943C574091B33668EE72E10C943C5789
:10AF00004091B4366AEB72E10C943C574091B536EF
:10AF10006DE972E10C943C57E091DF36F091E03638
:10AF2000E55BFF4F408167EC73E10C943C57E09187
:10AF3000DF36F091E036E45BFF4F408163ED71E175
:10AF40000C943C57E091DF36F091E036448169E3A0
:10AF500071E10C943C57E091DF36F091E036E65B0E
:10AF6000FF4F408166E071E10C943C57E091DF3681
:10AF7000F091E036E25BFF4F40816CEB70E10C94A6
:10AF80003C57E091DF36F091E036E15BFF4F4081C6
:10AF90006BE770E10C943C57E091DF36F091E036BE
:10AFA000E75BFF4F40816CE070E10C943C57E0910F
:10AFB000DF36F091E036EF5AFF4F408150E060E01D
:10AFC00070E0FC01418752876387748722E0278302
:10AFD00080E00895E091DF36F091E03640815181C4
:10AFE00062817381FC01418752876387748722E005
:10AFF000278380E00895CF93DF93EC018091B336EF
:10B00000811105C019861A861B861C8614C00E94F1
:10B01000FF9769877A878B879C872091F45A211143
:10B020000AC025E832E441E25DE30E941FD8698747
:10B030007A878B879C878C819D81FC01EE0FFF1F97
:10B04000E80FF91FEE0FFF1FEE0FFF1FEE0FFF1FA0
:10B05000EE54FA4E85919491888784E08F8380E046
:10B06000DF91CF910895CF93DF93EC012091DF36EC
:10B070003091E036F901FD96608171818281938182
:10B0800069877A878B879C873E96208121110AC029
:10B0900025E832E441E25DE30E941FD869877A87A0
:10B0A0008B879C878C819D81FC01EE0FFF1FE80F31
:10B0B000F91FEE0FFF1FEE0FFF1FEE0FFF1FEE54E5
:10B0C000FA4E85919491888784E08F8380E0DF91A8
:10B0D000CF910895CF93DF93EC018C819D810E94E5
:10B0E0006048682F8091DF369091E0360E94FD4BDA
:10B0F00069877A878B879C878C819D81FC01EE0F05
:10B10000FF1FE80FF91FEE0FFF1FEE0FFF1FEE0FDF
:10B11000FF1FEE54FA4E85919491888784E08F83C7
:10B1200080E0DF91CF910895CF93DF93EC018C8184
:10B130009D810E9460482091DF363091E036215E8B
:10B14000364369F4E82FF0E0EE0FFF1FEE0FFF1F0C
:10B15000E55CF84C608171818281938102C00E941C
:10B16000089869877A878B879C878C819D81FC01F1
:10B17000EE0FFF1FE80FF91FEE0FFF1FEE0FFF1F6F
:10B18000EE0FFF1FEE54FA4E85919491888784E06C
:10B190008F8380E0DF91CF910895CF93DF93EC010F
:10B1A0008C819D810E946048E091DF36F091E0360D
:10B1B00094E0899FE00DF11D1124458D568D678D1A
:10B1C00070A149875A876B877C878C819D81FC01A0
:10B1D000EE0FFF1FE80FF91FEE0FFF1FEE0FFF1F0F
:10B1E000EE0FFF1FEE54FA4E85919491888784E00C
:10B1F0008F8380E0DF91CF910895CF93DF93EC01AF
:10B200000E94A15D498563EF73E1CE01DF91CF918B
:10B210000C943C57CF93DF93EC018C819D810E946D
:10B220006048833054F48F3F91F407C0CE010E94F0
:10B230007A5E80E016C08DE614C049855A856B851C
:10B240007C854430510561057105A8F7EFCF49852C
:10B250005A856B857C85433051056105710558F72A
:10B26000E5CFDF91CF91089595E3899FF0011124F7
:10B27000ED57FA4C60817181828193810895CF925C
:10B28000DF92EF92FF92CF93DF936A017B0125E378
:10B29000829FC001112482559B4CFC01EB52FF4F51
:10B2A0004083518362837383EC01C352DF4F20E0FC
:10B2B00034E244E759E4C701B6010E941FD89B015C
:10B2C000AC0160E070E080E89FE30E9481D5688374
:10B2D00079838A839B83DF91CF91FF90EF90DF90FA
:10B2E000CF900895CF92DF92EF92FF92CF93DF93AA
:10B2F000EC01C984DA84EB84FC8420E034E244E786
:10B3000059E4C701B6010E947DD7181664F420E005
:10B3100034E244E759E4C701B6010E9481D5698748
:10B320007A878B879C87CE010E949263C984DA84D6
:10B33000EB84FC848C819D810E94604825E3829F80
:10B34000C001112482559B4CFC01EB52FF4FC0827F
:10B35000D182E282F382EC01C352DF4F20E034E27B
:10B3600044E759E4C701B6010E941FD89B01AC0114
:10B3700060E070E080E89FE30E9481D56883798374
:10B380008A839B8380E0DF91CF91FF90EF90DF90E5
:10B39000CF900895CF92DF92EF92FF92CF93DF93F9
:10B3A000EC01C984DA84EB84FC8420E034E244E7D5
:10B3B00059E4C701B6010E947DD7181664F420E055
:10B3C00034E244E759E4C701B6010E9481D5698798
:10B3D0007A878B879C87CE010E94926380E0DF9101
:10B3E000CF91FF90EF90DF90CF90089581E0809310
:10B3F000D93680E00895FC0181859285A385B485C6
:10B400000197A105B10511F40E944C6B80E00895ED
:10B410006091DB367091DC368091DD369091DE36BE
:10B4200008950E94525F80E00E94CF6D80E00895F1
:10B430000E94525F81E00E94CF6D80E008950E94DB
:10B44000525F82E00E94CF6D80E008950E94525FBB
:10B4500083E00E94CF6D80E00895CF93DF93EC01ED
:10B46000E091DF36F091E036E55BFF4FE081F0E000
:10B47000EE0FFF1FEA5DFB4E659174914FE450E0C3
:10B480008AE591E40E94B4E1AC0165EF7FE0CE0172
:10B49000DF91CF910C948CC1CF93DF93EC01E091BD
:10B4A000DF36F091E036E55BFF4FE081F0E0EE0F34
:10B4B000FF1FEA5DFB4E659174914FE450E08AE511
:10B4C00091E40E94B4E1AC016DED7FE0CE01DF912B
:10B4D000CF910C948CC1CF93DF93EC0181EF90E27C
:10B4E0000E9415E3CE010E942D5ACE010E944C5AB3
:10B4F0006AEC7FE0CE010E94B8C161EB7FE0CE0133
:10B500000E9402C168E97FE0CE010E9402C16FE79C
:10B510007FE0CE010E9402C166E67FE0CE010E947C
:10B5200002C16DE47FE0CE010E9402C164E37FE0CE
:10B53000CE010E9402C16BE17FE0CE010E9402C1F8
:10B5400062E07FE0CE010E9402C169EE7EE0CE01A2
:10B550000E9402C160ED7EE0CE010E9402C167EB55
:10B560007EE0CE010E9402C16EE97EE0CE010E9423
:10B5700002C165E87EE0CE010E9402C16CE67EE079
:10B58000CE010E9430C180E0DF91CF9108956AEC36
:10B590007FE00C94B8C161EB7FE00C9402C168E9D4
:10B5A0007FE00C9402C16FE77FE00C9402C166E675
:10B5B0007FE00C9402C16DE47FE00C9402C164E36F
:10B5C0007FE00C9402C16BE17FE00C9402C162E069
:10B5D0007FE00C9402C169EE7EE00C9402C160ED44
:10B5E0007EE00C9402C167EB7EE00C9402C16EE930
:10B5F0007EE00C9402C165E87EE00C9402C16CE62A
:10B600007EE00C9430C160EF7DE00C9430C16FEBB4
:10B610007DE00C9430C16AE87DE00C9430C16FE4A9
:10B620007DE00C9430C16BE17DE00C9430C1CF9390
:10B63000DF93EC01E091DF36F091E036E55BFF4F00
:10B64000E081F0E0EE0FFF1FEA5DFB4E6591749123
:10B650004FE450E08AE591E40E94B4E1AC0167EF69
:10B660007CE0CE01DF91CF910C948CC1CF93DF931E
:10B67000EC01E091DF36F091E036E55BFF4FE081D1
:10B68000F0E0EE0FFF1FEA5DFB4E659174914FE411
:10B6900050E08AE591E40E94B4E1AC0166ED7CE003
:10B6A000CE01DF91CF910C948CC169EB7CE00C94BE
:10B6B000B8C1CF93DF93EC01E091DF36F091E03633
:10B6C000E55BFF4FE081F0E0EE0FFF1FEA5DFB4E10
:10B6D000659174914FE450E08AE591E40E94B4E1F1
:10B6E000AC016AE97CE0CE01DF91CF910C948CC172
:10B6F0000F931F93CF93DF93CDB7DEB7C058D10917
:10B70000CDBFDEBF8C01DC011996EC91F0E0EE0FAD
:10B71000FF1FED50FC4E659174914FE450E08AE5B7
:10B7200091E40E94B4E19801235F3F4F9F938F9370
:10B73000F80181851F928F933F932F930F5E1F4FC8
:10B740001F930F933F932F938EE79CE09F938F93CC
:10B750008E010F5F1F4F1F930F930E946BE3C80171
:10B760000E94DDC0CDBFDEBFC058DF4FCDBFDEBF02
:10B77000DF91CF911F910F91089566E57CE00C94C5
:10B78000D2486EE27CE00C94D2486CE07CE00C94F1
:10B79000D2486AEE7BE00C94D24868EB7BE00C94D4
:10B7A000D24867E87BE00C94D2486EE47BE00C94CE
:10B7B000D2486EE27BE00C94D2486CEE7AE00C94B6
:10B7C000A0486AEA7AE00C94A04863E87AE00C9416
:10B7D000D2486DE57AE00C94D2486CE37AE00C94A0
:10B7E000D2486CE17AE00C94D2486FEF79E00C9487
:10B7F000364960EE79E00C943649BC01675F7F4FB3
:10B8000020912C3746E55EE0FC01848195810C9403
:10B810009D49BC01675F7F4F21E04CE35EE0FC0186
:10B82000848195810C949D49BC01675F7F4F21E025
:10B8300043E25EE0FC01848195810C949D490F9365
:10B840001F93CF93DF93EC010C811D810E94FF6455
:10B8500008171907C4F48C819D81FC01EE0FFF1FAE
:10B86000E80FF91FEE0FFF1FEE0FFF1FEE0FFF1F78
:10B87000E954FA4E25913491CE01F901DF91CF912F
:10B880001F910F91199485E1DF91CF911F910F9135
:10B8900008950F931F93CF93DF93EC010C811D81CB
:10B8A0000E94FF6408171907C4F48C819D81FC0174
:10B8B000EE0FFF1FE80FF91FEE0FFF1FEE0FFF1F28
:10B8C000EE0FFF1FEB54FA4E25913491CE01F90192
:10B8D000DF91CF911F910F91199485E1DF91CF9165
:10B8E0001F910F9108950F931F93CF93DF93EC0156
:10B8F0000C811D810E94FF6408171907C4F48C8114
:10B900009D81FC01EE0FFF1FE80FF91FEE0FFF1FD7
:10B91000EE0FFF1FEE0FFF1FED54FA4E25913491ED
:10B92000CE01F901DF91CF911F910F911994DF9111
:10B93000CF911F910F910895CF93DF93EC018C81EC
:10B940009D810E9412658823C9F08C819D81FC0134
:10B95000EE0FFF1FE80FF91FEE0FFF1FEE0FFF1F87
:10B96000EE0FFF1FEF54FA4EE491E1FF05C0CE0148
:10B97000DF91CF910C94898280E001C085E1DF9155
:10B98000CF910895AF92BF92CF92DF92EF92FF9244
:10B990000F931F93CF93DF93EC0181E00E94284F18
:10B9A0001C821D8280E090E07E0121E1E20EF11C0C
:10B9B00054E0A52E62E0B62E51C00C811D816801B5
:10B9C000CC0CDD1C9601200F311F220F331F220FDC
:10B9D000331F220F331F2F543A4EF901849180FFF9
:10B9E00038C0F601E00FF11FEE0FFF1FEE0FFF1F33
:10B9F000EE0FFF1FE554FA4E659175918591949174
:10BA000069877A878B879C87F901249124FD08C078
:10BA10000E94EED569877A878B879C87BF8201C099
:10BA2000AF82B601600F711F660F771F660F771F19
:10BA3000660F771F65557A4E45E050E0C7010E94BA
:10BA4000B4E1CE010E941F5CCE010E949C5C0C817F
:10BA50001D810F5F1F4F0C831D83C8010E9402656B
:10BA60008111ABCF81E00E94A5A9DF91CF911F91F9
:10BA70000F91FF90EF90DF90CF90BF90AF900C941C
:10BA80008DA9CF92DF92EF92FF92CF93DF93EC01DB
:10BA9000C984DA84EB84FC8481E0C816D104E10413
:10BAA000F10449F0CE01DF91CF91FF90EF90DF904C
:10BAB000CF900C94647ACE010E94C25C82E08F83A6
:10BAC000C986DA86EB86FC8680E0DF91CF91FF9015
:10BAD000EF90DF90CF9008958091203E9091213E8D
:10BAE0008F3E924111F08AE508958091623E9091D7
:10BAF000633E8F3E9241B9F78091F2389091F338CE
:10BB00008F3E924181F78091183C9091193C8F3E75
:10BB1000924149F780911A3C90911B3C8F3E924193
:10BB200011F780911E3E90911F3E8F3E9241D9F6B3
:10BB30008091A9418111D7CF0895FC01178289E630
:10BB40000895CF93DF93DC0114968D919C91159706
:10BB5000FC01EE0FFF1FE80FF91FEE0FFF1FEE0FA6
:10BB6000FF1FEE0FFF1FE754FA4EC591D491488195
:10BB700050E060E070E019964D935D936D937C9377
:10BB80001C9782E017968C9380E0DF91CF91089507
:10BB9000CF93DF93DC0114968D919C911597FC0156
:10BBA000EE0FFF1FE80FF91FEE0FFF1FEE0FFF1F35
:10BBB000EE0FFF1FE754FA4EC591D4914881598189
:10BBC00060E070E019964D935D936D937C931C97A4
:10BBD00082E017968C9380E0DF91CF910895CF9308
:10BBE000DF93DC0114968D919C911597FC01EE0F6B
:10BBF000FF1FE80FF91FEE0FFF1FEE0FFF1FEE0FE5
:10BC0000FF1FE754FA4EC591D491488159816A814A
:10BC10007B8119964D935D936D937C931C9782E085
:10BC200017968C9380E0DF91CF910895CF93DF93A7
:10BC3000DC0114968D919C911597FC01EE0FFF1F6E
:10BC4000E80FF91FEE0FFF1FEE0FFF1FEE0FFF1F94
:10BC5000E754FA4EC591D491488159816A817B811C
:10BC600019964D935D936D937C931C9783E0179683
:10BC70008C9380E0DF91CF910895CF93DF93DC0127
:10BC800014968D919C911597FC01EE0FFF1FE80F04
:10BC9000F91FEE0FFF1FEE0FFF1FEE0FFF1FE75400
:10BCA000FA4EC591D491488159816A817B81199658
:10BCB0004D935D936D937C931C97FC01EE0FFF1FDA
:10BCC000E80FF91FEE0FFF1FEE0FFF1FEE0FFF1F14
:10BCD000EE54FA4E8591949118968C93189784E0BF
:10BCE00017968C9380E0DF91CF91089588E60895B0
:10BCF00080E00895FC0124813581F901EE0FFF1FDA
:10BD0000E20FF31FEE0FFF1FEE0FFF1FEE0FFF1FDF
:10BD1000E754FA4EA591B491FC0181858C9380E0A3
:10BD20000895FC0124813581F901EE0FFF1FE20F18
:10BD3000F31FEE0FFF1FEE0FFF1FEE0FFF1FE75465
:10BD4000FA4EA591B491FC01818592858D939C93C7
:10BD500080E00895CF93DF93FC0124813581F901C0
:10BD6000EE0FFF1FE20FF31FEE0FFF1FEE0FFF1F7F
:10BD7000EE0FFF1FE754FA4EC591D491FC01818567
:10BD80009285A385B48588839983AA83BB8380E049
:10BD9000DF91CF910895FC014185528563857485BB
:10BDA0004230510561057105A0F484819581FC0143
:10BDB000EE0FFF1FE80FF91FEE0FFF1FEE0FFF1F23
:10BDC000EE0FFF1FE754FA4EA591B4914C9380E01B
:10BDD00008958EE60895FC0141855285638574853A
:10BDE0004330510561057105A0F484819581FC0102
:10BDF000EE0FFF1FE80FF91FEE0FFF1FEE0FFF1FE3
:10BE0000EE0FFF1FE754FA4EA591B4914C9380E0DA
:10BE100008958EE60895FC014185528563857485F9
:10BE20004430510561057105A0F484819581FC01C0
:10BE3000EE0FFF1FE80FF91FEE0FFF1FEE0FFF1FA2
:10BE4000EE0FFF1FE754FA4EA591B4914C9380E09A
:10BE500008958EE60895CF93DF93DC0114968D91BB
:10BE60009C911597FC01EE0FFF1FE80FF91FEE0FD5
:10BE7000FF1FEE0FFF1FEE0FFF1FE754FA4EC59195
:10BE8000D49119964D915D916D917C911C97488349
:10BE900059836A837B8383E017968C9380E0DF91DC
:10BEA000CF910895CF93DF93DC0114968D919C91EF
:10BEB0001597FC01EE0FFF1FE80FF91FEE0FFF1F94
:10BEC000EE0FFF1FEE0FFF1FE754FA4EC591D491FE
:10BED00019964D915D916D917C911C974883598382
:10BEE0006A837B83FC01EE0FFF1FE80FF91FEE0F43
:10BEF000FF1FEE0FFF1FEE0FFF1FEE54FA4E85914E
:10BF0000949118968C93189784E017968C9380E000
:10BF1000DF91CF9108951F93CF93DF93EC01809130
:10BF2000783E8823D1F01DE10A80DB81C02D209767
:10BF300011F480E013C08F818F3FD9F3811104C0C9
:10BF4000CE010E94495C06C0CE010E941F5CCE015A
:10BF50000E949C5C115041F7ECCF85E6DF91CF91B8
:10BF60001F910895CF93DF93EC01BC018FEF90E216
:10BF70000E94EDE1892B41F0BE0182E091E20E9436
:10BF8000EDE121E0892B09F420E0822FDF91CF91B0
:10BF9000089541E02091F4383091F5382817390799
:10BFA00009F040E0842F08950F931F93CF93DF9300
:10BFB000CDB7DEB72997CDBFDEBF8B0144E050E09F
:10BFC000BC01CE0101960E940DE246E050E0B801AE
:10BFD000CE0101960E94FDE10E94FF641816190629
:10BFE0000CF03FC07981AA81BB811C810D812BEAB5
:10BFF00035E140E050E0F9016491671327C03196C4
:10C00000E491E11103C0A11121C029C0EA131EC0AF
:10C01000F9013296E491E11103C0B11117C01FC0BC
:10C02000EB1314C0F9013396E491E11103C011112F
:10C030000DC015C0E1130AC0F9013496E491E11175
:10C0400003C0011103C00BC0E01749F04F5F5F4F01
:10C05000285E3F4F4817590709F0CDCF02C0CA01EB
:10C0600002C08FEF9FEF2996CDBFDEBFDF91CF914A
:10C070001F910F910895CF93DF93FC012189222313
:10C0800071F1EC016196BE0186E091E20E94EDE162
:10C09000892B39F1BE018FEF90E20E94EDE1892BEF
:10C0A00011F1BE0189E091E20E94EDE1892BD9F006
:10C0B000BE018DEE90E20E94EDE1892BB1F0BE0150
:10C0C0008CE091E20E94EDE1892B79F0BE0188EECF
:10C0D00091E20E94EDE1892B51F485E009C080E0F6
:10C0E00007C082E005C083E003C084E001C081E0B6
:10C0F000DF91CF910895FC018FEF87831482158221
:10C1000011861286138614861086118A1586178A60
:10C11000108EA081B181109711F416820DC0179670
:10C120008C911797873029F416968C918F5F8683B0
:10C1300003C016968C918683CF010895EF92FF92EB
:10C140000F931F93CF93DF93EC010C811D810E940D
:10C15000FF64081719070CF06FC00C811D81CE0118
:10C160000E947B600C831D837E0181E1E80EF11C3F
:10C17000B801660F771F600F711F660F771F660F7C
:10C18000771F660F771F65557A4EC7010E9495E1AC
:10C190008E01035F1F4F2C813D81B901660F771F10
:10C1A000620F731F660F771F660F771F660F771F6B
:10C1B00069557A4EC8010E9495E18D85882311F159
:10C1C0008C819D81FC01EE0FFF1FE80FF91FEE0F20
:10C1D000FF1FEE0FFF1FEE0FFF1FEF54FA4EE4910B
:10C1E000E2FF02C01D8610C0F80101900020E9F7AF
:10C1F000BF01601B710B605F7F4F6C0F7D1FC7011C
:10C200000E94F6E18C819D81FC01EE0FFF1FE80F7B
:10C21000F91FEE0FFF1FEE0FFF1FEE0FFF1FEB5476
:10C22000FA4E25913491CE01F901DF91CF911F9102
:10C230000F91FF90EF901994DF91CF911F910F9183
:10C24000FF90EF9008958F929F92AF92BF92CF92FE
:10C25000DF92EF92FF920F931F93CF93DF9300D063
:10C260001F92CDB7DEB76C015C0181E1A80EB11C55
:10C2700087E0F601878367EAE62E65E1F62E00E0A7
:10C2800010E01DC0B701CE0101960E9495E1BE01EC
:10C290006F5F7F4FC5010E94EDE1892B59F4460184
:10C2A000F9E18F0E911CF601058F168FC4010E94D3
:10C2B0009E6064010F5F1F4FF8E1EF0EF11CC80193
:10C2C0000E9402658111DECF2496CDBFDEBFDF91D3
:10C2D000CF911F910F91FF90EF90DF90CF90BF9083
:10C2E000AF909F908F900895CF93DF9310921C3C56
:10C2F00010921D3C21E0FC013081311101C020E091
:10C30000AFEDB8E3E8EFF8E33FEFA083B1837996B0
:10C310005B96ED93FC935C975D961D921C925E97E5
:10C32000EF016397288322961882219738832A96F3
:10C33000188259964CE3E831F40739F71092013C22
:10C340001092023C1092F8381092F938FC012081CA
:10C35000222369F01092FE3827E02093FF38BC01B9
:10C3600089E099E30E94F6E181E199E302C088EF58
:10C3700098E3DF91CF910895EF92FF920F931F936F
:10C38000CF93DF938AE091E20E947461EC018FEE1B
:10C3900092E18093203E9093213E8093623E909361
:10C3A000633E8093F2389093F3388093183C9093D7
:10C3B000193C80931A3C90931B3C80931E3E9093B3
:10C3C0001F3E81E00E94284F1C821D82CE010E94E8
:10C3D000608220916A3E30916B3E40916C3E50915C
:10C3E0006D3E69857A858B859C850E94D1D39F7728
:10C3F0002CEA35EC47E257E30E947DD7181624F467
:10C40000CE010E94C25C58C00E9492A91C821D826B
:10C4100080E090E08E010F5E1F4F42E0E42E54E07A
:10C42000F52E44C06C817D81CB01880F991FFC01E2
:10C43000E60FF71FEE0FFF1FEE0FFF1FEE0FFF1FA0
:10C44000EF54FA4EE491E0FF2CC0680F791F660F9D
:10C45000771F660F771F660F771F65557A4E45E089
:10C4600050E0C8010E94B4E1CE010E9460828C813C
:10C470009D81FC01EE0FFF1FE80FF91FEE0FFF1F5C
:10C48000EE0FFF1FEE0FFF1FEF54FA4EE491E4FF93
:10C4900002C0FF8201C0EF82CE010E941F5C6C814E
:10C4A0007D816F5F7F4F6C837D83CB010E9402652E
:10C4B0008111B8CF0E94A5A960E171E287E493E2FF
:10C4C0000E94D45F8093F4389093F53864E171E270
:10C4D00087E493E20E94D45F8093F6389093F73814
:10C4E000DF91CF911F910F91FF90EF900895EF9200
:10C4F000FF920F931F93CF93DF938C0120911C3CED
:10C5000030911D3CEB0109900020E9F72197C61BF3
:10C51000D70BAE01420F531F41305240D8F4F901FE
:10C52000E25EF34C7F01AE014F5F5F4FCF010E948F
:10C53000CEE140911C3C50911D3C4F5F5F4F4C0F32
:10C540005D1F40931C3C50931D3CF801E78AF08E20
:10C5500080E001C08DE0DF91CF911F910F91FF909E
:10C56000EF900895CF93DF932EE1C1E1D9E33F81AE
:10C570003F3F59F00A80DB81C02D209719F480E0FD
:10C5800090E010C0215099F7FACFBC0187E493E204
:10C590000E94D45F8C839D83019689F3CE010E9413
:10C5A0009E60CE01DF91CF910895EF92FF920F939D
:10C5B0001F93CF93DF938B012EE1C1E1D9E33F813C
:10C5C0003F3F59F00A80DB81C02D209719F480E0AD
:10C5D00090E01DC0215099F7FACF7E0121E1E20ED3
:10C5E000F11C45E050E0BC01C7010E940DE2B8011A
:10C5F000CE010E9477628111EACFB70187E493E20E
:10C600000E94D45F8C839D8385E08F83CE01DF9170
:10C61000CF911F910F91FF90EF9008952091783E58
:10C62000213021F420915641213029F4BC018DEEB6
:10C6300090E20C94D56280E090E008959091783E6D
:10C64000913019F4642F0C940D810C94D5C0CF93C4
:10C65000DF93EC0180916B3481110BC00E9410D2EA
:10C66000482F50E060E070E049875A876B877C87ED
:10C670000AC00E941EC9482F50E060E070E0498760
:10C680005A876B877C8782E08F8380E0DF91CF9130
:10C6900008950F931F93CF93DF93CDB7DEB7C058A4
:10C6A000D109CDBFDEBFDC011996EC918FEF8E0F63
:10C6B000863030F088E491E20E940E638EE629C055
:10C6C000E093663481E080936734F0E0EE0FFF1F63
:10C6D000EE58FA4E659174914FE450E08AE591E48A
:10C6E0000E94B4E19F938F9389E394E19F938F938A
:10C6F0008E010F5F1F4F1F930F930E946BE3C801C2
:10C700000E940E630F900F900F900F900F900F905C
:10C7100080E0C058DF4FCDBFDEBFDF91CF911F91CA
:10C720000F9108950F931F93CF93DF93EC0181EE48
:10C7300096E30E94D84A882329F009851A858B85BB
:10C740009C8511C023E333E34BEC51E469857A8582
:10C750008B859C850E941FD88B01AB01BC0149874A
:10C760005A876B877C872C813D81F901EE0FFF1F73
:10C77000E20FF31FEE0FFF1FEE0FFF1FEE0FFF1F65
:10C78000E754FA4EA591B491A801BC014D935D9375
:10C790006D937C931397F901EE0FFF1FE20FF31FC8
:10C7A000EE0FFF1FEE0FFF1FEE0FFF1FEE54FA4EAE
:10C7B00085919491888784E08F8380E0DF91CF9189
:10C7C0001F910F91089563E475E10C94B8C16FE176
:10C7D00075E10C94B8C163EE74E10C94B8C16FEAD2
:10C7E00074E10C94B8C162E674E10C94B8C11F9373
:10C7F000CF93DF93EC0110E08881882311F18AE068
:10C8000091E20E94746145E050E0BE0182E299E34A
:10C810000E940DE262E279E387E493E20E94D45F32
:10C82000809315399093163981E199E30E949E60B7
:10C8300042E063E080E00E941E631F5F26961D3188
:10C84000D9F684E0DF91CF911F910895CF93DF93C4
:10C85000CDB7DEB7EC97CDBFDEBF8CE3E8E1F0E209
:10C86000DE01119601900D928A95E1F7CE010196B5
:10C870000E94F763EC96CDBFDEBFDF91CF910895A4
:10C88000CF93DF93CDB7DEB7AA97CDBFDEBF8AE2E5
:10C89000E4E5F0E2DE01119601900D928A95E1F750
:10C8A000CE0101960E94F763AA96CDBFDEBFDF914D
:10C8B000CF910895CF93DF93CDB7DEB76E97CDBFFD
:10C8C000DEBF8EE1EEE7F0E2DE01119601900D92FF
:10C8D0008A95E1F7CE0101960E94F7636E96CDBF6F
:10C8E000DEBFDF91CF910895CF93DF93EC0143E753
:10C8F00059E763E770E0498B5A8B6B8B7C8B0E9406
:10C90000236142E063E080E00E941E63CE010E944A
:10C910005A64CE010E94406420E731E340E0298B55
:10C920003A8B4B8BCE010E94236142E063E080E0B2
:10C930000E941E63CE01DF91CF910C942664FC010E
:10C9400081859285A385B48583309105A105B105C4
:10C95000A0F480936A34892B8A2B8B2B39F064E006
:10C9600070E080E00E94F7C680E0089568E070E023
:10C9700080E00E94F7C680E008958EE60895FC01ED
:10C9800081859285A385B48582309105A105B10585
:10C99000A0F480936934892B8A2B8B2B39F060E1CA
:10C9A00070E080E00E94F7C680E0089560E270E0E9
:10C9B00080E00E94F7C680E008958EE60895FC01AD
:10C9C00081859285A385B48582309105A105B10545
:10C9D000A0F480936834892B8A2B8B2B39F060E488
:10C9E00070E080E00E94F7C680E0089560E870E0A3
:10C9F00080E00E94F7C680E008958EE6089583E9FE
:10CA000091E0089521E08A34914008F020E0822FDF
:10CA100008959C012656314081E02932310508F005
:10CA200080E0089521E08736914008F020E0822FD1
:10CA30000895CF92DF92EF92FF92CF93DF93EC01B4
:10CA4000C984DA84EB84FC84A7019601C701B6018E
:10CA50000E9440D981113CC0E894F7F82FEF3FEFD6
:10CA60004FE75FE7C701B6010E9440D981110AC0B4
:10CA70002FEF3FEF4FE75FE7C701B6010E947AD57E
:10CA8000181634F18C819D81FC01EE0FFF1FE80F19
:10CA9000F91FEE0FFF1FEE0FFF1FEE0FFF1FEF54EA
:10CAA000FA4EE491E3FF14C081EE96E30E94D84A67
:10CAB00081110EC025E832E441E25DE369857A85A3
:10CAC0008B859C850E941FD869877A878B879C8776
:10CAD000DF91CF91FF90EF90DF90CF9008958091FC
:10CAE0006734882349F0109267346091663480E09F
:10CAF0000E94FFC680E0089583E00895CF93DF93FE
:10CB0000E0919A3EF0919B3E04C0E0939A3EF093F0
:10CB10009B3EEF018191982F9D7F9032B1F3893038
:10CB2000A1F34FE750E0BE018EE990E40E940DE2D0
:10CB30001092963E1092973E1092983E1092993E17
:10CB40006881611105C08091783E81116FC039C044
:10CB5000613221F4DF91CF910C94CF55653221F4ED
:10CB6000DF91CF910C94D3556E3721F4DF91CF91A3
:10CB70000C94D7556F3379F4FE0101900020E9F74A
:10CB80003197EC1BFD0B329780F02196C0939A3EB3
:10CB9000D0939B3E4BC06B3741F481E08093783E4D
:10CBA000CE01DF91CF910C94427E70E088E791E254
:10CBB0000E94E2E1892B59F01092783ECE010E944A
:10CBC000C7BE6EE970E4DF91CF910C942FC08091C5
:10CBD000783E811109C0CE010E949B706EE970E41D
:10CBE000DF91CF910C942FC08AE091E20E94746192
:10CBF000EC0127E633E640E0298B3A8B4B8B6091C2
:10CC00009A3E70919B3E0E94776285E08F8380916F
:10CC10009A3E90919B3E0E949B7042E060E00E9491
:10CC20001E6380E0DF91CF910C94E7ABDF91CF9151
:10CC30000895FF920F931F93CF93DF931F921F923C
:10CC4000CDB7DEB7F82EE4E6FEE32CEB32E0DF01F1
:10CC5000C9011D920197E9F72FEE32E1208331835C
:10CC600020931E4130931F4103E313E32CED33E483
:10CC700000936A3E10936B3E20936C3E30936D3E62
:10CC80000CEE11E528E73FE300936E3E10936F3EF4
:10CC90002093703E3093713E81E08093723E83E03A
:10CCA0008093793E8F2D4A8369830E940FC76981E3
:10CCB000862F0E941AC74A81842F0E9425C7F092AE
:10CCC0006534F09263340F900F90DF91CF911F91F4
:10CCD0000F91FF900895CF93DF931F921F92CDB7CE
:10CCE000DEB780E6F82E01E010E00E942279823063
:10CCF000E1F30E9429798230C1F30E94B74A86305D
:10CD000009F0D9C00E94F2C480907F3E9090803E8E
:10CD1000A090813EB090823E86169706A806B9067E
:10CD200020F70E94F2C46C597F4F8F4F9F4F609342
:10CD30007F3E7093803E8093813E9093823E0E941E
:10CD40009878D3CF0E94ADBD882329F08CEC0E9447
:10CD5000014F823051F20E942856823031F20E94F7
:10CD6000FC9E823011F20E946C5D8093AA41811179
:10CD70002EC08091643E9091653E8F3E924109F0B5
:10CD8000AAC080911E4190911F418F3E924109F0AF
:10CD9000A2C097C00E94F6828093AA41811117C059
:10CDA0000E941CB48093AA41811111C00E94667038
:10CDB0008093AA4181110BC00E941EC68093AA4194
:10CDC000811105C00E9414B5823031F48ECF0E94CB
:10CDD000014F8230B9F789CF0E9419AC823009F433
:10CDE00084CF0E946BAD823009F47FCF0E9427AEC2
:10CDF000823009F47ACF09831A836CE97EE3CE018D
:10CE000001960E9434C780939A3E90939B3E8F3F39
:10CE10002FEF920739F483E10E94EA4E823009F441
:10CE200064CF04C0892B11F00E947E650E945B8D47
:10CE3000823009F45ACF0E949B6B823009F455CF9F
:10CE40000E945A6E823009F450CF0E9441708230A5
:10CE500009F449CF0E94864C823009F444CF0E94E5
:10CE6000AB838430F0F53FCF8091793E843038F445
:10CE700084E08093793E0E94D3550E9497A983E075
:10CE800090E089839A836CE97EE3CE0101960E944B
:10CE900034C780939A3E90939B3E8F3F2FEF92072B
:10CEA00021F482E10E94EA4E1ECF892B09F41BCFA8
:10CEB0000E947E6518CF0E94B74A823009F44BCF9A
:10CEC00041CF1092AA410E94B44E8093AA41882378
:10CED00009F460CF7CCFF092AA4180E60E94014F16
:10CEE00078CF8091E4299091E5290E9484D0682F21
:10CEF00070E080E090E00E941CD620E030E048E442
:10CF000051E40E947DD787FFEECE0E946F6582308C
:10CF100009F0AACFE8CE80916534809363340895F8
:10CF2000809363340895809364340895CF93C82F19
:10CF300080919323882379F040E050E0BA018C2F50
:10CF40000E947950EC2FFF27E7FDF095EA54F94C49
:10CF500081E080830AC06C2F89EA9AE50E94FD4B2C
:10CF6000AB01BC018C2F0E9479504091BA235091A3
:10CF7000BB236091BC237091BD238C2F0E943F592D
:10CF800081E699E6809394239093952382E0CF9154
:10CF90000895CF92DF92EF92FF920F931F93CF935A
:10CFA000DF93CDB7DEB7E097CDBFDEBF98E17E015E
:10CFB000A9E1EA0EF11CF701A92F1192AA95E9F750
:10CFC000FE0131966F0111929A95E9F7F60194E00E
:10CFD0008902E00DF11D1124408F518F628F738FF4
:10CFE00080E090E0A0E8BFE380839183A283B383D5
:10CFF00000931E3710931F3720932037309321372B
:10D000000E942E840E94D755B601C7010E94A153E9
:10D010008093AA41811101C082E0E096CDBFDEBFBE
:10D02000DF91CF911F910F91FF90EF90DF90CF9004
:10D0300008950F931F93E0918D23FF27E7FDF0954F
:10D04000E557FB4C9381913099F400919E23109108
:10D050009F232091A0233091A1234091A62350919A
:10D06000A7236091A8237091A9230E94C9671DC0BE
:10D07000E0918E23FF27E7FDF095E557FB4C938168
:10D08000913099F400919E2310919F232091A02329
:10D090003091A1234091A6235091A7236091A8230A
:10D0A0007091A92370580E94C9678FE598E6809314
:10D0B00094239093952382E01F910F9108950F93ED
:10D0C0001F93CF93C82F85E3C802F0011124E957BD
:10D0D000FA4C40815181628173818C2F0E943F59AB
:10D0E00000919E2310919F232091A0233091A12392
:10D0F00040919A2350919B2360919C2370919D2392
:10D100008C2F0E94C9678EEE98E6809394239093AB
:10D11000952382E0CF911F910F9108950F931F9354
:10D1200000919E2310919F232091A0233091A12351
:10D130004091AA235091AB236091AC237091AD2311
:10D140000E94C96786E997E680939423909395237C
:10D1500082E01F910F9108950E942E848091B32345
:10D160000E94E24F8091B2230E94284F8091B42305
:10D170000E942C4F8091B5230E948D538091B6233D
:10D180009091B723A091B823B091B92380931E3713
:10D1900090931F37A0932037B093213764E081EE3E
:10D1A00096E30E94F54A0E9484561092B23680E0BF
:10D1B0000895CF93C82F4091BA235091BB2360911B
:10D1C000BC237091BD230E943F598C2F0E94AC68F4
:10D1D00080E00E94E7AB80EFCF9108950F931F93FB
:10D1E000E0918D23FF27E7FDF095E557FB4C9381F8
:10D1F000913039F089ED98E68093942390939523AC
:10D2000018C00091A2231091A3232091A423309150
:10D21000A5234091A6235091A7236091A823709144
:10D22000A9230E94C9678EE898E68093942390937F
:10D23000952382E01F910F910895FF920F931F9302
:10D24000CF93DF93CDB7DEB7C058D109CDBFDEBFD6
:10D25000F82E8AE091E20E9474618EEFF81205C008
:10D260008DE791E20E940E6319C08F2D0E9419571D
:10D270001F928F932FE63BE33F932F938E010F5F17
:10D280001F4F1F930F930E946BE3C8010E940E6310
:10D290000F900F900F900F900F900F9042E062E070
:10D2A00080EF0E941E638F2D0E94AC6880EFC058F3
:10D2B000DF4FCDBFDEBFDF91CF911F910F91FF9068
:10D2C00008954F925F926F927F929F92AF92BF921A
:10D2D000CF92DF92EF92FF920F931F93CF93DF9342
:10D2E0008F3F09F045C02CEA35EC47E257E36091E7
:10D2F000193870911A3880911B3890911C380E940F
:10D300007DD718160CF469C12CEA35EC47E257E3D7
:10D3100060911138709112388091133890911438BF
:10D320000E947DD718160CF45DC12CEA35EC47E25B
:10D3300057E36091153870911638809117389091A5
:10D3400018380E947DD718160CF455C12CEA35EC1C
:10D3500047E257E360911D3870911E3880911F3865
:10D36000909120380E947DD718160CF43FC171C1EE
:10D370008230A1F52CEA35EC47E257E36091113891
:10D380007091123880911338909114380E947DD793
:10D3900018160CF427C12CEA35EC47E257E36091EC
:10D3A00015387091163880911738909118380E946E
:10D3B0007DD718160CF41FC12CEA35EC47E257E371
:10D3C00060911D3870911E3880911F3890912038DF
:10D3D0000E947DD718160CF409C131C18823D9F2F7
:10D3E000813051F32CC17E018DEEE80EF11CF70166
:10D3F00080819181A281B381BC01CD019F772CEA0C
:10D4000035EC47E257E30E947AD587FD46C06E01AE
:10D41000F1EFCF0ED11CF601408051806280738005
:10D4200020E030E0A901C301B2010E947AD587FD56
:10D4300034C0FE01EF52FF4F208131814281538180
:10D44000349760817181828193810E94D1D39B0145
:10D45000AC015F77C301B2010E94D2D32B013C0122
:10D460009F772CEA35EC47E257E30E947AD587FD97
:10D4700014C0AB2CAA0C8A2D0E94A7BD80938B23CD
:10D48000992493949A0C892D0E94A7BD80938C2394
:10D4900020918B23822780FD02C08B2DDBC0B092B0
:10D4A0008A23F80180819181A281B381BF77809323
:10D4B0009E2390939F23A093A023B093A123F701D1
:10D4C00040815181628173817F774093A223509381
:10D4D000A3236093A4237093A52320FF2DC0A092C3
:10D4E0008D2390928E2377FA709477F870944092FF
:10D4F0009A2350929B2360929C2370929D23F60165
:10D5000080819181A281B3818093A6239093A723E8
:10D51000A093A823B093A923CB50DF4F8881998192
:10D52000AA81BB818093AA239093AB23A093AC23C1
:10D53000B093AD238A2D2AC090928D23A0928E2382
:10D5400040929A2350929B2360929C2370929D2339
:10D55000F60180819181A281B381B0588093A62386
:10D560009093A723A093A823B093A923CB50DF4F78
:10D5700088819981AA81BB81B0588093AA23909316
:10D58000AB23A093AC23B093AD23892D0E94A7BDFC
:10D590008D7F813039F081E699E6809394239093D2
:10D5A000952369C080918E230E94A7BD811103C07D
:10D5B0008FEF80938E238B2D0E9434596093BA2372
:10D5C0007093BB238093BC239093BD2389E198E69D
:10D5D00080939423909395234EC082E090E032E0B4
:10D5E000B32E0DC080E090E0B12C09C083E090E044
:10D5F00023E0B22E04C081E090E0BB24B394FC0190
:10D60000EA54F94C108225E3289FE001299FD00DB0
:10D610001124C255DB4C8E0107511F4FF801808148
:10D620009181A281B381BC01CD019F772CEA35ECB9
:10D6300047E257E30E947AD587FFD5CE2ECF81E00F
:10D640008093B5368CEA98E6809394239093952343
:10D6500012C08EEFDF91CF911F910F91FF90EF904D
:10D66000DF90CF90BF90AF909F907F906F905F9032
:10D670004F900C941D6982E0DF91CF911F910F9123
:10D68000FF90EF90DF90CF90BF90AF909F907F90F2
:10D690006F905F904F900895CF93DF93CFEDD6E3D7
:10D6A000888199810E94D84A8093B2238881998188
:10D6B0000E94D34A8093B323888199810E94E24AD1
:10D6C0008093B423888199810E94E74A8093B5238F
:10D6D000888199810E94EE4A6093B6237093B723A4
:10D6E0008093B8239093B92381E00E94284F81E072
:10D6F0000E942C4F80E00E94E24F81E00E948D53F7
:10D7000081E0809393238FEF80938A2381E699E6CB
:10D71000809394239093952383E08093B236109264
:10D72000B53680E0DF91CF9108950E944C6B109246
:10D73000932380E008958091B236833059F40E949B
:10D74000EC4A813049F0E0919423F0919523809147
:10D750008A23199483E0089582E0089586EB9BE67E
:10D760008093CF239093D02382E008952F923F920D
:10D770004F925F926F927F928F929F92AF92BF92E1
:10D78000CF92DF92EF92FF920F931F93CF93DF938D
:10D79000CDB7DEB7CA54D109CDBFDEBF98E19E0137
:10D7A000275E3F4F29AB3AABD901E92F1D92EA958D
:10D7B000E9F7285131091901D9011D929A95E9F724
:10D7C00024E08202F00111242B96EEAFFFAF2B97DD
:10D7D000E20DF31D80E090E0A0E8BFE38083918339
:10D7E000A283B383C090C723D090C823E090C923FD
:10D7F000F090CA234090C3235090C4236090C52367
:10D800007090C6238090BF239090C023A090C12326
:10D81000B090C223A5019401C301B2010E947AD540
:10D8200018165CF080E090E0A0E8BFE329968CAF8A
:10D830009DAFAEAFBFAF29970AC080E090E0A0E8EF
:10D84000BFEB29968CAF9DAFAEAFBFAF2997A301B9
:10D850009201C501B4010E94D1D30E94E9D59B0178
:10D8600077FF04C022273327261B370BB9018827EF
:10D8700077FD8095982F0E941CD625966CAF7DAFC2
:10D880008EAF9FAF2597C0921E37D0921F37E09280
:10D890002037F09221370E942E840E94D75520E035
:10D8A00030E040E050E425966CAD7DAD8EAD9FAD8F
:10D8B00025970E947DD718166CF08091CB2390910C
:10D8C000CC23A091CD23B091CE238BAF9CAFADAF35
:10D8D000BEAFDBC02AE037ED43E25CE325966CADDA
:10D8E0007DAD8EAD9FAD25970E947DD718162CF784
:10D8F00009E110E08AE0882E87ED982E83E2A82EB9
:10D900008CE3B82E412C512C32012B96AEADBFAD1D
:10D910002B97A20DB31D58962196AEAFBFAF21979E
:10D920004BAA5CAA6DAA7EAA8FAA98AEA9AEBAAE7F
:10D9300029962CAD3DAD4EAD5FAD29976FA978AD61
:10D9400089AD9AAD0E941FD89B01AC016091C323A1
:10D950007091C4238091C5239091C6230E94D2D395
:10D960002196EEADFFAD219760837183828393830F
:10D97000C0921E37D0921F37E0922037F0922137A5
:10D98000B101CE0149960E94A1538093AA41811111
:10D99000AAC020E030E040E85FE36BA97CA98DA934
:10D9A0009EA90E94D2D36BAB7CAB8DAB9EAB20E02B
:10D9B00030E048EC51E40E9481D59B01AC0160E06D
:10D9C00070E080E291E40E9482D82B013C018091BA
:10D9D000CB239091CC23A091CD23B091CE238BAFBC
:10D9E0009CAFADAFBEAFC090C723D090C823E0902E
:10D9F000C923F090CA23A7019601BC01CD010E9462
:10DA0000D1D34B015C0120E030E040E251E4C3019E
:10DA1000B2010E9481D59B01AC01C501B4010E94F5
:10DA20001FD89B01AC01C701B6010E94D2D36B0184
:10DA30007C012BA93CA94DA95EA9CA01B9010E948C
:10DA4000D2D320E030E048EC51E40E9481D59B0124
:10DA5000AC016FA978AD89AD9AAD0E94D2D36FABFE
:10DA600078AF89AF9AAF9B01AC0125966CAD7DADC7
:10DA70008EAD9FAD25970E947DD7181634F40150C6
:10DA800011090115110509F053CF8BAD9CADADAD5A
:10DA9000BEAD80931E3790931F37A0932037B0936D
:10DAA00021372B96EEADFFAD2B97E20DF31D809144
:10DAB000BF239091C023A091C123B091C223808F36
:10DAC000918FA28FB38FB101CE0149960E94A153CD
:10DAD0008093AA41811107C08AE89DE68093CF23F5
:10DAE0009093D02382E0C65BDF4FCDBFDEBFDF91D6
:10DAF000CF911F910F91FF90EF90DF90CF90BF904B
:10DB0000AF909F908F907F906F905F904F903F90DD
:10DB10002F900895CF93DF931F92CDB7DEB78983FF
:10DB20000E942E844091D9235091DA236091DB2307
:10DB30007091DC2389810E943F598091D6230E94F5
:10DB4000E24F8091D5230E94284F8091D7230E94D5
:10DB50002C4F8091D8230E948D538091D123909196
:10DB6000D223A091D323B091D42380931E379093D6
:10DB70001F37A0932037B093213764E081EE96E3FE
:10DB80000E94F54A0E9484561092B23689EA91E2C8
:10DB90000E9415E380E00F90DF91CF9108950F93DD
:10DBA0001F93CF93C82F0FED16E3F8018081918169
:10DBB0000E94D84A8093D523F801808191810E94E8
:10DBC000D34A8093D623F801808191810E94E24A52
:10DBD0008093D723F801808191810E94E74A809346
:10DBE000D823F801808191810E94EE4A6093D1236D
:10DBF0007093D2238093D3239093D4238C2F0E94AD
:10DC000034596093D9237093DA238093DB23909364
:10DC1000DC2381E00E94284F80E00E942C4F80E0AE
:10DC20000E94E24F81E00E948D5340E050E060E2AC
:10DC300071E44093C7235093C8236093C923709322
:10DC4000CA2385E3C89FF0011124E958FA4C4081AA
:10DC50005181628173814093CB235093CC23609395
:10DC6000CD237093CE236C2F89EA9AE50E94EA4B6C
:10DC70006093C3237093C4238093C5239093C623DA
:10DC80000E94085A6093BF237093C0238093C123DE
:10DC90009093C223C093BE238EEA9BE68093CF234A
:10DCA0009093D02384E08093B23680E0CF911F918F
:10DCB0000F9108958091B236843059F40E94EC4A55
:10DCC000813049F0E091CF23F091D0238091BE23A1
:10DCD000199483E0089582E00895E091DF23F0E055
:10DCE000E557FB4C8381882341F088E89EE68093CA
:10DCF000DD239093DE2382E008956CE274E284E1F8
:10DD000094E20E94A1538093AA41882371F308955D
:10DD10001F93CF93DF93E091DF23F0E0E557FB4CB7
:10DD200081E09381913009F080E08093BC36CDEBA7
:10DD3000D6E310E0812F0E941C98AB01BC01812F1B
:10DD40000E947950612F8091DF369091E0360E94D9
:10DD5000EA4B69937993899399931F5F163051F732
:10DD600083EB91E20E94427E84EF9EE68093DD2366
:10DD70009093DE2382E0DF91CF911F9108951F934E
:10DD8000CF93DF930E942E848091E02380938B3485
:10DD9000E091DF23F0E08091E123E557FB4C83879E
:10DDA0000E94C4BDC4EED3E210E04991599169913B
:10DDB0007991812F0E943F591F5F1630B1F78091F2
:10DDC000E3230E94E24F8091E2230E942C4F64E003
:10DDD00081EE96E30E94F54A0E9484561092B23674
:10DDE000DF91CF911F9108950E94BF6E80E008954A
:10DDF0000F931F93CF93DF93CDB7DEB7C058D109F0
:10DE0000CDBFDEBF182F8AE091E20E9474611E3FF1
:10DE100029F480EC91E20E940E6319C0812F0E94C8
:10DE200019571F928F938DE99BE39F938F938E01D8
:10DE30000F5F1F4F1F930F930E946BE3C8010E9457
:10DE40000E630F900F900F900F900F900F9042E085
:10DE500062E08AEF0E941E630E94BF6E8AEFC05884
:10DE6000DF4FCDBFDEBFDF91CF911F910F9108959E
:10DE7000FF920F931F93CF93DF931092BC3682E0F3
:10DE80008093B23604EE13E2C7E8D5E3F12C8F2D70
:10DE90000E943459F80161937193819391938F019A
:10DEA000488159816A817B818F2D0E943F596F2D56
:10DEB0008091DF369091E0360E94EA4BF801648B46
:10DEC000758B868B978BF394E596F6E0FF12DFCF88
:10DED00064E174E28CEF93E20E94F5C12AE43CE035
:10DEE00042E85EE30E947AD587FF03C08EEF0E946E
:10DEF000F86EC8E0D4E213E0699179918991999123
:10DF00002C893D894E895F890E94D1D39F772CEA65
:10DF100035EC47E257E30E947DD718161CF4812F99
:10DF20000E94F86E1F5F163039F784E08093DF237C
:10DF300080919A348093E12381E080939A34809198
:10DF40008B348093E02310928B340E94C4BD809167
:10DF5000DF369091E0360E94D34A8093E32380918C
:10DF6000DF369091E0360E94E24A8093E22380E01F
:10DF70000E942C4F80E00E94E24F80E00E94F6AFAA
:10DF80008DE69EE68093DD239093DE2382E0DF9191
:10DF9000CF911F910F91FF9008950F931F93CF93EF
:10DFA000DF938C01EB0180912A37882399F08091CF
:10DFB0001E3790911F37A0912037B0912137BC01B7
:10DFC000CD019F772CEA35EC47E257E30E947AD5E2
:10DFD00087FD4FC088819981AA81BB81BC01CD0199
:10DFE0009F772CEA35EC47E257E30E947DD718165D
:10DFF000F4F48C819D81AE81BF81BC01CD019F77FE
:10E000002CEA35EC47E257E30E947DD718167CF4E2
:10E0100088859985AA85BB85BC01CD019F772CEAAF
:10E0200035EC47E257E30E947DD7181624F188E1CA
:10E03000F801A4E1B4E201900D928A95E1F788E13C
:10E04000FE01ACE2B4E201900D928A95E1F788E11D
:10E05000EDEBF6E3DF011D928A95E9F782E080930C
:10E06000BC3688E39FE68093DD239093DE2380E037
:10E0700003C08EE801C086E8DF91CF911F910F9118
:10E0800008958091B236823021F08091BC36823082
:10E0900049F40E94EC4A813039F0E091DD23F0919F
:10E0A000DE23199483E0089582E00895E0E2F1E42C
:10E0B00080E2DF011D928A95E9F78FEE92E180936D
:10E0C0003E4190933F4180839183089580913E41EA
:10E0D00090913F418F3E924111F08CE508958091DF
:10E0E0002041909121418F3E9241B9F780E00895FF
:10E0F000CF93DF93C82FCB01BA010E94CED827E07F
:10E10000C29FE0011124C05EDE4B0E94E9D56D8301
:10E110007E838F839887DF91CF91089597E0899FC1
:10E12000F0011124E05EFE4B658176818781908548
:10E130000E941CD608952F923F924F925F926F9249
:10E140007F928F929F92AF92BF92CF92DF92EF9287
:10E15000FF920F931F93CF93DF93CDB7DEB727972F
:10E16000CDBFDEBF8C011B828091B136823009F4B5
:10E1700040C7D801BC90B11069C780E06E01B3E020
:10E18000CB0ED11C3DC0F6018081811108C0B72C97
:10E19000D7011C926E01B3E0CB0ED11C54C788325C
:10E1A00039F4B72CF7011082FFEFCF1ADF0A4BC703
:10E1B0008B33B9F3A82EB12CC5010E9469E1892BDC
:10E1C00039F4B5018AEE91E20E94E2E1892B51F027
:10E1D00047018FEF881A980AC5010E948DE1D70187
:10E1E0008C937401BFEFCB1ADB0AF7018081811198
:10E1F000CACFB72CD8018C916E01B3E0CB0ED11CE5
:10E20000F8011CC08E32E1F090E0C0970A97A0F0B0
:10E210008181803391F4228130E0205331092A300A
:10E22000310558F4DF01119611968C9111978D9359
:10E230008111FACF808102C0818131968111E2CFB4
:10E24000F601A080A11007C068C0D6011196AC905D
:10E25000BFEFCB1ADB0A76018A2C912CC4010E94F5
:10E260007DE1892B91F7EBE7AE122FC0D601119615
:10E270008C9190E00E9485E18437910531F5F6019B
:10E28000828190E00E9485E189369105F1F4D60102
:10E2900013968C9190E00E9485E184369105A9F453
:10E2A000BE016F5F7F4FC60105960E94E5DD0E94AB
:10E2B000EED56093963E7093973E8093983E9093F0
:10E2C000993EF601A0808A2C912CC4010E9485E120
:10E2D0008D369105A1F4D60111968C9190E00E94A3
:10E2E00085E18337910559F4F601828190E00E941F
:10E2F00085E18736910519F4F601339602C0FE01D7
:10E300003396AA2061F08A2DD701893209F41C9234
:10E3100011968C918111F9CF02C0FE0133968FE2E4
:10E32000B81609F468C68081882319F0CF010E94CD
:10E33000CA5580E1E0E4F1E4DF011D928A95E9F736
:10E340008BE5EAE0F8E3DF01982F1D929A95E9F753
:10E35000EFEAF7E3DF011D928A95E9F781EE96E394
:10E360000E94D04A8093B037812C912C80E8A82E4F
:10E370008FE3B82E5524539492E0492E24E0322E98
:10E3800023C4C701B6010E94EED5862F90E08F35D9
:10E39000910508F034C6FC01EC50FF4F0C94C5DD2C
:10E3A0001092B03750920B38809141418F5F80932B
:10E3B00041410AC45092B03750920B38809141418C
:10E3C0008F5F8093414100C44092B03750920B3828
:10E3D000809141418F5F80934141F6C383E08093F8
:10E3E000B03750920B38809141418F5F809341410B
:10E3F000EBC38DE08093AF3750920A38E5C388E0D5
:10E40000B2C01092DF3750923A38809142418F5F0C
:10E4100080934241D9C35092DF3750923A3880916D
:10E4200042418F5F80934241CFC34092DF37509289
:10E430003A38809142418F5F80934241C5C3109228
:10E44000E03750923B38809145418F5F8093454142
:10E45000BBC35092E03750923B38809145418F5F6B
:10E4600080934541B1C3C701B6010E9439D96C837D
:10E470007D838E839F8320E030E040E251E4C7013A
:10E48000B6010E941FD86B017C0120E030E040E221
:10E4900051E46C817D818E819F810E941FD89B01F8
:10E4A000AC01C701B6010E94D1D30E94EED5623003
:10E4B00001F128F4662341F0613089F0A0C5633092
:10E4C000E9F0643001F19BC5B5E0B093AF375092ED
:10E4D0000A38809140418F5F8093404175C33092EC
:10E4E000AF3760930A38809140418F5F80934041FD
:10E4F0006BC35092AF3750920A3866C34092AF3721
:10E5000050920A3861C383E08093AF3750920A3843
:10E510005BC3C701B6010E9439D96C837D838E83AA
:10E520009F8320E030E040E251E4C701B6010E9441
:10E530001FD86B017C0120E030E040E251E46C81A7
:10E540007D818E819F810E941FD89B01AC01C701F4
:10E55000B6010E94D1D30E94EED5662319F0613036
:10E5600061F04DC587E08093AF3750920A388091B3
:10E5700040418F5F8093404127C3E6E0E093AF378F
:10E5800060930A38809140418F5F809340411CC363
:10E59000C701B6010E9439D96C837D838E839F8326
:10E5A00020E030E040E251E4C701B6010E941FD8EC
:10E5B0006B017C0120E030E040E251E46C817D8120
:10E5C0008E819F810E941FD89B01AC01C701B601BB
:10E5D0000E94D1D30E94EED5623009F010C58EE0C2
:10E5E0008093AF3750920A38EFC25092E237509280
:10E5F0003D38EAC25092E13750923C38809149410F
:10E600008F5F80934941E0C24092E13750923C389D
:10E61000809149418F5F80934941D6C283E016C003
:10E620003092E13750923C38809149418F5F80931E
:10E630004941CAC2F5E0F093E13750923C388091ED
:10E6400049418F5F80934941BFC286E08093E137A3
:10E6500050923C38809149418F5F80934941B4C2C8
:10E66000C701B6010E9439D96C837D838E839F8355
:10E6700020E030E040E251E4C701B6010E941FD81B
:10E680006B017C0120E030E040E251E46C817D814F
:10E690008E819F810E941FD89B01AC01C701B601EA
:10E6A0000E94D1D30E94EED5662319F0613059F053
:10E6B000A6C41092E43750923F3880914A418F5F50
:10E6C00080934A4181C26093E43760933F388091E0
:10E6D0004A418F5F80934A4177C24092E43750921B
:10E6E0003F3880914A418F5F80934A416DC230929A
:10E6F000B03750920B38809141418F5F80934141F8
:10E7000063C2C701B6010E9439D96C837D838E83B1
:10E710009F8320E030E040E251E4C701B6010E944F
:10E720001FD86B017C0120E030E040E251E46C81B5
:10E730007D818E819F810E941FD89B01AC01C70102
:10E74000B6010E94D1D30E94EED5662319F0613044
:10E7500059F055C41092E5375092403880914341AA
:10E760008F5F8093434130C21092E6376093413807
:10E77000809143418F5F8093434126C2C701B60118
:10E780000E9439D96C837D838E839F8320E030E0A3
:10E7900040E251E4C701B6010E941FD86B017C0121
:10E7A00020E030E040E251E46C817D818E819F81E8
:10E7B0000E941FD89B01AC01C701B6010E94D1D3B2
:10E7C0000E94EED5662319F0613059F018C45092BA
:10E7D000E53750924038809143418F5F80934341A9
:10E7E000F3C16093E63760934138809143418F5F76
:10E7F00080934341E9C1C701B6010E9439D96C83B6
:10E800007D838E839F8320E030E040E251E4C701A6
:10E81000B6010E941FD86B017C0120E030E040E28D
:10E8200051E46C817D818E819F810E941FD89B0164
:10E83000AC01C701B6010E94D1D30E94EED5613070
:10E8400089F028F06230A1F06330C1F0D8C399E0BC
:10E850009093AF3750920A38809140418F5F8093F8
:10E860004041B2C1AAE0A093AF3760930A38ACC16F
:10E87000BBE0B093AF3750920A38A6C1ECE0E0930A
:10E88000AF3750920A38A0C11092DA37509235381B
:10E89000809144418F5F8093444196C15092DA3712
:10E8A00050923538809144418F5F809344418CC1B0
:10E8B000C701B6010E94EED5862F90E08D339105F9
:10E8C00008F09BC3FC01ED5AFE4F0C94C5DD10927D
:10E8D000B13750920C3880914B418F5F80934B4100
:10E8E00073C15092B13750920C3880914B418F5F79
:10E8F00080934B4169C15092EC37509247388091D8
:10E900004D418F5F80934D415FC14092EC375092F3
:10E91000473880914D418F5F80934D4155C1109292
:10E92000EC375092473880914D418F5F80934D4135
:10E930004BC15092E9375092443846C15092EA3761
:10E940005092453880914E418F5F80934E413CC13B
:10E950005092EB375092463880914E418F5F8093B2
:10E960004E4132C11092EB375092463880914E4161
:10E970008F5F80934E4128C15092DD3750923838D6
:10E9800080914F418F5F80934F411EC11092DD37C0
:10E990005092383880914F418F5F80934F4114C11E
:10E9A0005092DB375092363880914F418F5F809381
:10E9B0004F410AC15092F5375092503880914F41E3
:10E9C0008F5F80934F4100C1C701B6010E9439D9C2
:10E9D0000E94EED56093E83750924338F5C0C0925C
:10E9E000CE37D092CF37E092D037F092D1378092A5
:10E9F000293890922A38A0922B38B0922C38E4C053
:10EA0000C092F637D092F737E092F837F092F937A4
:10EA10008092513890925238A0925338B092543824
:10EA2000D3C0C092ED37D092EE37E092EF37F0923C
:10EA3000F0378092483890924938A0924A38B09284
:10EA40004B38C2C0C092B637D092B737E092B837D1
:10EA5000F092B9378092113890921238A092133800
:10EA6000B0921438B1C0C092BA37D092BB37E0929E
:10EA7000BC37F092BD378092153890921638A0922C
:10EA80001738B0921838A0C0C092BE37D092BF37A6
:10EA9000E092C037F092C1378092193890921A38BC
:10EAA000A0921B38B0921C388FC0C092C237D0924F
:10EAB000C337E092C437F092C53780921D389092E8
:10EAC0001E38A0921F38B09220387EC0C092C63740
:10EAD000D092C737E092C837F092C9378092213878
:10EAE00090922238A0922338B09224386DC0C09200
:10EAF000CA37D092CB37E092CC37F092CD378092A4
:10EB0000253890922638A0922738B09228385CC0D9
:10EB1000C092FE37D092FF37E0920038F092013871
:10EB20008092593890925A38A0925B38B0925C38F3
:10EB30004BC0C0920238D0920338E0920438F09271
:10EB4000053880925D3890925E38A0925F38B0921E
:10EB500060383AC0C0920638D0920738E092083840
:10EB6000F09209388092613890926238A0926338AE
:10EB7000B092643829C0C092FA37D092FB37E09245
:10EB8000FC37F092FD378092553890925638A0921B
:10EB90005738B092583818C0C701B6010E94EED558
:10EBA0006093B2377093B3378093B4379093B5378F
:10EBB00081E090E0A0E0B0E080930D3890930E38B3
:10EBC000A0930F38B0931038D8012C90222009F46C
:10EBD00024C2822D90E00E9474E1892B09F42FC297
:10EBE0003801BFEF6B1A7B0AF8018181803349F449
:10EBF0008281883531F40E5F1F4FC12CD12C7601F4
:10EC000000C2BE016F5F7F4FC3010E94E5DD6B0153
:10EC10007C0109811A816016710609F0F2C111C2E6
:10EC20008091DA370E948D53182F01C010E0609157
:10EC3000293870912A3880912B3890912C380E9475
:10EC4000EED5662359F06091CE377091CF37809121
:10EC5000D0379091D1370E945C53182F60912D3896
:10EC600070912E3880912F38909130380E94EED5D7
:10EC7000662371F06091D2377091D3378091D43789
:10EC80009091D5370E94EED5862F0E943855182FC7
:10EC900060913138709132388091333890913438A6
:10ECA0000E94EED5662371F06091D6377091D73708
:10ECB0008091D8379091D9370E94EED5862F0E9447
:10ECC0007755182F609148387091493880914A38AB
:10ECD00090914B380E94EED5662359F06091ED3744
:10ECE0007091EE378091EF379091F0370E942AB003
:10ECF000182F60914C3870914D3880914E3890911A
:10ED00004F380E94EED5662371F06091F137709113
:10ED1000F2378091F3379091F4370E94EED5862F29
:10ED20000E94B655182F80914338882329F080918E
:10ED3000E8370E94F553182F80914438882329F032
:10ED40008091E9370E942954182F809147388823F1
:10ED500029F08091EC370E94F6AF182F809145384A
:10ED6000882329F08091EA370E945E54182F809101
:10ED70004638882329F08091EB370E949254182F4F
:10ED800080913638882329F08091DB370E940D5519
:10ED9000182F80913738882329F08091DC370E9422
:10EDA0004C55182F80915038882329F08091F537E1
:10EDB0000E948B55182F80913838882329F0809134
:10EDC000DD370E940555182F8091AF378D3029F01F
:10EDD00080913A388823A9F00FC06091F63770917E
:10EDE000F7378091F8379091F9370E9495538093C7
:10EDF000AA41882369F32FC18091DF370E94244FF5
:10EE0000182F80913B38882329F08091E0370E94A9
:10EE1000284F182F80913C38882329F08091E137C2
:10EE20000E94E24F182F80913F38882329F080916B
:10EE3000E4370E949153182F80914038882329F09D
:10EE40008091E5370E942C4F182F4091AF3750E04A
:10EE50004F30510508F0B6C0FA01E057FE4F0C9450
:10EE6000C5DD0E94DE52182FADC061E178E386EB6C
:10EE700097E30E94E952182FA5C00E941D53182F36
:10EE8000A1C061E178E386EB97E30E942853182F35
:10EE900099C00E944C6B182F95C061E178E386EB16
:10EEA00097E30E94A850182F8DC00E94956B182FD1
:10EEB00089C061E178E386EB97E30E94CD6F182F5C
:10EEC00081C06091F6377091F7378091F837909153
:10EED000F9370E94EED5862F21E138E346EB57E360
:10EEE0006091DE370E94304F182F6CC061E178E3EB
:10EEF00086EB97E30E942551182F64C00E94D851D9
:10EF0000182F60C00E943F52182F5CC00E9476529A
:10EF1000182F58C06091E23781EE96E30E946B4B48
:10EF20008091B037843038F48230D8F4882349F0A7
:10EF3000813079F047C0843009F044C08093E536D1
:10EF400041C061E178E386EB97E30E94AE52182F4F
:10EF500039C061E178E386EB97E30E94A153182F53
:10EF600031C0A0900638B0900738C0900838D090D3
:10EF70000938E0900238F09003380091043810917D
:10EF800005382091FE373091FF374091003850917D
:10EF900001388F938091FD378F938091FC378F9349
:10EFA0008091FB378F938091FA378F9361E178E3FB
:10EFB00086EB97E30E94BE85182F0F900F900F905D
:10EFC0000F900F9060E081EE96E30E946B4B809172
:10EFD0000C38813061F48091B137811104C00E94F6
:10EFE000B756812F38C00E94E856812F34C0812F38
:10EFF00032C08BEC30C083E02EC084E82CC083E8A4
:10F000002AC0822D90E0FC01E154F109EA31F105BA
:10F01000B0F7E156FE4F0C94C5DD1092AA41609105
:10F02000B2377091B3378091B4379091B5370E9461
:10F03000054B80913538882309F4F8CDF1CD85E66C
:10F040000AC086E608C0D8018C91DAC868018B2D09
:10F0500078017B2CA4C82796CDBFDEBFDF91CF916E
:10F060001F910F91FF90EF90DF90CF90BF90AF90E6
:10F070009F908F907F906F905F904F903F902F90D8
:10F080000895CF93DF93EC016EE970E40E947762FC
:10F090008093AA41811102C095E09F83DF91CF91B7
:10F0A0000895FC018789908D0C949B7083FF06C0A6
:10F0B000E0918334F091843490E2958382FF06C01E
:10F0C000E0918534F091863490E2958381FF06C00B
:10F0D000E0918734F091883490E2958380FF06C0F8
:10F0E000E0918934F0918A3480E28583089583FF2A
:10F0F00006C0E0918334F091843490E2968382FFDD
:10F1000006C0E0918534F091863490E2968381FFC9
:10F1100006C0E0918734F091883490E2968380FFB6
:10F1200006C0E0918934F0918A3480E286830895A4
:10F1300080917A3E811107C084E00E94567881E078
:10F1400080937A3E089584E00E94777810927A3E08
:10F150000895CF92DF92EF92FF920F931F93CF9378
:10F16000DF93C12C26E0D22EC0927334D092743437
:10F1700030EAE32E36E0F32EE0927534F0927634E6
:10F1800000E816E00093773410937834C0E6D6E0B8
:10F19000C0937934D0937A34C0927B34D0927C344B
:10F1A000C0937D34D0937E3400937F3410938034A9
:10F1B000E0928134F09282342DEC3CEC4CED50E442
:10F1C0000E947DD7C0928334D0928434E0928534FB
:10F1D000F092863418164CF4C0938734D093883458
:10F1E0000093893410938A3408C0009387341093B5
:10F1F0008834C0938934D0938A34DF91CF911F91A2
:10F200000F91FF90EF90DF90CF9008950E9424D34C
:10F2100060E070E080E091E40E94A9780C9443D310
:10F2200081E08093833E089520E093E088ED08B666
:10F2300018BE84BF909380002091820021FDFCCFF6
:10F2400008BEFFCF8091833E81110E94147983E034
:10F2500008958091843E882341F0F89461E089E725
:10F2600090E00E9426D382E0089583E00895CF9332
:10F27000DF93CDB7DEB7AD97CDBFDEBF21E2EDEEB8
:10F28000F1E2DE01119601900D922A95E1F722E05C
:10F290002093CA01DE019296E8E0F0E024912D93DC
:10F2A0003196EE30F105D1F72DE228A7E0E1F0E04C
:10F2B000E491EF7121E030E02C0F3D1F2E0F311D46
:10F2C000F901208129A7E2E1F0E0E491EF719E01CC
:10F2D0002E0F311DF90121812AA7E4E1F0E0E4912C
:10F2E000EF719E012E0F311DF90121812BA71CA664
:10F2F0001092CA0125E0FC012783BE016E5D7F4F9D
:10F300000E9477628093AA41AD96CDBFDEBFDF91A8
:10F31000CF91089581E08093843E80E00895CF935B
:10F32000DF93EC0120E030E040E051E469857A852C
:10F330008B859C850E947DD718166CF0CE010E94AB
:10F34000525F69857A858B859C850E94A9780E9489
:10F35000C4BD80E001C08DE6DF91CF9108956DE3DB
:10F360007CE30C94B8C16FE17CE30C94B8C162E01B
:10F370007CE30C94B8C164EE7BE30C94B8C160EDFF
:10F380007BE30C94B8C1CF93DF9383E897E49F931A
:10F390008F93C2E6DEE589818F9388818F930E94E7
:10F3A00090E28DE495E49F938F9389818F93888178
:10F3B0008F930E9490E285EC94E49F938F938981D0
:10F3C0008F9388818F930E9490E28BEF93E49F93B9
:10F3D0008F9389818F9388818F930E9490E20E94FE
:10F3E00097A98DB79EB740968DBF9EBF80E0DF91F5
:10F3F000CF910895CF93DF9386ED93E49F938F93FE
:10F40000C2E6DEE589818F9388818F930E9490E226
:10F4100088E692E49F938F9389818F9388818F935D
:10F420000E9490E28DED90E49F938F9389818F935A
:10F4300088818F930E9490E285EC94E49F938F9350
:10F4400089818F9388818F930E9490E28BEF93E460
:10F450009F938F9389818F9388818F930E9490E2ED
:10F460008DB79EB744968DBF9EBF80E0DF91CF9150
:10F470000895CF93DF938CEB90E49F938F93C2E634
:10F48000DEE589818F9388818F930E9490E28EE3DD
:10F490009DE39F938F9389818F9388818F930E949F
:10F4A00090E28BEF93E49F938F9389818F93888170
:10F4B0008F930E9490E28DB79EB70C968DBF9EBF32
:10F4C00080E0DF91CF910895CF93DF9386E19DE3B4
:10F4D0009F938F93C2E6DEE589818F9388818F9316
:10F4E0000E9490E285EA9CE39F938F9389818F939A
:10F4F00088818F930E9490E28BEF93E49F938F9388
:10F5000089818F9388818F930E9490E28DB79EB7F7
:10F510000C968DBF9EBF80E0DF91CF910895CF9371
:10F52000DF9382E89CE39F938F93C2E6DEE58981B7
:10F530008F9388818F930E9490E289E59CE39F934B
:10F540008F9389818F9388818F930E9490E28BEFB4
:10F5500093E49F938F9389818F9388818F930E94E7
:10F5600090E28DB79EB70C968DBF9EBF80E0DF9175
:10F57000CF9108953F924F925F926F927F928F92B8
:10F580009F92AF92BF92CF92DF92EF92FF920F9332
:10F590001F93CF93DF93CDB7DEB76497CDBFDEBFA8
:10F5A0006C018B014A0182E29CE2ABE7B0E08F8301
:10F5B0009887A987BA8782E29AE3A0E08E879F871F
:10F5C000A88B8CE29DE7A0E08B879C87AD8786E0C7
:10F5D000EEE0F2E2DE01119601900D928A95E1F7DC
:10F5E000DB01ED91FC918081811102C083E0AEC10D
:10F5F000C6010E947B60F801608071802301530185
:10F60000F9E0AF0EB11C72012FEF421A520AD70176
:10F610006C9170E0CE0107960E94E2E1892B41F4E3
:10F62000F801408251823701F2E26F0E711C0DC069
:10F63000D3018C918823D1F24A145B0411F48FE634
:10F6400085C1F80140825182DECF5201FFEF4F1A8F
:10F650005F0AD5016C9170E0CE010E960E94E2E146
:10F66000892BE9F0F80140825182D5011C9246E0D5
:10F6700050E0B7017601B1E1EB0EF11CC7010E9429
:10F680000DE2B70187E493E20E94D45F8B8B9C8BE1
:10F69000F60184839583019649F484E657C14614A4
:10F6A0005704D9F3D8014D925C92CFCFF801608016
:10F6B00071805301F9E0AF0EB11C2301D3013D90DD
:10F6C0003D01E32CF12CC7010E9469E1892B71F403
:10F6D000B701CE0101960E94E2E1892B39F46A1448
:10F6E0007B04D9F2F80160827182E7CFFEE63F1613
:10F6F00049F022E2321209C0D20111968C91823275
:10F7000009F053C0F6011782E9C0F0E3EF1AF108DF
:10F710002AE0E216F10418F08DE2381238C0EB89C5
:10F72000FC89EE0FFF1FAB89BC89EA0FFB1FEE0FB0
:10F73000FF1FEE0FFF1FEE0FFF1FEF54FA4EE49175
:10F74000E4FF17C0BE016F5E7F4FC2010E94E5DD7E
:10F75000F6016187728783879487D8014D905C900A
:10F7600089899A894816590609F4EBC084E0878391
:10F77000B5C0C2010E946AE0F60161877287838783
:10F78000948782E08783D8014D905C90A7C0BBE747
:10F790003B1270C087E0F6018783FFEF4F1A5F0AC4
:10F7A000D8014D925C9282E0D1C0B2016F5F7F4F71
:10F7B000F8016083718385E0D60117968C93B1E8D8
:10F7C0004B0E511C9B01FB01D9018C918C3571F4BE
:10F7D00011969C919232F1F49083D8012D913C9135
:10F7E00011972F5F3F4F2D933C9318C0823291F4B5
:10F7F0001082F801A081B181CD01019680839183AF
:10F80000FC0101900020E9F73197E81BF90B3397D1
:10F8100078F428C08083D8012D913C912F5F3F4F11
:10F82000D8012D933C933196E415F50569F68BC00C
:10F8300011962C9111972033A9F412962C91283708
:10F8400089F440E050E060E070E00E9456DFF6018D
:10F85000618772878387948783E08783D8014D907F
:10F860005C903CC0C6010E9477628093AA418823C5
:10F8700091F16CC0B4E73B120FC081E0F6018783C1
:10F8800081E090E0A0E0B0E081879287A387B48711
:10F89000D8014D905C9022C0B6E63B120BC081E0CF
:10F8A000F60187831186128613861486F80140803C
:10F8B000518014C0FBE53F12C2CE86E0D6011796F8
:10F8C0008C93B201C6010E9477628093AA41811194
:10F8D0003DC087E63BC0F80140805180BE01655FB6
:10F8E0007F4FC2010E9427E2FC01D8018D939C93B7
:10F8F000009709F4A4CE208120C0213210F02F37C8
:10F9000041F4CF010196D8018D939C932181FC0194
:10F9100014C02D3781F4F401808181508083D80197
:10F920008D919C911197FC013196ED93FC93DC0134
:10F9300011962C9102C02C3241F02111DECF80E0D3
:10F9400005C086E603C081E701C082E06496CDBFB2
:10F95000DEBFDF91CF911F910F91FF90EF90DF906D
:10F96000CF90BF90AF909F908F907F906F905F905F
:10F970004F903F9008952F923F924F925F926F92D7
:10F980007F928F929F92AF92BF92CF92DF92EF922F
:10F99000FF920F931F93CF93DF93CDB7DEB72897D6
:10F9A000CDBFDEBF8C016E837F831D8219821A82D8
:10F9B0001B821C82809153418F5F8093534183301F
:10F9C00008F045C17B01FB0101900020E9F7319768
:10F9D000E61BF70BE130F24008F03BC1FB01208150
:10F9E0006B01222309F448C051E040E0E2E29E2E80
:10F9F000F701223E99F48181803881F497012E5FCE
:10FA00003F4FF701828194E6980F923048F4F60157
:10FA10009082C60101966C01790126C0808101C0E7
:10FA20007901411118C041E0883209F040E05523C6
:10FA300021F08132C8F08F37B9F05601FFEFAF1ACD
:10FA4000BF0A90E048870E9485E1F6018083650146
:10FA500050E0488509C041E0893209F440E0F601F0
:10FA60008083C60101966C01C7010196F7012181CF
:10FA7000222311F07C01BCCFF60110821092AA4122
:10FA800027E6422E23E6522E612C32E0332E7724D5
:10FA900073944AE9C42E47E4D42E5CE9852E57E4DA
:10FAA000952E6AEAA62E67E4B62E7EEF272EAE01CB
:10FAB0004B5F5F4FBE016A5F7F4FC8010E94BA7AF9
:10FAC000843008F0C9C0833011F480E0C5C0F8016B
:10FAD00087818730A9F4E280F380AE014B5F5F4FEE
:10FAE000BE016A5F7F4FC7010E94BA7A833009F472
:10FAF00084C0F701E280F380E114F10471F77DC066
:10FB00008981882349F043E050E0BE016F5F7F4F59
:10FB1000C8010D960E940DE2F801848195810E9432
:10FB20000965882381F07801F1E1EF0EF11CC7012E
:10FB30000E94B25F882339F043E050E0B701CE0164
:10FB400001960E940DE2F801848195812091F6389A
:10FB50003091F7388217930709F427820E94C95F12
:10FB6000882309F44AC0F801E788F08CF701608126
:10FB70006B3729F4B701C8010E94BB7C3EC070E01E
:10FB800088E791E20E94E2E1892B41F180915141A5
:10FB9000811107C0BF92AF920E94F1E20F900F90C7
:10FBA00006C09F928F920E94F1E20F900F903092C8
:10FBB000783EC7010E94C7BE7092783EDF92CF9216
:10FBC0000E94F1E280E090E00E94746170925441E2
:10FBD000F801828193810F900F9035C0F801418A1E
:10FBE000528A638AC7010E949B706EE970E40E948A
:10FBF0002FC0F8018281938126C0F80187818F3F51
:10FC000019F4828193811FC0811104C0C8010E9430
:10FC1000495C10C08091B136823061F0C8010E9409
:10FC20001F5CC8010E949C5C05C0F80127812F3F22
:10FC300051F08C01F801828193810097B1F782B174
:10FC400093B100E010E0892B09F031CF3ECF82E77D
:10FC500003C08BE68093AA412896CDBFDEBFDF911B
:10FC6000CF911F910F91FF90EF90DF90CF90BF90B9
:10FC7000AF909F908F907F906F905F904F903F904C
:10FC80002F900895CF93DF93EC011092544110927E
:10FC900053418AE091E20E947461BE010E94BB7CE4
:10FCA00042E060E00E941E6381E0DF91CF910C94FE
:10FCB000E7AB2F923F924F925F926F927F928F921B
:10FCC0009F92AF92BF92CF92DF92EF92FF920F93EB
:10FCD0001F93CF93DF935C011B018A01060F171F4F
:10FCE000DC0116969C9080915441EB01219688236B
:10FCF00021F08CE2FB01808303C08BE7DB018C9356
:10FD000090E0412CFBE76F2EA5E07A2EB8E1CB2ED8
:10FD1000B2E2DB2E84E1E82E82E2F82E2CE2822E83
:10FD20003DE7532EF50187818E5F823008F4E5C0F0
:10FD3000992311F08882219680915141811113C03D
:10FD4000C50141969F938F93FF92EF92DF93CF93DC
:10FD50000E9442E3C80FD91F0F900F900F900F9091
:10FD60000F900F9012C0C50141969F938F93DF9221
:10FD7000CF92DF93CF930E9442E3C80FD91F0F9019
:10FD80000F900F900F900F900F90D50117968C91B8
:10FD9000811103C0EEE1F2E2A0C0823019F5D50175
:10FDA0001C968C911C978F931B968C911B978F930D
:10FDB0001A968C911A978F9319968C918F93A3E230
:10FDC000B2E2BF93AF93DF93CF930E9442E3C80F99
:10FDD000D91FD50117968C91EDB7FEB73896EDBFB8
:10FDE000FEBF84C0833019F5D5011C968C911C97F9
:10FDF0008F931B968C911B978F931A968C911A97C1
:10FE00008F9319968C918F93A7E2B2E2BF93AF9331
:10FE1000DF93CF930E9442E3C80FD91FD5011796F5
:10FE20008C91EDB7FEB73896EDBFFEBF5FC0853051
:10FE300059F4D50158968C9158978F9357968C9179
:10FE40008F93AFE2B2E209C08630C9F4F501808D2C
:10FE50008F9387898F93A4E3B2E2BF93AF93DF932D
:10FE6000CF930E9442E3C80FD91FD50117968C91FA
:10FE70000F900F900F900F900F900F9037C084301D
:10FE800091F4C5010E941965F5014185528563858C
:10FE900074852085CE010E94E9C3C80FD11DD5010C
:10FEA00017968C9123C0813009F5F50181859285E3
:10FEB000A385B485892B8A2B8B2B69F4E9E3F2E2C5
:10FEC000DE0186E001900D928A95E1F72596D50135
:10FED00017968C910BC0EFE3F2E2DE01872D0190C3
:10FEE0000D928A95E1F72496F5018781873021F4F8
:10FEF0006882219690E001C091E0C017D10718F008
:10FF00008FEF9FEF48C0D5011296AD90BC9013972C
:10FF1000A114B10441F0F50186812FEF240D841561
:10FF20002CF0482EFFCE9414A4F01EC0FE01D50183
:10FF3000CF010196EC01508216964C9016973FEF38
:10FF4000320F42161CF4232FFC01F2CF5D0191E029
:10FF5000E9CEFE012DE7CF010196EC0120834A9402
:10FF6000941414F4FC01F7CF80915441882329F0B4
:10FF7000109254418DE7888321968DE79AE0A0E0A6
:10FF800088839983AA8322960C171D0708F4B8CF9B
:10FF9000CE0182199309DF91CF911F910F91FF90AC
:10FFA000EF90DF90CF90BF90AF909F908F907F9019
:10FFB0006F905F904F903F902F90089540E052E0F7
:10FFC0006EE97EE30E94597E8EE99EE39F938F93B4
:10FFD0000E94DFE20F900F900895BF92CF92DF92C0
:10FFE000EF92FF920F931F93CF93DF93CDB7DEB7BE
:10FFF0006297CDBFDEBFB82E80915041882309F4AF
:020000021000EC
:10000000FFC08FE6B81214C08AE091E20E947461CA
:100010006EE970E480919A3E90919B3E0E94C9C324
:10002000BC018CE091E20E94D56201E119E332C08B
:100030008091B13601E119E3882361F1FF24FA943C
:10004000C8010E943B60882329F1823029F4809105
:100050005941811119C016C0843029F4809156414C
:10006000811112C00FC0853079F4809158418823E6
:1000700049F0F8014185528563857485452B462BEF
:10008000472B11F0F801F782F80102811381011565
:100090001105B1F6C090963ED090973EE090983E04
:1000A000F090993EC701B6010E941AD62CEA35ECB1
:1000B00047E257E30E947DD7181654F14EC0F8016D
:1000C000028113810115110519F581E70E941FA90D
:1000D0008091963E9091973EA091983EB091993E26
:1000E00089B99AB9ABB9BCB984E799E6A4E6B0E09E
:1000F00081BB92BBA3BBB4BB82E087B916B840E01A
:1001000052E06EE97EE388EF98E30E94597E78C062
:10011000F80187818F3F99F6C186D286E386F486FF
:1001200084E799E6A4E6B0E0818B928BA38BB48B35
:1001300082E087831682028113810FC0F801028159
:1001400013810115110549F440E052E06EE97EE3A8
:1001500088EF98E30E94597E53C0F80187818F3F52
:1001600069F780916B3481111AC080919D3E8F9305
:1001700080919C3E8F931F92BF9284E492E29F9362
:100180008F93CE0101967C01FF928F930E9442E3F0
:1001900010929C3E10929D3ECDBFDEBF13C00E94C8
:1001A0001EC91F928F931F92BF928CE492E29F937D
:1001B0008F93CE0101967C01FF928F930E9442E3C0
:1001C000CDBFDEBFB701C8010E947762F801168279
:1001D00086E0878386E690E0818B928B1282138281
:1001E00040E052E06EE97EE388EF98E30E94597E9A
:1001F0008EE99EE39F938F930E94DFE20F900F9012
:100200006296CDBFDEBFDF91CF911F910F91FF901E
:10021000EF90DF90CF90BF900895613019F0623079
:1002200029F0089588EF98E30C94DE7F0C94ED7F1D
:10023000FC0181859285A385B48586309105A10551
:10024000B10580F58093504110925541109256416E
:100250001092574110925841109259410097A105B0
:10026000B10511F121E02093554181309105A1059F
:10027000B105D1F02093564182309105A105B10519
:1002800099F02093574183309105A105B10561F0A4
:10029000209358410597A105B10531F420935941A8
:1002A00080E008958EE6089580E008956FE378E495
:1002B0000C94B8C168EE77E40C94B8C164EB77E4B1
:1002C0000C94B8C1BF92CF92DF92EF92FF920F933E
:1002D0001F93CF93DF93CDB7DEB76897CDBFDEBF57
:1002E0006B0128E1FC01DE01119601900D922A9527
:1002F000E1F782E7E82E85E3F82E8E010F5F1F4FAE
:10030000B12CF7018081823029F4F801108211822A
:10031000128213828091E45C8B1114C02091F75CEF
:100320003091F85C4091F95C5091FA5CF801608181
:100330007181828193810E941FD8F601608371834D
:10034000828393838091035D8B1114C02091165D8D
:100350003091175D4091185D5091195DF8016081F1
:100360007181828193810E941FD8F6016483758315
:10037000868397838091225D8B1114C02091355D17
:100380003091365D4091375D5091385DF801608164
:100390007181828193810E941FD8F60160877187E5
:1003A000828793878091415D8B1114C02091545DA9
:1003B0003091555D4091565D5091575DF8016081D7
:1003C0007181828193810E941FD8F60164877587AD
:1003D00086879787B394F5E3EF0EF11C0C5F1F4FF0
:1003E00086E0B8128ECF6896CDBFDEBFDF91CF9189
:1003F0001F910F91FF90EF90DF90CF90BF900895E5
:10040000F8940E9406790E9457820E9443D30E946A
:10041000DCC50E9461B40E9456700E94C4BD0E9457
:1004200000A740E060E080E00E9419660E94BC6185
:100430000E9445820E940A840E9418500E943BD369
:100440008091A20084608093A2008091A2008260CB
:100450008093A2008091A20081608093A200789492
:100460000E9497A90E94C6BE0E946B66FDCFE82F2E
:10047000F0E0EE0FFF1FE559F74B659174914FE4E3
:1004800050E08AE591E40C94B4E18091773E8230AB
:1004900041F440E060E081E00E94196680E00E9443
:1004A00093670C9417CA682F81E00C94B9C6109218
:1004B000AB411092AC411092AD411092AE41089503
:1004C000CF93DF93EC018C819D81880F991F880F5A
:1004D000991F2091AD413091AE41820F931F8093BF
:1004E000AF419093B04144E050E065EB71E40E946D
:1004F0003BD24091B5415091B6416091B741709166
:10050000B84149875A876B877C8780E0DF91CF911C
:1005100008950F931F93CF93DF93EC018091B23630
:10052000882339F089E0DF91CF911F910F910C94CE
:100530001FA949855A856B857C854093B1415093AD
:10054000B2416093B3417093B441CE010E94608286
:100550008093AA41811141C00091B1411091B241F3
:100560002091B3413091B44149855A856B857C8592
:10057000401751076207730739F10093B541109393
:10058000B6412093B7413093B8418C819D81880F4B
:10059000991F880F991F2091AD413091AE41820F74
:1005A000931F8093AF419093B04144E050E065EBDE
:1005B00071E40E94CCD23091B1412091B24190912E
:1005C000B3418091B44104C0342F252F962F872F3B
:1005D00039872A879B878C8780E0DF91CF911F9195
:1005E0000F9108950E94DCB980E008958091B9418F
:1005F0009091BA418F3E924111F08EE5089580911D
:10060000DF419091E0418F3E9241B9F78091E14105
:100610009091E2418F3E924181F780916A59909189
:100620006B598F3E924149F780916C5990916D5969
:100630008F3E924111F78091FF5A9091005B8F3E5F
:100640009241D9F680E0089594E0899FF001112449
:10065000E754FE4B4283538364837583089594E08B
:10066000899FF0011124E459F64A45AB56AB67ABBC
:1006700070AF08955F926F927F928F929F92AF9228
:10068000BF92CF92DF92EF92FF920F931F93CF937F
:10069000DF93CDB7DEB76097CDBFDEBFBE016F5F22
:1006A0007F4F81EA99E50E946281CE0101964C015B
:1006B00089E1A82E8AE5B82E99E2C92E9AE5D92EAD
:1006C00029E3E22E2AE5F22E09E51AE53BE7632E3F
:1006D0003DE5732E512CF40141915191619171913D
:1006E0004F01F50141935193619371935F01F601BD
:1006F00041935193619371936F01F701419351932A
:10070000619371937F01852D0E947870F801119299
:100710001192119211928F01F301108211821282B3
:1007200013825394F8E16F0E711C84E05812D3CFFA
:100730006096CDBFDEBFDF91CF911F910F91FF90EB
:10074000EF90DF90CF90BF90AF909F908F907F9071
:100750006F905F9008958091E34108951F93CF9328
:10076000DF938BE897E1E1EEF1E4DF019C011D925C
:1007700021503040E1F78FEE92E18093E141909378
:10078000E24180936A5990936B59CAEED1E4C093C9
:10079000E441D093E541C093E641D093E741C09353
:1007A000E841D093E94181E090E06EEA78E520E00D
:1007B00030E01CEB129FA001139F500D1124FA0191
:1007C000EF51FE4BD90111961A9F90011B9F300DDE
:1007D000112426513E4B2387348761877287BA01E3
:1007E00066517E4B9C0101968032910519F78CEB86
:1007F000829FF001839FF00D1124EF51FE4BC387C0
:10080000D4876187728780E28093E341DF91CF9143
:100810001F910895CF93DF93ECE6F9E585E991E028
:10082000DF01EC011D922197E9F7A9EBB1E488E221
:10083000ED0119928A95E9F78FEE92E18D939C93E1
:100840008093DF419093E041808391838093FF5AAE
:100850009093005BDF91CF910C94AE830E94278E22
:100860000E94AE8380E00C94BA4AE091E441F0919A
:10087000E541848581111BC0228133818081918172
:100880004CEBDF011D924A95E9F722833383808385
:10089000918381E084878091E34181508093E3419B
:1008A000828193818093E4419093E54105C08CE17E
:1008B0000E941FA9E0E0F0E0CF010895A6EEB1E4A8
:1008C000ED91FC911197858781E0878782E084878D
:1008D000828193818D939C9381E00E941EAD0C9444
:1008E00022B7EF92FF920F931F93CF93DF9300D025
:1008F0001F92CDB7DEB78C014B835C8369837A830B
:100900000E943584FC014B815C8169817A8100976A
:1009100061F48EE02496CDBFDEBFDF91CF911F91B1
:100920000F91FF90EF900C94014F83E0858782EF49
:1009300092E884839583068317838B017A0126E0EE
:10094000D8014D915D916D917D918D01CF018559BA
:100950009F4FDC014D935D936D937C931397D7016B
:100960004D915D916D917D917D01418B528B638B9A
:10097000748B215034962111E3CF83E02496CDBFB0
:10098000DEBFDF91CF911F910F91FF90EF900C94FC
:100990005E84CF92DF92EF92FF926B017C010E9406
:1009A0003584009739F48EE0FF90EF90DF90CF9080
:1009B0000C94014F2CE435E8FC0124833583E55683
:1009C000FF4FC082D182E282F38221E0FC012787BF
:1009D00082E00E945E8480E0FF90EF90DF90CF90F5
:1009E00008958091E8419091E941FC0124853EEF12
:1009F000320F323018F424E024870895243011F0A7
:100A000080E090E00895E091E841F091E941228191
:100A10003381808191814CEBDF011D924A95E9F78A
:100A20002283338380839183E091E841F091E9410F
:100A30000280F381E02DE093E841F093E941848561
:100A4000823011F483E084878091E3418F5F80934B
:100A5000E3418FEF0E941EAD81E04091E44150914F
:100A6000E5412091E8413091E9414217530709F0EF
:100A700080E00895BC016F5E7F4FDC011696ED911A
:100A8000FC91179785599F4F19950E9403858111F5
:100A90000E94845680E0089585569F4F20E034E2FE
:100AA00044E759E4FC0160817181828193810E9455
:100AB0001FD80E94EED50E941AD60E94E6B90E9465
:100AC000038581110E94845680E008958091E84159
:100AD0009091E941FC0124853EEF320F323018F449
:100AE00024E024870895243011F080E090E00895F8
:100AF000CF93DF93C091E841D091E9418C859EEF7F
:100B0000980F923018F484E08C8705C0843019F077
:100B100080E090E010C02097D9F3DE011296ED91AD
:100B2000FC9113978785882329F0EC17FD0711F0B6
:100B3000DF01F4CFCD01DF91CF910895CF93DF9303
:100B4000EC012A813B81888199814CEBFB01DE011C
:100B500001900D924A95E1F72A833B83888399831C
:100B6000DF91CF9108958FEE92E18093015B909396
:100B7000025B8093BE5B9093BF5B08952F923F9280
:100B80004F925F926F927F928F929F92AF92BF929D
:100B9000CF92DF92EF92FF920F931F93CF93DF9349
:100BA000CDB7DEB76A97CDBFDEBF4C011B0129016F
:100BB0003A01E986FA860B871C871A2D0B2DE8A8C7
:100BC000B9A8AAA82BA9298380912A37882399F04C
:100BD00080911E3790911F37A0912037B091213717
:100BE000BC01CD019F772CEA35EC47E257E30E9428
:100BF0007AD587FD11C78091553890915638A091CC
:100C00005738B0915838BC01CD019F7731E03D8312
:100C10002CEA35EC47E257E30E947DD7181614F012
:100C20001D8210C02DEC3CEC4CEC5DE36091FA377A
:100C30007091FB378091FC379091FD370E947AD5F7
:100C400087FDECC6F10180819181A281B381BC0155
:100C5000CD019F77F1E0FD872CEA35EC47E257E3C1
:100C60000E947DD718160CF01D86F10184819581B4
:100C7000A681B781BC01CD019F77F1E0F98B2CEA09
:100C800035EC47E257E30E947DD718160CF0198A1D
:100C9000F10180859185A285B385209159383091E5
:100CA0005A3840915B3850915C382E8B3F8B488F7F
:100CB000598F20915D3830915E3840915F38509166
:100CC00060382A8B3B8B4C8B5D8B40916138509107
:100CD00062386091633870916438F0902B37F1106E
:100CE00021C01092495B81E080934A5B82E080934F
:100CF0004B5B3D81332341F04D85411195C65989A8
:100D0000511192C68CE9C1C6CB01BA019F772CEA7A
:100D100035EC47E257E30E947DD718160CF089C6E0
:100D20008BE9B3C6BC01CD019F77A1E0AA8F2CEA65
:100D300035EC47E257E30E947DD718160CF01A8E67
:100D4000B1E0FB1216C01092495B82E080934A5BCF
:100D5000F0924B5BED81EE2339F0FD85F11164C615
:100D60002A8D222379F260C66A897B898C899D89C4
:100D7000CDCF32E0F31217C081E08093495BF0924F
:100D80004A5B10924B5B4D81442341F059895111CC
:100D90004BC68A8D882309F4B5CF46C66E897F89F4
:100DA000888D998DB3CFB101C4010E94094D9D81F9
:100DB000992309F451C02091E6363091E7364091ED
:100DC000E8365091E93660913B3770913C3780911D
:100DD0003D3790913E370E94D1D39F772CEA35EC76
:100DE00047E257E30E947AD587FF36C02091EA3662
:100DF0003091EB364091EC365091ED3660913F37B3
:100E00007091403780914137909142370E94D1D301
:100E10009F772CEA35EC47E257E30E947AD587FFAB
:100E20001BC02091EE363091EF364091F036509154
:100E3000F1366091433770914437809145379091F6
:100E400046370E94D1D39F772CEA35EC47E257E32F
:100E50000E947AD587FDE4C58CA98093E53681EEA2
:100E600096E30E94114B86E5E1EEF6E3A8E6BBE5CA
:100E700001900D928A95E1F788E1EBE3F7E3A4E0B6
:100E8000BBE501900D928A95E1F780912C37811195
:100E9000D5C523E333E34BEC51E46E2D7B2D8A2D36
:100EA00099810E941FD84B015C016093345B709361
:100EB000355B8093365B9093375B23E333E34BECF6
:100EC00051E4C301B2010E941FD860931C5B709370
:100ED0001D5B80931E5B90931F5B23E333E34BEC1E
:100EE00051E469857A858B859C850E941FD8609323
:100EF000205B7093215B8093225B9093235B23E3C1
:100F000033E34BEC51E4612F702FC6010E941FD8D0
:100F1000162F072F412F502FBC014093245B509375
:100F2000255B6093265B7093275B8091F6379091E9
:100F3000F737A091F837B091F937BC01CD019F7711
:100F40000E9457D60E94EED56093455B7093465B36
:100F50008093475B9093485BA091495BA98BB091CC
:100F60004A5BBA8BEB2FF0E0ED83FE837F01EE0C42
:100F7000FF1CEE0CFF1CF101EE0DFF1D8081918125
:100F8000A281B381BC01CD019F772CEA35EC47E209
:100F900057E30E947AD5D82EDD1CDD24DD1C39896B
:100FA000232F30E029833A838901000F111F000F9E
:100FB000111FF101E00FF11F80819181A281B381A6
:100FC000BC01CD019F772CEA35EC47E257E30E9444
:100FD0007AD5881F8827881F8D218093445B2CEA4F
:100FE00035EC47E257E3C501B4019F770E947DD7F6
:100FF00018160CF0F9C0F801EA51F94CD801A55CBB
:10100000B84C2D913D914D915C91608171818281AF
:1010100093810E94D1D36B017C01ED81FE81EE0FA3
:10102000FF1FEE0FFF1FEA51F94CAD81BE81AA0FE1
:10103000BB1FAA0FBB1FA55CB84C2D913D914D91D4
:101040005C9160817181828193810E94D1D3698793
:101050007A878B879C87A5019401C501B4010E9402
:101060001FD820E030E040E850E40E941FD86D8790
:101070007E878F87988BA7019601C701B6010E94D2
:101080001FD82B013C0129853A854B855C85CA0117
:10109000B9010E941FD89B01AC01C301B2010E949B
:1010A000D2D39B01AC016D857E858F8598890E9486
:1010B000D1D32B013C0120E030E0A9010E947DD773
:1010C0001816C4F4C301B2010E94F8D82B013C01E8
:1010D00029853A854B855C85C701B6010E948AD770
:1010E0009B01AC01C301B20190580E9481D52B0134
:1010F0003C0103C0412C512C32018091E5368330F4
:1011000021F477FA709477F8709420E030E0A90128
:10111000C501B4010E947AD587FF04C077FA7094A4
:1011200077F8709409811A81000F111F000F111FA9
:10113000A8014F5F544A5A01A301920169857A853B
:101140008B859C850E941FD89B01AC01C701B6010D
:101150000E94D1D320E030E040E05FE30E941FD83E
:10116000D5015B966D937D938D939C935E97AD8037
:10117000BE80AA0CBB1CAA0CBB1CF501EF5FF44A95
:101180004F01A3019201C701B6010E941FD89B0124
:10119000AC0169857A858B859C850E94D2D320E03D
:1011A00030E040E05FE30E941FD8D4015B966D936E
:1011B0007D938D939C935E97E0914B5BF0E0EE0FF7
:1011C000FF1FEE0FFF1FEF5FF44A138E148E158E74
:1011D000168EB091345BB987E091355BED87209036
:1011E000365B3090375B25C05701F701EF5FF44A5B
:1011F000838D948DA58DB68D9C01AD015058F8015D
:10120000EF5FF44A838D948DA58DB68DBC01CD0121
:1012100090580E948AD79B01AB01BC014093345B7C
:101220005093355B6093365B7093375B29873D87BE
:101230001C01D801AF5FB44A5B96CD90DD90ED9074
:10124000FC905E97E981FA81EE0FFF1FEE0FFF1F02
:10125000E359F44A13962D913D914D915C91169767
:1012600060817181828193810E94D1D3A70196010F
:101270000E94D1D369837A838B839C83D501AF5F2E
:10128000B44A5B964D905D906D907C905E97ED8139
:10129000FE81EE0FFF1FEE0FFF1FE359F44A139676
:1012A0002D913D914D915C91169760817181828164
:1012B00093810E94D1D3A30192010E94D1D36D8367
:1012C0007E838F8398879B01AC0169817A818B81B2
:1012D0009C810E948AD729853D85A1010E94D1D396
:1012E0004B015C01E894B7F820E030E040E85FE3B0
:1012F000C501B4010E947DD718160CF4C3C32AE0BF
:1013000037ED43EA5BE3C501B4010E947AD587FF5C
:1013100012C02AE037ED43E25CE369857D85C101B7
:101320000E941FD89B01AC01C501B4010E947DD76A
:1013300018160CF4A7C3A30192015058C701B601B7
:1013400090580E9445D44B015C0160932C5B7093D4
:101350002D5B80932E5B90932F5B80912B37813098
:1013600039F4412C512C30E8632E3FEB732E06C02C
:10137000412C512C20E8622E2FE3722E8091445B89
:101380008823D1F16091455B7091465B8091475B0A
:101390009091485B0E941AD66B017C012CEA35ECD7
:1013A00047E257E30E947AD587FD10C01091E536D9
:1013B0002BED3FE049EC50E4C701B6010E941FD875
:1013C0009B01AC01C12CD12C7601B9C081E090E029
:1013D000A0E0B0E08093455B9093465BA093475BB1
:1013E000B093485B1091E5362BED3FE049EC50E4BB
:1013F000C12CD12C7601A3C02D813E814F8158850F
:1014000069817A818B819C810E9445D469837A832A
:101410008B839C836093305B7093315B8093325BF2
:101420009093335BA50194010E94D1D36B017C01A1
:101430009F772CEA35EC47E257E30E947AD587FF85
:1014400018C01091E5366091455B7091465B8091C4
:10145000475B9091485B0E941AD62BED3FE049EC28
:1014600050E40E941FD89B01AC01C12CD12C760105
:1014700066C029813A814B815C81C501B4010E941B
:101480007DD71816F4F42BED3FE049EC50E4C3018E
:10149000B2010E941FD89B01AC0169817A818B81C6
:1014A0009C810E94D2D36093305B7093315B8093B8
:1014B000325B9093335BA50194010E94D1D36B0101
:1014C0007C011091E536133099F06091455B709185
:1014D000465B8091475B9091485B0E941AD62BED4A
:1014E0003FE049EC50E40E941FD89B01AC0127C0AB
:1014F0002BED3FE049EC50E4C301B2010E941FD83C
:101500009B01AC01C701B6010E94D1D37B018C01C4
:101510006091455B7091465B8091475B9091485B21
:101520000E941AD62BED3FE049EC50E40E941FD8F0
:101530009B01AC01C701D8016C017D010BC01230C9
:1015400049F4C301B2010E941FD8A70196010E946D
:10155000D2D30AC0C301B2010E941FD89B01AC01C3
:10156000C701B6010E94D1D37B01AB01BC014093FE
:10157000385B5093395B60933A5B70933B5B8C01B3
:1015800050904B5BA52DB0E0FD01EE0FFF1FEE0F5D
:10159000FF1FE359F44AAA0FBB1FAA0FBB1FAF5F7F
:1015A000B44A13962D913D914D915C9116976081AF
:1015B0007181828193810E94D1D34B015C01609340
:1015C0003C5B70933D5B80933E5B90933F5B9701E8
:1015D000A80169857D85C1010E941FD86B017C012E
:1015E0006093405B7093415B8093425B9093435B5D
:1015F000A50194010E948AD769837A838B839C8397
:101600006093285B7093295B80932A5B90932B5B9C
:1016100080912A37811117C0F0911E37FD834090C9
:101620001F37209120372E8B309121373A8F10921F
:101630001E3710921F37109220371092213781E009
:1016400080932A3712C020911E3730911F37409166
:1016500020375091213769817A818B819C810E944A
:1016600081D56D83472E8E8B9A8F598945E3549F80
:10167000F0011124ED58FA4C2081318142815381CF
:10168000C701B6010E9481D5662E072F182F792E2B
:101690002D81342D4E895A8D0E947AD587FF04C042
:1016A0006D80042D1E897A8C9A8985E3989FF001BC
:1016B0001124ED58FA4C2081318142815381C701B8
:1016C000B6010E9481D56B017C019B01AC01662DA6
:1016D000702F812F972D0E947DD7181624F06C2C27
:1016E0000D2D1E2D7F2C862D902FA12FB72D809391
:1016F0004C5B90934D5BA0934E5BB0934F5B20E0AF
:1017000030E0A901C501B4019F770E947DD718166A
:1017100084F5A5E35A9EF0011124ED58FA4C20817E
:10172000318142815381C501B4010E9481D54B01B1
:101730005C01E894B7F8A5019401662D702F812F04
:10174000972D0E947DD7181614F4A72C04C0682C7E
:10175000092D1A2DAB2C862D902FA12FBA2D8093F9
:101760004C5B90934D5BA0934E5BB0934F5BB62C5C
:1017700002C0B62CA72CC090B434D090B534E09001
:10178000B634F090B73420E030E040E850E4C701D0
:10179000B6010E941FD82B013C0129853D85A1017E
:1017A00069857D85C1010E94D2D3A70196010E945F
:1017B000D1D39B01AC01C301B2010E941FD80E948A
:1017C000F8D82B013C0120EC31EE44E65CE46B2DB3
:1017D000702F812F9A2D0E941FD820E030E44CE119
:1017E00056E40E9481D56B017C012091BD3430917B
:1017F000BE344091BF345091C03469817A818B816D
:101800009C810E9481D54B015C01A30192016981F9
:101810007A818B819C810E9481D587017601A50107
:1018200094010E94D1C20E9457D67B018C0120E016
:1018300030E040E85FE30E947DD718163CF4B70122
:10184000C8010E94E9D54B015C0108C0812C912C94
:1018500054018394E12CF12C00E81FE3C701D80167
:101860008093505B9093515BA093525BB093535B1A
:101870009701A80160914C5B70914D5B80914E5B2C
:1018800090914F5B0E9481D560939D5B70939E5BAE
:1018900080939F5B9093A05B8092545B9092555B8A
:1018A000A092565BB092575B9701A8016091385B9C
:1018B0007091395B80913A5B90913B5B0E9481D53E
:1018C0006093585B7093595B80935A5B90935B5B1A
:1018D0009701A80160913C5B70913D5B80913E5BFC
:1018E00090913F5B0E9481D560935C5B70935D5BE0
:1018F00080935E5B90935F5B80902C5B90902D5B00
:10190000A0902E5BB0902F5BC501B4010E94EED871
:10191000C090345BD090355BE090365BF090375BE5
:101920000091495B10E0000F111F000F111F0F5FA6
:10193000144AA70196010E941FD89B01AC01F8012F
:1019400063817481858196810E94D1D36093605BAD
:101950007093615B8093625B9093635BC501B4019C
:101960000E947ED59B01AC0100914A5B10E0000F04
:10197000111F000F111F0F5F144AC701B6010E940B
:101980001FD89B01AC01D80113966D917D918D916B
:101990009C9116970E94D1D36093645B7093655BB2
:1019A0008093665B9093675BA0914B5BB0E0FD0119
:1019B000EE0FFF1FEE0FFF1FE359F44AAA0FBB1FE4
:1019C000AA0FBB1FAF5FB44A13968D919D910D90E6
:1019D000BC91A02D80839183A283B3831092AA41EE
:1019E0008091285B9091295BA0912A5BB0912B5B41
:1019F000BC01CD019F772CEA35EC47E257E30E940A
:101A00007AD587FD0FC00E94775682E08093035BF2
:101A10000E946C4C80E039C08EE837C08EE935C03A
:101A20008FE933C089EC31C0B101C4010E94094D76
:101A3000C2C9B101C4010E94094D0ECA8E2D9B2D51
:101A4000AA2DB9818093345B9093355BA093365B6C
:101A5000B093375B40921C5B50921D5B60921E5BA3
:101A600070921F5B29853A854B855C852093205BAE
:101A70003093215B4093225B5093235B4C015D01CB
:101A8000C60148CA8BE98093AA416A96CDBFDEBFE2
:101A9000DF91CF911F910F91FF90EF90DF90CF904A
:101AA000BF90AF909F908F907F906F905F904F907E
:101AB0003F902F9008958F929F92AF92BF92CF92B6
:101AC000DF92EF92FF92CF93DF938091035B8823A5
:101AD00009F4B1C00E94AB83843010F482E0ACC042
:101AE0002091585B3091595B40915A5B50915B5B00
:101AF00060912C5B70912D5B80912E5B90912F5BA0
:101B00000E94D2D36B017C0160932C5B70932D5BA0
:101B100080932E5B90932F5B0E94EED88090345B75
:101B20009090355BA090365BB090375BC091495B7D
:101B3000D0E0CC0FDD1FCC0FDD1FC359D44AA50167
:101B400094010E941FD89B01AC016091605B709171
:101B5000615B8091625B9091635B0E94D2D36883EA
:101B600079838A839B83C701B6010E947ED59B013E
:101B7000AC01C0914A5BD0E0CC0FDD1FCC0FDD1F64
:101B8000C359D44AC501B4010E941FD89B01AC01BE
:101B90006091645B7091655B8091665B9091675B1F
:101BA0000E94D2D3688379838A839B83C0914B5BE5
:101BB000D0E0CC0FDD1FCC0FDD1FC359D44A2091DC
:101BC0005C5B30915D5B40915E5B50915F5B6881D7
:101BD00079818A819B810E94D2D3688379838A83A9
:101BE0009B8388E69BE50E943D9888E1EDE6FBE556
:101BF000A4E0BBE501900D928A95E1F78091545BDA
:101C00009091555BA091565BB091575B0197A109EC
